:100000000C9483140C941C890C94B4140C94B414A4
:100010000C94B4140C9407930C9482A70C94B4140D
:100020000C94B4140C94B4140C94B4140C94B41430
:100030000C94B4140C94B4140C94B4140C94B41420
:100040000C94B4140C94CC4F0C948A920C94B41469
:100050000C94B4140C94B4140C94B4140C94098738
:100060000C94B4140C94B5580C948B580C94B41490
:100070000C94B4140C94B4140C94B4140C94B414E0
:100080000C94CD470C94B4140C94B4140C94B41484
:100090000C9461580C9437580C94B4140C94B41408
:1000A0000C94B4140C94B4140C94B4140C94B414B0
:1000B0000C94B4140C944E8C0C94B4140C94B4148E
:1000C0000C94B4140C94B4140C94B4140C940D58F3
:1000D0000C94E3570C94B4140C94B9570C948F57A8
:1000E0000C94B414012204220B220E221122142299
:1000F0001B22222225222C2233223A229828C6288B
:10010000FD2834290F2A462A742AA22A602B602B44
:10011000602B602B602B602B602B602B602B602B87
:10012000602B602B602B602B602B602B602B602B77
:10013000602B602B602B602B602B602B602B602B67
:10014000602B602B602B6B29A229D929D02AFE2A8B
:100150002C2B922D982D9E2DA42DAA2DB02DB62D91
:10016000BC2DC22DC82DCE2DD42DE62DEC2DF22D7B
:100170000A2E102E162E1C2E222E282E2E2E342E17
:100180003A2E402E462E4C2E522E582E642E702E75
:10019000762E7C2E822E9A2EA02EA62EAC2EB22E3D
:1001A000B82EA82FAE2FB42FC62FCC2FD22FE42FCE
:1001B000EA2FF02FF62FFC2F02302C3032305C303B
:1001C000623068306E3086308C30923098302D310D
:1001D0002D312D312D312D312D312D312D31AE30AF
:1001E000B230B630BC30C030C430C830CC30D03083
:1001F000D430DA30F830FE300431882EBE2EC42ED2
:10020000CA2ED02ED62EDC2E74307A3080309E301E
:10021000A430AA300A311031163108300E30E22EE7
:10022000E82EEE2EF42EFA2E002FBA2FD82F6A2E9B
:10023000DA2DE02D8E2E942E1C31223128315E2EA7
:1002400038303E3044304A3050305630062F0C2F74
:10025000122F182F1E2F242F2A2F302F362F3C2FEE
:10026000422F482F4E2F542F5A2F602F662F6C2F5E
:10027000782F7E2F842F8A2F902F962F9C2FA22F9E
:10028000EC30E630E030F230C02FDE2FF82DFE2DBE
:10029000042E1430722F1A3020302630F837D5371C
:1002A000AE3715386C383438633852381D39003958
:1002B000D9386D393A393A395C3945392A402A40BA
:1002C00039402A4046405F407A40954049544C545A
:1002D0003B543F5445548354505454545A545E54E0
:1002E000625468546C547054835476547A547E54D7
:1002F000245A295A2E5A385A425ABB5A4C5A545ADE
:100300005C5A665A705A7A5A895A935ABB5A9D5AFD
:10031000A75AB15A985C9C5CA05CA45CA85CAC5CDD
:10032000B05CB45CB85CBC5CC05CEC5CF05CF75C82
:10033000045D115D245D375D505D695D875D9D5D88
:10034000B96DED6D226E426E776EDF6EEF6E1970D5
:10035000636F6D6FA16FD66FE46F1970AB6E7D8C9C
:10036000868C8E8CA28CB48CC68CD18CF2A109A206
:1003700020A237A24EA27CA293A2AAA2C1A2E0A26E
:10038000F8A20FA32EA344A365A2C7A6C1A6C7A621
:10039000C1A6C7A6C1A6C7A605A84CCDB2D44EB962
:1003A0003836A9020C50B9918688083CA6AAAA2A18
:1003B000BE000000803F0C9493A20C9462540C94F5
:1003C0001E2F0C94636F0C9425860C94A45C0C94E3
:1003D000FE850C94922D0C9428620C946C540C9411
:1003E00056300C94FC2F0C9404220C948F8A0C949D
:1003F0004A940C9419690C94282E0C943A8C0C9401
:10040000AA300C94998A0C9402860C9437860C942A
:1004100082A10C94A98A0C945DA00C9427830C945F
:10042000B48C0C94308C0C947CA00C943A2E0C94CC
:1004300022220C946F750C94878A0C946C610C9436
:10044000385A0C94E02D0C94A3890C94D0300C9461
:10045000B28B0C945E9C0C945C390C94C09F0C94F1
:100460002A2F0C9482BF0C9447750C94C0A10C9455
:10047000EF940C94838A0C94F0890C94D9A00C947A
:10048000AE370C94A68B0C94302F0C94182F0C9430
:10049000C49E0C94D18C0C94FD9E0C94C02F0C9493
:1004A00079A00C94DE2F0C949C9B0C9498300C94A7
:1004B00070960C944A300C9413750C94C4300C94C0
:1004C000BC5C0C9449690C949C2F0C9458950C942A
:1004D000CC2F0C9495400C9483540C947A400C943B
:1004E000E62D0C94AFA00C9444300C944F9F0C94C8
:1004F000AAA10C94545A0C94798A0C94978A0C945F
:1005000020300C94DD890C94AC9E0C94782F0C94C4
:10051000367E0C94DF530C94FE2D0C947CA20C942C
:1005200091A00C948B8A0C94722F0C945A9C0C946E
:100530001A770C9444850C94AE300C9450300C9483
:10054000B42F0C94BC2D0C94F22D0C94B48D0C94FF
:1005500076A00C94422F0C946C750C9439400C943A
:10056000AF9E0C946D390C94B89E0C9465A20C94BB
:10057000B6300C9420A20C9420940C947A540C94D1
:10058000978B0C945F400C9464950C94A38B0C9403
:1005900038300C9469A00C94358C0C94505D0C94FC
:1005A000898A0C94B6940C944E2F0C94EF6E0C9494
:1005B0000F2A0C94EC2D0C94B88D0C942F840C9471
:1005C000702E0C94208B0C94D9380C9425220C940A
:1005D000B15A0C94B5A00C94BE2E0C94B89A0C94FD
:1005E0007C2E0C9411220C9426760C9403AA0C9465
:1005F000888B0C9498280C943F540C9465A00C9410
:10060000375D0C9467A10C94695D0C9444A10C9423
:10061000E46F0C94CD960C9496830C94935A0C949E
:1006200054540C949C5C0C9408300C94A82F0C949B
:10063000462A0C9445540C944F9C0C94768A0C9446
:100640008D8A0C944C5A0C94C62F0C9400390C943F
:10065000295A0C945AA10C9404310C94E9760C9408
:10066000B59E0C9402300C946E750C94FA2E0C947A
:1006700059A00C94918A0C94C99E0C946A750C94A0
:10068000B28D0C9460750C94242F0C94B62D0C94A0
:10069000982D0C94AF8B0C9444A00C94AA960C94B7
:1006A00015A10C94DDA00C94638A0C941D390C9454
:1006B000EA2F0C94CF7F0C94568B0C94BB5A0C945D
:1006C00080300C94D02A0C94C2930C94A39E0C946A
:1006D00018760C94222E0C944C950C94A4300C9407
:1006E0000D8E0C94B22E0C94DE750C94EC930C943D
:1006F000A2290C9401220C943C970C94B96D0C9493
:10070000B48A0C947BA10C944E8B0C94F8A20C949C
:100710008E960C9412530C94CE2D0C949B9E0C949C
:100720007FA00C94348B0C94E0300C9448750C949E
:1007300000AA0C941D9B0C9497A00C9409A20C94F5
:1007400067840C94A6A00C94B45C0C94A4A90C949B
:10075000E0A20C949E750C94A8800C9486680C946E
:100760002C300C947E8A0C94868C0C94C79E0C942E
:10077000C22D0C9426950C945C5A0C94AA2D0C94C2
:10078000582E0C94902F0C94942E0C94D28B0C9485
:10079000D22F0C94788A0C94B2A00C940A2E0C944C
:1007A000EF800C94968A0C94748A0C94F75C0C94E9
:1007B00061A00C9444620C949D5D0C94AC8B0C94E1
:1007C000C4960C946E300C94B7890C94D4300C946D
:1007D000DF9F0C94057F0C94B02D0C94D78D0C9456
:1007E00014220C9465A10C94665A0C9435530C9405
:1007F0001A7E0C946C380C948BA00C945C960C9420
:10080000C6280C94C4A00C94FE930C94BA2F0C949C
:100810000EA10C946C2F0C94D5940C9419700C941C
:10082000BEA00C94628B0C9482A00C940DA00C942E
:100830004B750C942D310C94B7960C9419830C9431
:10084000A22A0C94536A0C94948A0C94A9A00C9438
:10085000CE8B0C942B8C0C94245A0C94342E0C9428
:10086000F42E0C9462300C941A300C947B750C941A
:10087000542F0C94AD930C94A98B0C94122F0C94C0
:10088000115D0C94CC610C9443770C9477630C94B9
:10089000C0300C948C300C9476540C94BA8B0C941D
:1008A000E22E0C94529C0C9492940C94CC5A0C947E
:1008B000A16F0C946B290C9450C50C94AE9C0C94B5
:1008C0009E2D0C94DC2E0C94882E0C94238B0C946F
:1008D00069750C94BA8A0C94DA2D0C9463380C94D4
:1008E00023750C942C8E0C9498530C945E540C9499
:1008F0006D750C94842F0C9485A00C940A310C9483
:100900001B220C94002F0C9458A10C94602B0C9477
:1009100039640C944C2E0C94888A0C948C8A0C9418
:10092000178C0C94A3760C944DA00C945C760C94CC
:10093000948B0C94E2940C9400950C9470A00C94FD
:100940008B8B0C94402E0C94E39E0C947A5A0C944E
:10095000FE300C946E940C94EE2E0C94E18F0C945B
:10096000FF760C9426300C94B58B0C94C1A00C949B
:10097000FA850C94999E0C94D4930C9451A00C94E9
:10098000D62E0C9416310C9452380C9490610C9421
:10099000C08E0C94FD280C94AAA20C945C9C0C9420
:1009A000818A0C94AB8A0C94858A0C94EC610C942B
:1009B0003C2F0C94A42D0C940E300C94B18A0C9402
:1009C0000E940C945D970C94CAA00C9437800C94F0
:1009D00046400C94E6300C94CC300C949DA00C94C2
:1009E0000D800C94F4670C94522E0C94CC800C94D3
:1009F0005C940C9428310C9438940C94A85C0C945E
:100A0000218C0C94C3680C9412750C94038A0C947A
:100A1000B78A0C94425A0C94E82E0C94A3A00C9420
:100A2000A4610C94C45A0C948A2F0C94EC300C944E
:100A30007D8A0C9415380C9411750C94A02E0C948E
:100A4000AD890C94D9290C9492300C94F62F0C9407
:100A500064970C94C7A60C9422310C9436960C948F
:100A60008EA00C9419670C94758A0C94162E0C9415
:100A70009D8B0C94D0A00C94C1A20C94B8610C94E2
:100A80007D8C0C9477A10C9433220C9473A00C945D
:100A9000B6140C940E220C94A75A0C94F8370C94AC
:100AA00044750C94918B0C949D9E0C9488A00C948E
:100AB000067E0C9446830C9410750C94E4990C9467
:100AC000C85A0C9449750C9449960C94A08B0C94BC
:100AD000CA520C94F82D0C943A390C94E7420C94B9
:100AE00084610C94245D0C942C220C942A400C9468
:100AF0007B8B0C94C98B0C9452750C94B5840C941C
:100B000066760C94D66F0C9428AB0C941D6C0C94E8
:100B100034290C94875D0C94A62E0C94F05C0C94F4
:100B2000B9A10C942E900C9472750C943E760C9492
:100B3000B05C0C94AC5C0C940E8A0C945A7F0C94B0
:100B400094950C9434380C949F9E0C944A750C9494
:100B50006A8A0C9488950C94C5970C94045D0C9447
:100B6000B99B0C94C7A00C94A2990C940A760C948F
:100B70007A8A0C94087E0C94268C0C94988A0C9497
:100B8000C1A60C947A300C940C770C94A22F0C9480
:100B900070540C9484540C94A59E0C94ED6D0C949C
:100BA00010310C94D49A0C94042E0C94C79A0C9483
:100BB000AE8A0C9455A00C94C48B0C94B29E0C94E9
:100BC000A88A0C94A19F0C94F2300C94AC2E0C9437
:100BD00014750C94D5370C94C39B0C9433AB0C94C4
:100BE000DF6E0C9434760C94776E0C94CDA00C943C
:100BF00043610C94895A0C949A2E0C94E42F0C9413
:100C0000C05C0C9445390C943BA00C947E540C941D
:100C1000A3A10C94BC300C941C8C0C94DB680C9439
:100C200044A30C94BBA00C94B85C0C94218A0C9443
:100C300077830C9448760C9459610C940B220C9495
:100C4000928A0C947E2F0C94C28E0C9446A10C9424
:100C5000659C0C948E8A0C942E5A0C946F8B0C9479
:100C6000868A0C94808A0C94A28C0C948E8C0C94A2
:100C7000985C0C9479A10C941F770C945A540C94A2
:100C80008B6A0C94438B0C943B540C9452760C94CA
:100C9000938A0C942EA30C94C42E0C94F2A10C9461
:100CA000822E0C94BA9A0C943E300C94F1760C94EB
:100CB0007B8A0C94A57F0C949AA00C945E2E0C94C5
:100CC00088750C94962F0C9456A10C945A2F0C9462
:100CD000B2300C949A8B0C94CA2E0C9437A20C94BC
:100CE000848A0C94B8A00C94742A0C940FA30C94CE
:100CF000D82F0C945C300C940E680C9461750C9495
:100D0000D3A00C94908A0C94062F0C94AB6E0C9488
:100D10006DA00C943A220C9432300C9409840C94FB
:100D2000D02E0C94468B0C9491770C942E2E0C9410
:100D300059750C940C2F0C94227E0C94188A0C94E8
:100D4000D6A00C945CA10C94C8300C94DC660C9476
:100D5000227F0C94A19E0C9493670C94EB950C94B9
:100D60009E300C9460990C9443530C94077E0C9421
:100D7000DBA00C949D5A0C94426E0C9414300C948D
:100D800095750C941C2E0C94226E0C9471770C9417
:100D900070750C94ACA00C9468540C9421530C9472
:100DA000705A0C94AE2F0C94C82D0C94C68C0C94D5
:100DB0007C950C94AA8A0C94A05C0C9430AB0C9497
:100DC000B18D0C94102E0C94268B0C94362F0C9411
:100DD00090960C941C310C9471750C9494A00C9406
:100DE00086300C94C6960C946E960C944EA20C947D
:100DF000828A0C94F8300C9480940C947C8A0C9425
:100E0000B2930C94642E0C9410C40C9474300C9413
:100E1000A8750C948E2E0C9470950C948A8A0C9460
:100E2000A0950C94A0A00C94C19E0C94B38D0C942E
:100E3000A4940C949F8A0C948E8B0C94B2750C9491
:100E40009C8A0C94462E0C94889B0C94662F0C94D0
:100E5000CA890C94C8940C9446970C94F2420C9452
:100E6000DA300C94ED660C94BD8A0C9433770C94B4
:100E7000B1670C94D42D0C94448C0C9463770C942F
:100E8000799B0C947B900C9463A10C940F750C943B
:100E9000D69E0C942C2B0C944C540C9450540C94C3
:100EA000602F0C9468300C94762E0C94F02F0C94D8
:100EB0000C620C9449540C946D6F0C94FE2A0C94A3
:100EC00062750C94B82E0C94482F0C94EC5C0C9426
:100ED0006A2E0C94778A3400330032004E6F6E65B0
:100EE0000053746F70706564004E65757472616C48
:100EF000205475726E004D6F76696E67205265766C
:100F000065727365004D6F76696E6720466F727704
:100F1000617264004272616B696E670054414E4BAE
:100F200020524553544F5245440025004865616C9A
:100F30007468204C6576656C3A20005645484943F4
:100F40004C452052455041495220434F4D504C454D
:100F500054450054414E4B2044455354524F59453B
:100F6000440025004865616C7468204C6576656CAA
:100F70003A2000290056454849434C4520524550E7
:100F8000414952205354415254454420280052456F
:100F900050414952204F5045524154494F4E2043F1
:100FA000414E43454C4C45440029004D414348497E
:100FB0004E452047554E204849542120280052458F
:100FC00050414952204F5045524154494F4E2043C1
:100FD000414E43454C4C454400290043414E4E4F41
:100FE0004E2048495421202800547572726574209F
:100FF000726F746174696F6E206973206E6F7420F4
:101000006F66207479706520536572766F2E204E5E
:101010006F20736574757020617661696C61626CB4
:10102000652E004E6F207374656572696E6720735C
:101030006572766F2061737369676E65642C2072C8
:10104000652D636865636B2076656869636C6520F0
:10105000747970652E0054757272657420656C65C4
:10106000766174696F6E206973206E6F74206F668D
:10107000207479706520536572766F2E204E6F2034
:10108000736574757020617661696C61626C652E40
:1010900000546F70204C65667400546F7020436577
:1010A0006E74657200546F70205269676874004DE9
:1010B0006964646C65204C656674004D6964646C99
:1010C000652043656E746572004D6964646C6520CB
:1010D000526967687400426F74746F6D204C656666
:1010E0007400426F74746F6D2043656E7465720096
:1010F000426F74746F6D205269676874004649527C
:101100004D574152452056455253494F4E3A2000C3
:101110006942757300534275730050504D004E6F15
:101120006E6520446574656374656400417A696D19
:101130007574682020202000456C65766174696FA5
:101140006E2020005475726E202020202020200068
:101150005468726F74746C65202020005374696346
:101160006B202020202020204D696E20202020434D
:10117000656E7465722020204D6178202020204407
:1011800065616462616E6420205265766572736584
:101190006400524144494F20494E464F202D2000C3
:1011A0004E4F542044455445435445440049474E0E
:1011B0004F52454400416E616C6F67004469676936
:1011C00074616C00417578204368616E2E20202088
:1011D0004D696E20202020204D6178202020202085
:1011E00054797065004368616E6E656C7320757428
:1011F000696C697A65643A20004368616E6E656C5B
:10120000732064657465637465643A200020284423
:10121000697361626C656429002028456E61626CA7
:10122000656429004D656368616E6963616C207255
:1012300065636F696C00416972736F6674004D6518
:101240006368616E6963616C2042617272656C3AB9
:10125000200020284D31290020284D322900202847
:1012600042290042617272656C20456C657661743A
:10127000696F6E3A20200020284D30290020284D2B
:10128000312900202841290054757272657420525A
:101290006F746174696F6E3A2020200020416D7078
:1012A000732900202843757272656E74204C696D35
:1012B00069743A20004472697665204D6F746F72CC
:1012C000733A202020202020004D4F544F522054AC
:1012D0005950455300496E646570656E64656E745F
:1012E00020547265616420436F6E74726F6C005499
:1012F000616E6B202854616D69796120444D4429E9
:101300000054616E6B2028444B4C4D204765617240
:10131000626F7829004361720048616C6674726183
:10132000636B0054616E6B00554E4B4E4F574E0031
:10133000596573004E6F002900252C2044656365B4
:101340006C65726174696F6E20666163746F722080
:101350000020284B69636B6261636B207370656565
:10136000642000547261636B205265636F696C2066
:10137000456E61626C65643A202020004E2F41204A
:10138000666F722076656869636C65207479706534
:10139000005475726E204D6F64653A202020202025
:1013A0002020202020202020200025005374656567
:1013B00072696E672050637420746F207472656167
:1013C00064733A20004E2F4120666F722076656864
:1013D00069636C65207479706500596573202854C1
:1013E000616D69796129002500202D20004E657509
:1013F0007472616C205475726E20416C6C6F7765ED
:10140000643A2020200020736563005472616E737B
:101410006D697373696F6E2044656C61793A202041
:10142000202020002073656300456E67696E65208B
:1014300050617573652054696D653A202020202025
:101440002000207365630053686966742054696DD9
:10145000653A20202020202020202020202020004D
:101460004175746F6D61746963004D616E75616C77
:10147000005472616E736D697373696F6E20547975
:1014800070653A2020202020200025005965732017
:101490002D20005265766572736520537065656412
:1014A000204C696D697465643A20200025005965F7
:1014B00073202D2000466F7277617264205370652F
:1014C0006564204C696D697465643A202000206D64
:1014D00073290025207468726F74746C6520666FC0
:1014E0007220002028004D6F746F72204E75646763
:1014F0006520456E61626C65643A202020200029D9
:10150000004E6F6E65004E6F6E65002C2050726548
:101510007365743A20002900202841646A75737449
:10152000656420746F200020284C6576656C3A2035
:1015300000446563656C2052616D7020456E616288
:101540006C65643A20202020200029004E6F6E65D3
:10155000004E6F6E65002C205072657365743A20E2
:10156000002900202841646A757374656420746FD3
:10157000200020284C6576656C3A20004163636545
:101580006C2052616D7020456E61626C65643A201A
:1015900020202020004163746976652044726976BA
:1015A000696E672050726F66696C653A20005665F7
:1015B0006869636C6520547970653A20202020208A
:1015C00020202020202000445249564520534554D5
:1015D00054494E47530020736563005265636F6939
:1015E0006C2064656C61793A202020202020202026
:1015F00020202020202020202020200025005965A8
:1016000073202D200042617272656C20456C6576F6
:101610006174696F6E205370656564204C696D69F3
:101620007465643A20002500596573202D2000540C
:10163000757272657420526F746174696F6E205395
:1016400070656564204C696D697465643A2020009A
:101650005455525245542053455454494E47530013
:10166000556E6B6E6F776E004578706572696D654B
:101670006E74616C005365706172617465204865B9
:10168000617420262046616E00436F6D62696E654D
:1016900064204865617420262046616E0025004460
:1016A000697361626C656400536D6F6B6520776868
:1016B000656E2064657374726F7965643A200046C4
:1016C000616E206D61782073706565643A2020201A
:1016D00020202020200046616E20666173742069FE
:1016E000646C652073706565643A20200046616E05
:1016F0002069646C652073706565643A2020202041
:1017000020202000202863757272656E746C792029
:1017100064697361626C65642900207365636F6E30
:101720006473004E2F41005072652D68656174200E
:1017300064656C61793A2020202020202000536DC0
:101740006F6B657220547970653A2020202020202C
:101750002020202000536D6F6B6572206F757470B0
:10176000757420636F6E74726F6C6C6564206D614C
:101770006E75616C6C7900534D4F4B455200466C51
:1017800069636B657220686561646C69676874730E
:1017900020647572696E6720656E67696E65207377
:1017A000746172743A200052756E6E696E67206CB7
:1017B000696768747320616C77617973206F6E3A22
:1017C00000250052756E6E696E67206C69676874DB
:1017D000732064696D206C6576656C3A00427261B5
:1017E0006B65206C6967687473206F6E207768651D
:1017F0006E2073746F707065643A004C49474854AA
:101800002053455454494E475300556E6B6E6F77C5
:101810006E004865617679004D656469756D004CB0
:101820006967687400437573746F6D00556E6B6EF5
:101830006F776E004E6F6E65004F70656E20506161
:101840006E7A65720054616D6979612053706563C9
:101850000020736563207265636F76657279290075
:10186000207365632072656C6F61642C2000204DCD
:101870004720686974732C20002063616E6E6F6E60
:1018800020686974732C20002800576569676874A4
:1018900020436C6173733A20202020200044616D46
:1018A0006167652050726F66696C653A2020200080
:1018B000596573202800416363657074204D47208B
:1018C00044616D6167653A200059657320280053B3
:1018D000656E64204D4720495220436F64653A206D
:1018E00020004E2F4100526570616972656420626C
:1018F000793A202020202020004E2F410048697492
:101900002050726F746F636F6C20323A2020200079
:10191000290020285465616D2000466972652050B9
:10192000726F746F636F6C3A2020202000466972DA
:10193000652050726F746F636F6C3A202020200016
:101940004973205265706169722054616E6B3F204B
:10195000202000495220262054616E6B2042617481
:10196000746C696E672044697361626C65640042DF
:101970004154544C4520494E464F00554E4B4E4F16
:10198000574E0042656E6564696E6920544253206B
:101990004D6963726F0042656965722055534D2D24
:1019A00052432D320054616967656E20536F756E26
:1019B000642043617264004F70656E2050616E7ADE
:1019C000657220536F756E642043617264004265D6
:1019D0006E6564696E6920544253204D696E6900DA
:1019E000536F756E6420636172643A2000534F55E3
:1019F0004E44204341524400556E6B6E6F776E002B
:101A000042617272656C20456C65766174696F6EB7
:101A100020436F6D6D616E64005475727265742041
:101A2000526F746174696F6E20436F6D6D616E6487
:101A3000005374656572696E6720436F6D6D616EEA
:101A4000640056656869636C652053706565640061
:101A5000456E67696E6520537065656400546872F1
:101A60006F74746C6520436F6D6D616E64005370AC
:101A70006565642064656372656173657320626582
:101A80006C6F772000537065656420696E637265C2
:101A9000617365732061626F766520005475726EA4
:101AA0002053746F70706564004C656674205475C3
:101AB000726E205374617274656400526967687451
:101AC000205475726E20537461727465640056659B
:101AD0006869636C652053746F70706564004D6F46
:101AE00076696E672052657665727365004D6F7614
:101AF000696E6720466F727761726400456E676930
:101B00006E652053746F7000456E67696E65205373
:101B1000746172740043616E6E6F6E2052656C6FFB
:101B2000616465640056656869636C65204465732B
:101B300074726F7965640043616E6E6F6E204869E0
:101B400074004272616B6573204170706C696564EA
:101B5000005661726961626C6500290020286F6619
:101B60002000506F732000417578204368616E6ECD
:101B7000656C20005661726961626C65004F6E0091
:101B80004F6666004200410045787465726E616C74
:101B900020496E7075742000070809090B0C0C0BA6
:101BA0000C0C54757272657420537469636B202D2C
:101BB000200046756E6374696F6E202300202D3EF1
:101BC00020002073656300547572726574206D6F18
:101BD00076656D656E742064656C61793A202000CD
:101BE0004E6F6E650059657300547572726574208E
:101BF000737469636B2066756E6374696F6E733A94
:101C0000200046554E4354494F4E205452494747B1
:101C10004552530076206375746F6666290020284C
:101C2000004C564320456E61626C65643A2020206A
:101C3000202020007600566F6C746167653A202082
:101C4000202020202020202000596573004E6F00A6
:101C50004261747465727920446574656374656467
:101C60003A2000424154544552590053657269610B
:101C70006C203320547820426175643A2020004162
:101C800075782053657269616C20426175643A20F1
:101C90002020004D6F746F722053657269616C2053
:101CA000426175643A200055534220536572696160
:101CB0006C20426175643A20202000424155442046
:101CC000524154455300212000464143544F52593C
:101CD00020524553455421200054616967656E20A8
:101CE00056322F563300536F6E79005243544120C1
:101CF0004D616368696E652047756E00436C617263
:101D00006B204D616368696E652047756E005243B4
:101D100054412052657061697200494255205265F4
:101D20007061697200436C61726B20526570616909
:101D300072004F70656E50616E7A65720056735412
:101D4000616E6B00464F560054616967656E2056A0
:101D5000310048656E67204C6F6E670054616D6995
:101D6000796120312F33350054616D6979612032FA
:101D70002D53686F740054616D69796100556E6B05
:101D80006E6F776E003A20004269742000476170E0
:101D90003A200000002100240027002A002D0030F6
:101DA00000330001010000040107010A01000022C4
:101DB00000250028002B002E003100340002010015
:101DC00000050108010B0100002000230026002966
:101DD000002C002F00320000010000030106010961
:101DE0000105050505070508080808020202020AA0
:101DF0000A080804040404010101010101010103AE
:101E000003030303030303040707070C0C0C0C0C68
:101E10000C0C0C0202020206060606060606060B5B
:101E20000B0B0B0B0B0B0B010210202008081020D2
:101E30004010204080020102010804020101020456
:101E40000810204080804020100804020180040215
:101E5000018040201008040201080402010102046C
:101E60000810204080010204081020408000000A71
:101E70000B02090C0D0E080703040100000000000E
:101E80000000000000000000000000000000000052
:101E9000000000000000000000121110000000000F
:101EA0000000000000000000000000000000000032
:101EB00000000044726976696E672050726F66692F
:101EC0006C652073657420746F20230025005370A7
:101ED000656564207265647563656420746F2000B5
:101EE000537065656420726573746F726564005425
:101EF00075726E20456E67696E65204F6E002073A7
:101F000065636F6E64732061676F202D20736D6F42
:101F10006B6572207072656865617420736B69709F
:101F200070656400456E67696E65206C617374202E
:101F300073746F707065642000207365636F6E64E6
:101F40007300536D6F6B6572207072652D686561EB
:101F5000742073746172746564202D20656E6769E6
:101F60006E652077696C6C207475726E206F6E20C0
:101F7000696E20004D616E75616C207472616E73C4
:101F80006D697373696F6E202D2070757420696E92
:101F9000206E65757472616C206765617220626580
:101FA000666F7265207374617274696E6720656E06
:101FB00067696E652100456E67696E6520417574BD
:101FC0006F2053687574646F776E00456E67616744
:101FD00065205472616E736D697373696F6E00442E
:101FE0006973656E67616765205472616E736D69B0
:101FF0007373696F6E00536574205475726E204D53
:102000006F64653A203100536574205475726E20F8
:102010004D6F64653A203200536574205475726EBA
:10202000204D6F64653A203300456E61626C652017
:102030004E65757472616C205475726E73004469DC
:102040007361626C65204E65757472616C205475A5
:10205000726E7300494F20506F72742041204F758B
:1020600074707574202D204F6E00494F20506F7290
:10207000742041204F7574707574202D204F666652
:1020800000494F20506F72742042204F7574707554
:1020900074202D204F6E00494F20506F72742042E3
:1020A000204F7574707574202D204F6666004C5655
:1020B000432045786974202D20566F6C74616765E4
:1020C00020526573746F726564007629004C564324
:1020D000207468726573686F6C64207265616368F0
:1020E0006564212028004C696768742031204F6E98
:1020F000004C696768742031204F6666004C696740
:1021000068742032204F6E004C696768742032205A
:102110004F666600326E64204D472053746F700026
:10212000326E64204D472053746172740052756E94
:102130006E696E67204C6967687473204F6E005239
:10214000756E6E696E67204C6967687473204F66A0
:102150006600417578204F7574707574204F6E005D
:10216000417578204F7574707574204F6666005302
:10217000746F70205265766F6C76696E672041755A
:1021800078204C696768740053746F7020417578CB
:10219000204F757470757420426C696E6B696E6740
:1021A00000417578204F7574707574205072657396
:1021B00065742044696D00537461727420417578B0
:1021C000204F757470757420426C696E6B696E6710
:1021D00000401F7017D007A00FA00FDC05D007C468
:1021E0000910278813983A102758026C0258026C7D
:1021F0000258026C0258026C0258026C0258026CBF
:102200000258026C0258026C025802B0366C023A54
:10221000026C023A026C023A026C02B036384A5C36
:10222000121C255C125C121C255C12BC7FC7F2C01C
:102230007887A5B7C5A00F8813B80B401FB80BB897
:102240000B7017401F526164696F20526561647999
:10225000202D200052657665727365643A20200057
:102260004D61782050756C73653A20004D696E2081
:1022700050756C73653A2000456E642056616C752C
:10228000657300456E64205265636F696C20536509
:1022900072766F20536574757000456E6420526FBE
:1022A000746174696F6E20536572766F2053657424
:1022B000757000456E64205374656572696E6720A1
:1022C000536572766F20536574757000456E642097
:1022D0005374656572696E6720536572766F20531B
:1022E0006574757000456E6420456C65766174692F
:1022F0006F6E20536572766F20536574757000534E
:102300006572766F20756E2D726576657273656481
:1023100000536572766F207265766572736564002E
:1023200052657665727365643A2020004D617820AD
:1023300050756C73653A20004D696E2050756C7352
:10234000653A200053746172742056616C75657330
:1023500000494E56414C494420534552564F2E2079
:102360004E4F2053455455502E00536574757020C0
:102370005265636F696C20536572766F00536574A4
:1023800075702054757272657420526F746174692F
:102390006F6E2050616E20536572766F00536574C6
:1023A0007570205374656572696E67205365727627
:1023B0006F20284F7574707574203229005365742E
:1023C0007570205374656572696E67205365727607
:1023D0006F20284F7574707574203429005365740C
:1023E00075702054757272657420456C65766174E1
:1023F000696F6E20536572766F00556E6B6E6F77E6
:102400006E004F6E626F617264204D6F746F722048
:102410004472697665727320432026204400446527
:102420007461636865642F4E41005265636F696C27
:1024300020536572766F0050616E20536572766F1F
:1024400000536572766F2F455343004F6E626F6184
:102450007264204D6F746F722044726976657200E9
:102460004F70656E2050616E7A65722053636F7590
:10247000742053657269616C204553430053616257
:102480006572746F6F74682053657269616C005077
:102490006F6C6F6C752053657269616C0053657267
:1024A000766F203100536572766F2032005365726B
:1024B000766F203300536572766F20340053657257
:1024C000766F203500536572766F20360053657243
:1024D000766F203700536572766F203800466F7232
:1024E000776172642047656172004E657574726130
:1024F0006C2047656172005265766572736520478E
:102500006561720053657420416363656C2052619C
:102510006D70204C6576656C3A20005365742044DC
:102520006563656C2052616D70204C6576656C3A10
:102530002000416E616C6F6720557365722046758F
:102540006E6374696F6E2031202D2000416E616CC6
:102550006F6720557365722046756E6374696F6E80
:102560002032202D20002D00202D2000200054524C
:1025700055450046414C5345002500576169746933
:102580006E6720666F7220726164696F2E2E2E2036
:102590000053657420766F6C756D653A2000202DB0
:1025A00020537461727420526570656174696E673E
:1025B00000202D2053746F70005573657220536F87
:1025C000756E64200041202D200042202D200053F4
:1025D0006F756E642042616E6B2000506C61792FC4
:1025E00053746F7000506C61792052616E646F6D2E
:1025F00000506C61792050726576696F7573005078
:102600006C6179204E6578740020287769746820A1
:1026100049522900466972652043616E6E6F6E00F3
:102620004669726520526570616972205369676EF0
:10263000616C00416972736F6674202D204D616E6C
:1026400075616C2054726967676572004D656368D7
:10265000616E6963616C205265636F696C202D2027
:102660004D616E75616C20547269676765720053C5
:102670006572766F205265636F696C202D204D6105
:102680006E75616C2054726967676572004869678E
:102690006820496E74656E7369747920466C617345
:1026A0006820556E6974202D204D616E75616C2017
:1026B00054726967676572004D4720537461727484
:1026C000004D472053746F70004952204E4F5420E4
:1026D000656E61626C6564202D206E6F204952200A
:1026E00070726F746F636F6C732073656C65637465
:1026F00065642E00556E61626C6520746F20656E96
:1027000061626C6520495200495220656E61626CBD
:1027100065640049522064697361626C65640041BC
:102720007578204F757470757420466C6173686598
:102730006400417578204F757470757420496E7609
:102740006572736520466C61736865640053746FCD
:102750007020417578204F757470757420426C69D3
:102760006E6B696E670053746F70205265766F6C84
:1027700076696E6720417578204C696768740053EC
:10278000746F7020416C6C205573657220536F75A7
:102790006E647300494F20506F72742041202D20C9
:1027A00050756C73656400494F20506F72742041FE
:1027B000202D20537461727420426C696E6B696EB7
:1027C0006700494F20506F72742042202D205075B1
:1027D0006C73656400494F20506F72742042202D45
:1027E00020537461727420426C696E6B696E67006D
:1027F000557365722046756E6374696F6E20310083
:10280000557365722046756E6374696F6E20320071
:10281000536D6F6B657220656E61626C6564005309
:102820006D6F6B65722064697361626C65640041F1
:102830006972736F6674202D20456E61626C6564E9
:10284000004D656368616E6963616C205265636FFA
:10285000696C202D20456E61626C6564004169726F
:10286000736F6674202D2044697361626C65640027
:102870004D656368616E6963616C205265636F6961
:102880006C202D2044697361626C656400436F6D38
:102890006D73206368616E67656420746F205553A3
:1028A0004200436F6D6D73206368616E67656420DD
:1028B000746F2053657269616C20310048656174E2
:1028C00020416D743A2000486561743A20005361DC
:1028D0006D652061732066616E00537461727420AF
:1028E0005265766F6C76696E6720417578204C6909
:1028F00067687400524144494F204641494C534156
:102900004645000082BF11241FBECFEFD1E2DEBFDB
:10291000CDBF00E00CBF17E0A0E0B2E0E3EDF6ECC5
:1029200001E00BBF02C007900D92A231B107D9F7A9
:1029300024E1A2E1B7E001C01D92AA3DB207E1F790
:1029400014E1C3E8D4E100E006C021970109802F1B
:10295000FE010E9491CFC238D10780E00807A9F795
:102960000E9400AD0C94EDD10C9400002F923F9288
:102970004F925F926F927F928F929F92AF92BF928F
:10298000CF92DF92EF92FF920F931F93CF93DF933B
:10299000CDB7DEB7E6970FB6F894DEBF0FBECDBF5A
:1029A00080917713909178130E9458560E941E9739
:1029B0006DEF70E180917713909178130E945957D1
:1029C0006BE676E0CE0101960E94D6558091771392
:1029D00090917813DC01ED91FC914D815E816981CC
:1029E0007A810280F381E02D199563E776E080918A
:1029F0007713909178130E9457572AE045EE51E0E3
:102A000060E070E080917713909178130E940F56E8
:102A100065EC76E080917713909178130E945C5674
:102A2000CE0101960E9478550E9409A680917713E5
:102A300090917813DC01ED91FC910680F781E02DF7
:102A4000199580917713909178130E9458560E949F
:102A50001E9762E971E180917713909178130E943B
:102A60005957E091F60BE4300CF0E0E08EE191E193
:102A70009A8389838AE191E19C838B8385E191E14B
:102A80009E838D8380E191E198878F83EE0FFF0B0A
:102A900021E030E02C0F3D1FE20FF31F60817181B8
:102AA00080917713909178130E947D570E941E9712
:102AB0006CE571E180917713909178130E947D57B6
:102AC0000E941E9760E571E18091771390917813D1
:102AD0000E945957E091A910F091AA10818192812A
:102AE000883E934014F40E940E97E091A910F09153
:102AF000AA106181728180917713909178130E945E
:102B0000007284E00E947AACE091A910F091AA10C2
:102B10006581768180917713909178130E9400727D
:102B200085E00E947AACE091A910F091AA1063812F
:102B3000748180917713909178130E94007284E0E1
:102B40000E947AACE091A910F091AA10678180915F
:102B50007713909178130E943F7088E00E947AACBE
:102B6000E091A910F091AA1080850E94F49664E487
:102B700071E180917713909178130E945957E091F9
:102B8000B310F091B41081819281883E934014F487
:102B90000E940E97E091B310F091B41061817281A0
:102BA00080917713909178130E94007284E00E94C4
:102BB0007AACE091B310F091B41065817681809188
:102BC0007713909178130E94007285E00E947AAC8E
:102BD000E091B310F091B410638174818091771308
:102BE000909178130E94007284E00E947AACE09188
:102BF000B310F091B410678180917713909178139E
:102C00000E943F7088E00E947AACE091B310F0918E
:102C1000B41080850E94F49668E371E18091771387
:102C2000909178130E945957E091BD10F091BE1019
:102C300081819281883E934014F40E940E97E09126
:102C4000BD10F091BE1061817281809177139091D7
:102C500078130E94007284E00E947AACE091BD106B
:102C6000F091BE10658176818091771390917813F1
:102C70000E94007285E00E947AACE091BD10F09154
:102C8000BE106381748180917713909178130E94B4
:102C9000007284E00E947AACE091BD10F091BE1009
:102CA000678180917713909178130E943F7088E03C
:102CB0000E947AACE091BD10F091BE1080850E9418
:102CC000F4966CE271E180917713909178130E94F1
:102CD0005957E091C710F091C81081819281883EC8
:102CE000934014F40E940E97E091C710F091C81021
:102CF0006181728180917713909178130E940072A4
:102D000084E00E947AACE091C710F091C810658110
:102D1000768180917713909178130E94007285E0FC
:102D20000E947AACE091C710F091C8106381748161
:102D300080917713909178130E94007284E00E9432
:102D40007AACE091C710F091C81067818091771339
:102D5000909178130E943F7088E00E947AACE091D5
:102D6000C710F091C81080850E94F4968091771367
:102D7000909178130E9458560E9406AAC82E64ECBF
:102D800071E180917713909178130E947D570E9492
:102D90001E970DE410E1E12CF12CD12C5701BFEF6F
:102DA000AB1ABB0AB50180917713909178130E94FA
:102DB0000072E9E0EE16F10410F48BE001C08AE045
:102DC0000E947AACD8012C9180917713909178135E
:102DD0002223C9F11596ED91FC91169761817281BC
:102DE0000E940072D8011596ED91FC911697818191
:102DF0009281883E934014F40E940E9784E00E94D2
:102E00007AACD8011596ED91FC9116976381748187
:102E100080917713909178130E94007284E00E9451
:102E20007AACD8011596ED91FC9116972781809187
:102E3000771390917813222319F06CEB71E10BC09A
:102E400065EB71E108C0EC14FD041CF46DEA71E15E
:102E500002C060EA71E10E947D57095F1F4F750152
:102E6000BCE0AB16B10409F099CF0E941E9769EF40
:102E700071E180917713909178130E9459570E94C5
:102E800006AA682F80917713909178130E9428707A
:102E900065EE71E180917713909178130E945957F4
:102EA0006091F30B7091F40B8091771390917813EC
:102EB0000E9436720E9409A6809177139091781330
:102EC000DC01ED91FC910680F781E02D1995809150
:102ED0007713909178130E9458560E941E9769ECC0
:102EE00072E180917713909178130E947D570E9430
:102EF0001E9765EB72E180917713909178130E9491
:102F000059578091AC120E94038FBC0180917713B6
:102F1000909178130E9459578091AC128A30C1F475
:102F200063EA72E180917713909178130E94595768
:102F300060916C1380917713909178130E943F7089
:102F40006CE972E180917713909178130E94595740
:102F500080917713909178130E94585668E872E137
:102F600080917713909178130E9459578091AD12F8
:102F70000E94038FBC0180917713909178130E9477
:102F800059572091AD1280917713909178132B307F
:102F90003CF4293054F4283069F467E772E107C043
:102FA0002B3041F463E872E102C06DE772E10E94E8
:102FB0007D5702C00E94585663E672E180917713F4
:102FC000909178130E9459578091AE120E94038FFE
:102FD000BC0180917713909178130E9459572091EA
:102FE000AE1280917713909178132B303CF42930F6
:102FF00054F4283069F462E572E107C02B3041F4E3
:103000006EE572E102C068E572E10E947D5702C080
:103010000E9458566EE372E1809177139091781375
:103020000E9459572091C012809177139091781384
:10303000222319F066E372E102C064E272E10E94A9
:1030400059572091E9138091771390917813222397
:1030500019F069E172E102C06DE072E10E94595716
:1030600080917713909178130E9458560E9409A678
:103070008091771390917813DC01ED91FC9106809B
:10308000F781E02D199580910002823011F00C94A7
:103090003523F090E7120091EA1210E08091771347
:1030A000909178130E9458560E941E9767EC75E124
:1030B00080917713909178130E947D570E941E97FC
:1030C0006EEA75E180917713909178130E945957B9
:1030D000E091F712E7300CF0E0E088E293E19A83A8
:1030E000898383E293E19C838B8389E193E19E83CF
:1030F0008D8385E193E198878F8381E093E19A87BF
:1031000089878FEE92E19C878B8785ED92E19E8780
:103110008D87EE0FFF0B21E030E02C0F3D1FE20FFB
:10312000F31F6081718180917713909178130E94D1
:103130007D5765E975E180917713909178130E942E
:1031400059576091000280917713909178130E94F3
:1031500028706CE775E180917713909178130E9445
:1031600059578F2D0E94DE96FF2009F44BC062E76D
:1031700075E180917713909178130E94595780914F
:10318000771390917813112339F06091E2120E9425
:103190003F709091E21206C06091E8120E943F7069
:1031A0009091E8128091951498130C943C2366E555
:1031B00075E180917713909178130E94595780910F
:1031C000771390917813112339F06091E312611114
:1031D0000CC061E575E106C06091E912611105C09E
:1031E0006CE475E10E94595705C0062E000C770B60
:1031F0000E9400726AE475E18091771390917813D0
:103200000E94595780917713909178130E945856D5
:1032100061E375E180917713909178130E9459577B
:10322000802F0E94DE96002309F44BC067E275E10F
:1032300080917713909178130E945957809177135A
:1032400090917813112339F06091E5120E943F703C
:103250009091E51206C06091EB120E943F70909130
:10326000EB128091971498130C9456236BE075E140
:1032700080917713909178130E945957809177131A
:1032800090917813112339F06091E61261110CC00E
:1032900066E075E106C06091EC12611105C061E065
:1032A00075E10E94595705C0062E000C770B0E944D
:1032B00000726FEF74E180917713909178130E9400
:1032C000595780917713909178130E94585666EE63
:1032D00074E180917713909178130E9459578091EF
:1032E0000013811103C00E94EC9635C060E373E1C6
:1032F00080917713909178130E94595763EE74E18F
:1033000080917713909178130E9459576091001320
:1033100080917713909178130E943F7063ED74E170
:1033200080917713909178130E945957409101131F
:103330005091021360E070E02AE080917713909141
:1033400078130E940F566EEC74E180917713909180
:1033500078130E947D5765EB74E18091771390910B
:1033600078130E9459578091F8128436C8F46EEA97
:1033700074E180917713909178130E94595760916E
:10338000F81280917713909178130E943F706CEA45
:1033900074E180917713909178130E947D5703C058
:1033A00080E00E94EC9663E974E18091771390913C
:1033B00078130E9459578091F9128436C8F46CE84A
:1033C00074E180917713909178130E94595760911E
:1033D000F91280917713909178130E943F706AE8F8
:1033E00074E180917713909178130E947D5703C008
:1033F00080E00E94EC9661E774E1809177139091F0
:1034000078130E9459572091A707809177139091C4
:103410007813222319F06AE674E102C060E674E1D1
:103420000E947D5767E474E180917713909178133F
:103430000E9459576091EE127091EF12072E000C06
:10344000880B990B0E94F8CB20E030E04AE754E467
:103450000E9417CEAB01BC0121E0809177139091BF
:1034600078130E94755662E474E18091771390910D
:1034700078130E947D5769E274E1809177139091EF
:1034800078130E9459576091F0127091F112072E33
:10349000000C880B990B0E94F8CB20E030E04AE743
:1034A00054E40E9417CEAB01BC0121E08091771358
:1034B000909178130E94755664E274E180917713BD
:1034C000909178130E947D576BE074E1809177139F
:1034D000909178130E9459576091F2127091F312F3
:1034E000072E000C880B990B0E94F8CB20E030E0EF
:1034F0004AE754E40E9417CEAB01BC0121E0809161
:103500007713909178130E94755666E074E180916C
:103510007713909178130E947D576DEE73E180913F
:103520007713909178130E9459579091F712913028
:1035300011F09430F9F48091F4120E94DE9680919B
:10354000F412882329F169EE73E180917713909149
:1035500078130E9459576091F512809177139091DA
:1035600078130E943F7067EE73E18091771390911A
:1035700078130CC02091771330917813953019F49B
:103580006AED73E102C065EC73E1C9010E9459570D
:1035900080917713909178130E9458568091F7127A
:1035A0008230C1F46CEA73E18091771390917813C3
:1035B0000E9459576091FA12809177139091781375
:1035C0000E943F706AEA73E18091771390917813BB
:1035D0000E947D5761E973E1809177139091781390
:1035E0000E9459579091F7122FEF290F809177136E
:1035F00090917813223028F4609112070E9428706D
:1036000004C06CE773E10E947D5763E673E180912B
:103610007713909178130E945957809104130E9458
:10362000DE9680910413882341F161E573E1809176
:103630007713909178130E945957609105138091E8
:103640007713909178130E943F7069E373E1809142
:103650007713909178130E945957609106138091C7
:103660007713909178130E943F7067E373E1809124
:103670007713909178130E94595780917713909106
:1036800078130E9458560E9409A680917713909152
:103690007813DC01ED91FC910680F781E02D1995FE
:1036A00080917713909178130E9458560E941E972C
:1036B00060E576E180917713909178130E947D57B1
:1036C0000E941E976FE276E18091771390917813B4
:1036D0000E9459578091B5128436C8F468E276E1A9
:1036E00080917713909178130E9459576091B51289
:1036F00080917713909178130E943F7066E276E193
:1037000080917713909178130E947D5703C080E0D9
:103710000E94EC9665E076E18091771390917813A2
:103720000E9459578091B4128436C8F46EEF75E147
:1037300080917713909178130E9459576091B41239
:1037400080917713909178130E943F706CEF75E130
:1037500080917713909178130E947D5703C080E089
:103760000E94EC966BED75E1809177139091781340
:103770000E9459576091C2127091C3121616170613
:1037800014F50091771310917813072E000C880B15
:10379000990B0E94F8CB20E030E04AE754E40E9405
:1037A00017CEAB01BC0122E0C8010E947556C801CA
:1037B0000E94585666ED75E18091771390917813C9
:1037C0000E947D5703C080E00E94EC960E9409A6EB
:1037D0008091771390917813DC01ED91FC91068034
:1037E000F781E02D199580917713909178130E94BD
:1037F00058560E941E9767E777E180917713909162
:1038000078130E947D570E941E972091CF128091BD
:10381000771390917813FE0131966F01211103C047
:1038200065E577E1C7C16EE377E10E945957E09102
:10383000D812E3300CF0E3E089E896E19A838983BB
:1038400085E796E19C838B8388E696E19E838D8352
:1038500080E696E198878F83EE0FFF0BEC0DFD1D40
:103860006081718180917713909178130E947D57C8
:10387000FF24F3948091D812811101C0F12C67E2EA
:1038800077E180917713909178130E945957609156
:10389000D9128091771390917813611105C063E27A
:1038A00077E10E947D571AC00E943F706AE177E17C
:1038B00080917713909178130E9459578091F40763
:1038C000811108C064E077E18091771390917813BB
:1038D0000E94595785ED99E00E9458566091D01288
:1038E0007091D112072E000C880B990B0E94F8CB17
:1038F00020E030E04FE753E40E9417CE20E030E0B4
:1039000048EC52E40E9457CC20E030E040E05FE316
:103910000E94ABCD0E9489CEE62E262F372F89013B
:10392000A090DA12B090DB126DEE76E18091771301
:10393000909178130E9459578E2D0E94CF9604368D
:1039400011053CF40E940E970A30110514F40E94F0
:103950000E9783E00E947AACFF2001F10E94E0AC58
:10396000B501BB0C880B990B0E94F8CB20E030E02E
:103970004FE753E40E9417CE20E030E048EC52E4D9
:103980000E9457CC20E030E040E05FE30E94ABCDE6
:103990000E9489CE862F0E94CF9604C00E94D8AC88
:1039A0000E94D0AC0E9408976091D2127091D312FD
:1039B000072E000C880B990B0E94F8CB20E030E01A
:1039C0004FE753E40E9417CE20E030E048EC52E489
:1039D0000E9457CC20E030E040E05FE30E94ABCD96
:1039E0000E9489CEE62E262F372F8901A090DC1267
:1039F000B090DD1266ED76E18091771390917813A7
:103A00000E9459578E2D0E94CF96043611053CF422
:103A10000E940E970A30110514F40E940E9783E05D
:103A20000E947AACFF2001F10E94E0ACB501BB0C12
:103A3000880B990B0E94F8CB20E030E04FE753E46D
:103A40000E9417CE20E030E048EC52E40E9457CCB0
:103A500020E030E040E05FE30E94ABCD0E9489CEE1
:103A6000862F0E94CF9604C00E94D8AC0E94D0AC92
:103A70000E9408976091D4127091D512072E000C05
:103A8000880B990B0E94F8CB20E030E04FE753E41D
:103A90000E9417CE20E030E048EC52E40E9457CC60
:103AA00020E030E040E05FE30E94ABCD0E9489CE91
:103AB000E62E262F372F8901A090DE12B090DF125C
:103AC0006FEB76E180917713909178130E945957AC
:103AD0008E2D0E94CF96043611053CF40E940E975D
:103AE0000A30110514F40E940E9783E00E947AAC0C
:103AF000FF2001F10E94E0ACB501BB0C880B990BD3
:103B00000E94F8CB20E030E04FE753E40E9417CE4C
:103B100020E030E048EC52E40E9457CC20E030E056
:103B200040E05FE30E94ABCD0E9489CE862F0E94C9
:103B3000CF9604C00E94D8AC0E94D0AC0E940897D7
:103B400068EA76E180917713909178130E94595733
:103B50006091D6127091D71200917713109178135B
:103B60006115710521F46FE976E1C80123C0072EC4
:103B7000000C880B990B0E94F8CB20E030E04FE757
:103B800053E40E9417CE20E030E048EC52E40E945B
:103B900057CC20E030E040E05FE30E94ABCD0E94D4
:103BA00089CEC8010E9400726DE976E18091771399
:103BB000909178130E947D570E9409A680917713F7
:103BC00090917813DC01ED91FC910680F781E02D56
:103BD000199580917713909178130E9458560E94FE
:103BE0001E976BEF77E180917713909178130E9485
:103BF0007D570E941E976DED77E18091771390912C
:103C000078130E9459578BE00E947AAC80915D1323
:103C10000E94EC9663EC77E1809177139091781392
:103C20000E9459578FE00E947AAC60915C1380919A
:103C30007713909178130E943F7061EC77E1809147
:103C40007713909178130E947D5767EA77E180910E
:103C50007713909178130E9459578FE00E947AACA5
:103C600080915B130E94EC966EE777E18091771369
:103C7000909178130E94595780916B130E94EC9693
:103C80000E9409A68091771390917813DC01ED9141
:103C9000FC910680F781E02D199580917713909122
:103CA00078130E9458560E941E976FE679E1809122
:103CB0007713909178130E947D570E941E97209150
:103CC00032078091771390917813222309F4B7C1BA
:103CD00060E479E10E9459570E9469970E94EC962E
:103CE0000E9469972091771330917813882389F087
:103CF0006DE279E1C9010E945957809135070E9410
:103D00003343BC0180917713909178130E947D57C3
:103D10004BC06AE179E1C9010E945957809132078D
:103D20000E943343BC0180917713909178130E94D5
:103D3000595780913307882389F162E179E18091B5
:103D40007713909178130E945957E0913307E4302C
:103D50000CF0E0E08CED9EE09A8389838AED9EE092
:103D60009C838B8388ED9EE09E838D8386ED9EE011
:103D700098878F83EE0FFF0BEC0DFD1D6081718125
:103D800080917713909178130E94595760E179E1FF
:103D900080917713909178130E94595780917713EF
:103DA000909178130E9458566DEF78E180917713C7
:103DB000909178130E94595780913407009177139E
:103DC00010917813882321F00E943343BC0102C074
:103DD00069EF78E1C8010E947D5766EE78E1809135
:103DE0007713909178130E9459578091350700916D
:103DF000771310917813882321F00E943343BC017C
:103E000002C062EE78E1C8010E947D576FEC78E154
:103E100080917713909178130E94595780913707BA
:103E20008823E1F069EC78E1809177139091781321
:103E30000E945957809136070E943343BC018091FC
:103E40007713909178130E94595765EC76E0809132
:103E50007713909178130E945C5603C080E00E9413
:103E6000EC9666EB78E180917713909178130E943D
:103E70005957809138078823E1F060EB78E1809111
:103E80007713909178130E945957809136070E94BA
:103E90003343BC0180917713909178130E94595756
:103EA00065EC76E080917713909178130E945C56D0
:103EB00003C080E00E94EC966DE978E18091771371
:103EC000909178130E945957E0913907E3300CF034
:103ED000E3E085E498E19A83898389E398E19C8310
:103EE0008B8384E398E19E838D838CE298E19887AD
:103EF0008F83EE0FFF0BEC0DFD1D608171818091B2
:103F00007713909178130E947D576AE878E1809149
:103F10007713909178130E945957E0912B07E43062
:103F20000CF0E4E085E298E19A8389838FE198E1DF
:103F30009C838B8388E198E19E838D8382E198E165
:103F400098878F838AE098E19A878987EE0FFF0B25
:103F5000EC0DFD1D60817181809177139091781334
:103F60000E947D5768E878E18091771390917813EB
:103F70000E94595760913007809177139091781380
:103F80000E943F7069E778E18091771390917813F0
:103F90000E94595780912B07811110C06091310701
:103FA00080917713909178130E943F706EE678E1CC
:103FB00080917713909178130E94595760912C0744
:103FC00070912D07072E000C880B990B0E94F8CBDF
:103FD00020E030E04AE754E40E9417CEAB01BC0178
:103FE00021E080917713909178130E94755660E6D6
:103FF00078E180917713909178130E9459576091DE
:104000002E0770912F07072E000C880B990B0E942A
:10401000F8CB20E030E04AE754E40E9417CEAB0131
:10402000BC0121E080917713909178130E9475561E
:1040300061E578E1809177139091781302C063E590
:1040400079E10E947D570E9409A680917713909193
:104050007813DC01ED91FC910680F781E02D199534
:1040600080917713909178130E9458560E941E9762
:104070006DEE79E180917713909178130E947D57CE
:104080000E941E9760EE79E18091771390917813EA
:104090000E945957E0910E13E6300CF0E6E08EE0F6
:1040A000D6011D928A95E9F78EEC99E19A8389836E
:1040B00087EB99E19C838B8385EA99E19E838D83CD
:1040C00086E999E198878F8383E899E19A878987C0
:1040D0008BE799E19C878B87EE0FFF0BEC0DFD1DA5
:1040E0006081718180917713909178130E947D5740
:1040F0000E9409A68091771390917813DC01ED91CD
:10410000FC910680F781E02D199520E834EA41E022
:1041100055272BAB3CAB4DAB5EAB809177139091A9
:1041200078130E9458560E941E9762E07CE18091AD
:104130007713909178130E947D570E941E9769EE25
:104140007BE180917713909178130E9459572091C9
:10415000F10B8091771390917813222319F065EE7B
:104160007BE102C060EE7BE10E947D578091F10B04
:10417000882349F167EC7BE1809177139091781364
:104180000E94595760910C1370910D13072E000C6B
:10419000880B990B0E94F8CB20E030E04AE754E40A
:1041A0000E9417CEAB01BC0122E080917713909161
:1041B00078130E94755662EC7BE1809177139091A1
:1041C00078130E947D5796E3E92E92E1F92E29E2B9
:1041D000622E3AE0232E312C44E6842E912CD70116
:1041E0002C91222309F4FFC1F7013297008111813C
:1041F0000115110509F4F7C18AED93EAA1E0BB2787
:10420000820F911DA11DB11DABBFFC0187917724C9
:104210007394811101C0712C209177133091781320
:10422000C8010197849790F562EA7BE1C9010E9479
:10423000595709500C3148F4E02FF0E0EE0FFF1F02
:10424000E15EFD4F6081718102C068EF79E180918C
:104250007713909178130E9459570C3130F4E02F66
:10426000F0E0E95AFD4F808101C080E090E088567F
:10427000944E092E000CAA0BBB0BABBFFC0187911F
:104280009EE0981B892F09F053C154C1C801845680
:1042900091098438934008F03FC068E87BE1C90188
:1042A0000E945957C801B4010E9469CF613071055D
:1042B00031F06230710559F464E87BE102C066E8D0
:1042C0007BE180917713909178130E9459570E9457
:1042D0001697A0907713B09078137720B1F0C801AB
:1042E0000E94C59C811107C060E87BE1C5010E9466
:1042F000595787E01DC1813009F01CC16DE77BE192
:10430000C5010E94595788E013C164E77BE1C501EC
:104310000E94595782E00CC1C801885E93408035E5
:10432000964408F05CC0C80168EE73E00E9469CF53
:104330005B0167E67BE1C9010E945957FAE0AF16BD
:10434000B10410F40E940E97B501809177139091FB
:1043500078130E9400720E94169740907713509035
:1043600078137720B1F1C8010E94C59C782E62E6CF
:104370007BE1C2010E945957672D8091771390917C
:1043800078130E943F706CE57BE1809177139091E8
:1043900078130E94595728E13CEFA29EC001A39ECA
:1043A000900DB29E900D1124800F911FB1010E94BB
:1043B0007DCF772780917713909178130E940072B8
:1043C0006AE57BE180917713909178130E945957A9
:1043D000B1C061E57BE1C2010E94595761C0F8019B
:1043E000E853FA44E83E43E0F40708F046C0EC30F6
:1043F000F10508F09FC08827EE58FF4F8F4F0C94AF
:1044000091CF62E47BE119C067E37BE1C9010E94BF
:10441000595783E18DC065E27BE127C065E17BE10F
:1044200016C068E07BE155C06CEF7AE1C9010E94DB
:10443000595782E17DC06DEE7AE1C9010E9459575A
:104440008FE076C06EED7AE1F8CF6EEC7AE1C901CB
:104450000E9459578EE06CC06BEB7AE1C9010E9453
:1044600059578BE065C069EA7AE1C9010E94595742
:104470008CE05EC06CE97AE12CC0C80180529E4499
:10448000883E934078F4005265E87AE1C9010E94C1
:1044900059570A3010F40E940E97802F0E94CF9631
:1044A00084E046C0C80188509245883E934020F47D
:1044B00008506EE67AE1EACF013FB5E51B0719F433
:1044C0006DE57AE11CC0023FE5E51E0739F460E5C1
:1044D0007AE1C9010E94595781E12AC0033FF5E5FD
:1044E0001F0739F462E47AE1C9010E94595780E15B
:1044F0001FC0043F45E5140739F461E37AE1C901BF
:104500000E9459578DE014C0053F55E5150739F451
:1045100069E17AE1C9010E94595786E009C0063F66
:10452000154541F460E07AE1C9010E94595785E0E0
:104530000E947AAC6DEB7BE18091771390917813B8
:104540000E94595762EB7BE1809177139091781329
:104550000E945957D7016C9170E080917713909128
:1045600078130E940072F70180818A3020F482E083
:104570000E947AAC04C0843610F40E940E970E9408
:104580001697D7014C91649EA0011124052E000CB2
:10459000660B770B8BA99CA9ADA9BEA9480F591F23
:1045A0006A1F7B1FD6018A019B010F5F1F4F2F4F90
:1045B0003F4F6BBFFA0187918D93B901A80181111B
:1045C000F2CFB60180917713909178130E945C56D8
:1045D0008091771390917813DC01ED91FC91068026
:1045E000F781E02D1995B3E0EB0EF11CEEEAEE1623
:1045F000E2E1FE0609F0F3CD0E9409A6809177134F
:1046000090917813DC01ED91FC910680F781E02D0B
:10461000199580917713909178130E9458560E94B3
:104620001E9763E67CE180917713909178130E9446
:104630007D570E941E9760E57CE1809177139091F1
:1046400078130E9459570E94B56B20E030E040E09B
:1046500050E40E94F1CB209177133091781387FFBB
:104660003FC06DE47CE1C90159C0F090E1120091B6
:10467000E41211E00C944E1863E675E18091771313
:10468000909178130E9459576091951480917713F7
:10469000909178130E943F7061E675E180917713E5
:1046A000909178130E9459570C94D71868E175E1DE
:1046B00080917713909178130E94595760919714C5
:1046C00080917713909178130E943F7066E175E1B5
:1046D00080917713909178130E9459570C94361952
:1046E00069E47CE1C9010E947D5766E37CE1809129
:1046F0007713909178130E9459570E94B56BAB01C4
:10470000BC0122E080917713909178130E94755636
:1047100064E37CE180917713909178130E947D5738
:1047200061E27CE180917713909178130E94595750
:10473000809158130E94DE96209158138091771330
:1047400090917813222379F06EE17CE10E94595711
:104750000E94B9AC64E17CE1809177139091781369
:104760000E947D5702C00E9458560E9409A680915F
:10477000771390917813DC01ED91FC910680F7811D
:10478000E02D199580917713909178130E945856D7
:104790000E941E976BEB7CE18091771390917813C8
:1047A0000E947D570E941E9767EA7CE180917713F3
:1047B000909178130E945957409148135091491392
:1047C00060914A1370914B138091771390917813F5
:1047D0000E94ED7163E97CE18091771390917813E9
:1047E0000E945957409150135091511360915213A8
:1047F0007091531380917713909178130E94ED710B
:104800006FE77CE180917713909178130E9459575C
:1048100040914C1350914D1360914E1370914F1372
:1048200080917713909178130E94ED716BE67CE193
:1048300080917713909178130E94595740915413A7
:1048400050915513609156137091571380917713BF
:10485000909178130E94ED710E9409A680917713C0
:1048600090917813DC01ED91FC910680F781E02DA9
:10487000199580917713909178130E9458560E9451
:104880001E97E6960FB6F894DEBF0FBECDBFDF9140
:10489000CF911F910F91FF90EF90DF90CF90BF903D
:1048A000AF909F908F907F906F905F904F903F90D0
:1048B0002F9008952F923F924F925F926F927F9226
:1048C0008F929F92AF92BF92CF92DF92EF92FF9220
:1048D0000F931F93CF93DF93CDB7DEB7AB970FB690
:1048E000F894DEBF0FBECDBF81EE91E00E942DCDCA
:1048F000683C7B498105910519F00E94704408C00D
:1049000045EE51E060E070E08DE891E10E9415CD48
:1049100040E052EC61E070E085ED99E00E94E277C2
:1049200040914C1350914D1360914E1370914F1361
:1049300088E399E00E94E27740915013509151131F
:1049400060915213709153138BE998E00E94E277C3
:104950004091541350915513609156137091571311
:104960008EEF97E00E94E2778BEA9EE09093F80743
:104970008093F7078CE69CE09093F6078093F50709
:1049800011E01093AD0E85ED99E09093A5148093FE
:10499000A4141092A6141092B10E1092AE0E1092A2
:1049A000B00E1092AF0E109384130E9489AB8091C9
:1049B0006D138093AE07109279131092800082E0FD
:1049C000809381008FE286BB10926F001092850069
:1049D000109284009BE29093A00099E09093A10034
:1049E00089BB109272001092A5001092A400109240
:1049F000A9001092A8001092AB001092AA00109289
:104A0000AD001092AC0099EA90932001109321011F
:104A10008ABB10927300109225011092240110920B
:104A200029011092280110922B0110922A01109254
:104A30002D0110922C0180912A1290912B128093BB
:104A4000430790934407813001F58FE38093140C62
:104A50001092150C61E00E94BF598AE09CE00E9410
:104A600048481092160C1092190C1092180C809154
:104A70004407882329F08AE09CE00E9463AC11C0BF
:104A80008AE09CE00E94024A0CC08091440788237F
:104A900011F062E001C060E08FE30E94BF590E9404
:104AA000576280912C1290912D1280934907909318
:104AB0004A07813001F58EE38093450C1092460C35
:104AC00061E00E94BF598BE39CE00E94484810922D
:104AD000470C10924A0C1092490C80914A07882387
:104AE00029F08BE39CE00E9463AC11C08BE39CE057
:104AF0000E94024A0CC080914A07882311F062E0AC
:104B000001C060E08EE30E94BF590E948C6C60E09F
:104B100085E40E94BF5962E08CE30E94BF5962E0C5
:104B20008BE30E94BF5962E080E40E94BF5962E0BB
:104B300081E40E94BF5962E082E40E94BF5962E0B2
:104B400081E20E94BF5962E084E40E94BF5961E0A3
:104B500089E30E94BF5961E08AE30E94BF590E9425
:104B60001F6A0E945B6A61E085E30E94BF5961E0B1
:104B700085E00E94BF5961E070E085E00E94FB592A
:104B800061E084E00E94BF5961E087E00E94BF5964
:104B900061E089E20E948F5961E089E20E94BF5979
:104BA000519A60E085E30E948F5960E085E00E94A1
:104BB0008F5960E084E00E948F5960E087E00E9496
:104BC0008F59599861E088E00E94BF5980E090E0D9
:104BD0009C0123573E4EF901E755FF4F40814F3668
:104BE00029F4329720813181232B31F403968837C1
:104BF000910571F760E001C061E088E00E948F5983
:104C000061E08DE20E94BF5961E08EE20E94BF59CF
:104C100061E08CE20E94BF5961E08BE20E94BF59C3
:104C200060E08BE20E948F5962E08CE00E94BF59E5
:104C300062E08EE10E94BF5962E08FE10E94BF599D
:104C400062E080E20E94BF5962E082E20E94BF59A6
:104C500062E083E20E94BF5962E084E20E94BF5991
:104C600062E085E20E94BF5962E086E20E94BF597D
:104C700062E087E30E94BF5962E088E30E94BF5967
:104C800062E08DE30E94BF5962E088E20E94BF5952
:104C900062E087E20E94BF5962E083E40E94BF594C
:104CA00062E08AE20E94BF5962E08FE20E94BF592F
:104CB00062E080E30E94BF5962E081E30E94BF5935
:104CC0006A98729A5498559856985C9A5D9A5E9A2A
:104CD0006F98779A9B989C98A39AA49A80910101C7
:104CE0008B7F80930101809101018F778093010177
:104CF00080910201846080930201809102018068AA
:104D000080930201809104018B7F80930401809144
:104D10000401877F80930401809104018F7E80933A
:104D20000401809104018F7D80930401809104012E
:104D30008F7B80930401809104018F77809304011D
:104D40008091050184608093050180910501886050
:104D50008093050180910501806180930501809118
:104D60000501806280930501809105018064809334
:104D70000501809105018068809305010E945B6AAE
:104D80000E947E718091FA0B813009F058C08091A9
:104D9000FD0B9091FE0BA091FF0BB091000C409188
:104DA000010C5091020C6091030C7091040C841B57
:104DB000950BA60BB70B84379E40A105B10500F3F8
:104DC0000E9470440E9408970E9408970E941E97B4
:104DD00069EC7CE180917713909178130E94595788
:104DE00001E010E00E94236A0E945B6A6EEE72E0AE
:104DF00080E090E00E94C38666EC7CE180917713AE
:104E0000909178130E9459570E941F6A0E94576A16
:104E10000530110531F064EF71E080E090E00E9410
:104E2000C3860F5F1F4F06301105E1F60E940897F9
:104E30000E941E970E9408970E94089702C0811145
:104E40009FCF80916F00826080936F00809184007B
:104E5000909185008056904F9093890080938800B0
:104E60000E947F338DE69CE09093B9148093B81430
:104E700010910613209105138091F4129091F6126F
:104E80003091F7123093FD07909312078093130728
:104E900030E0AFEFB0E00E949BCD24E630E040E090
:104EA00050E00E9447CD20939914612F70E080E07C
:104EB00090E00E94F6CB20ED34E448E55BE30E94ED
:104EC00057CC26E636E646E25FE30E94ABCD609320
:104ED000F9077093FA078093FB079093FC071093F0
:104EE00098141092950010929400109290008CE00B
:104EF0008093910084EF90E09093990080939800C4
:104F000081E088BB82E080937100809100020E9462
:104F10007D6680910E13863040F010920E1360E093
:104F200070E081E891E00E940F7110910E13123031
:104F300009F444C008F5112309F466C0113009F0E2
:104F40005BC08CE090E00E94A8CF2BE433E0DC0152
:104F500011963C932E932BE938E01B963C932E93AD
:104F60001A979093AB078093AA071093321410936B
:104F700035141093381467C0133009F45EC0143030
:104F8000D9F586E090E00E94A8CF8C0125EB33E0B4
:104F9000DC012D933D93CD0141E06DE67CE00E9464
:104FA000499A87E792E0F801918380831093AB07D9
:104FB0000093AA0781E08093321441C086E090E01C
:104FC0000E94A8CF21EE32E0FC0131832083909330
:104FD000AB078093AA078FB7F8942CED35E0309398
:104FE000CB102093CA101092D0108FBF81E0809315
:104FF00032148093351425C010920E1360E070E0D7
:1050000081E891E00E940F7186E090E00E94A8CFB5
:105010008C0125EB33E0DC012D933D93CD0140E085
:105020006DE67CE00E94499A87E792E0F80191835F
:1050300080831093AB070093AA071092321410924A
:105040003514109238148091AA079091AB07DC01B7
:10505000ED91FC910190F081E02D1995809126143D
:1050600081112FC08091291481112BC080912C14A3
:10507000811127C080912F14811123C08091321497
:1050800081111FC08091351481111BC0809138148B
:10509000811117C020915C1330E0AFEFB0E00E94A7
:1050A0009BCD24E630E040E050E00E9447CD2093C5
:1050B0007E0F80915B13882309F40BC30E94BB6AA7
:1050C00008C3A12CB12C1DA2412C912C512C612C78
:1050D000812C712C03E616E0EE24EA94A3E0FA2E6C
:1050E000CC24CA94DD24D39487E5282E86E0382E7C
:1050F000C50183579E4EFC01E755FF4FE081EE232B
:1051000009F4DEC2DC01A955BF4F8D919C91892B1A
:1051100009F4D6C28E2F90E0FC01F797EB32F1052F
:1051200008F0CEC28827E258FF4F8F4F0C9491CFE2
:1051300080912614882309F4C3C27110C1C289E189
:1051400090E00E94A8CF9C01FC011183008387E0BE
:1051500090E09383828315821482F782E682D1865F
:10516000C086108EC9012AA73BA70E949C502AA581
:105170003BA5E7E3F4E0D901ED93FC9330931714DA
:1051800020931614C9010E94057F7DC180912914C6
:10519000882309F495C2811093C289E190E00E94AE
:1051A000A8CF9C01DC0111961C930E93E6E0F0E081
:1051B0001396FC93EE93129715961C921E921497D9
:1051C0001796FC92EE9216971996DC92CE9218974B
:1051D00058961C922AA73BA70E949C502AA53BA543
:1051E000E7E3F4E0D901ED93FC9330931914209395
:1051F0001814C9010E94057F74C180912C14882362
:1052000009F45EC261105CC289E190E00E94A8CFFF
:105210009C01DC0111961C930E93E5E0F0E01396DF
:10522000FC93EE93129715961C921E921497179664
:10523000FC92EE9216971996DC92CE921897589699
:105240001C922AA73BA70E949C502AA53BA5E7E3F6
:10525000F4E0D901ED93FC9330931B1420931A14BE
:10526000C9010E94057F6BC180912F14882309F426
:1052700027C2511025C289E190E00E94A8CF9C016D
:10528000DC0111961C930E93E4E0F0E01396FC937E
:10529000EE93129715961C921E9214971796FC92F5
:1052A000EE9216971996DC92CE92189758961C9209
:1052B0002AA73BA70E949C502AA53BA5E7E3F4E060
:1052C000D901ED93FC9330931D1420931C14C90154
:1052D0000E94057F62C180913214882309F4F0C1D5
:1052E0009110EEC189E190E00E94A8CF9C01DC0101
:1052F00011961C930E93E2E0F0E01396FC93EE936C
:10530000129715961C921E9214971796FC92EE9285
:1053100016971996DC92CE92189758961C922AA747
:105320003BA70E949C502AA53BA5E7E3F4E0D901E6
:10533000ED93FC9330931F1420931E14C9010E9417
:10534000057F59C180913514882309F4B9C14110F2
:10535000B7C189E190E00E94A8CF9C01DC011196C1
:105360001C930E93E1E0F0E01396FC93EE931297FA
:1053700015961C921E9214971796FC92EE92169711
:105380001996DC92CE92189758961C922AA73BA7A2
:105390000E949C502AA53BA5E7E3F4E0D901ED93D8
:1053A000FC933093211420932014C9010E94057F9F
:1053B00050C180913814882309F482C12DA1211194
:1053C0007FC189E190E00E94A8CF9C01DC01119689
:1053D0001C930E9313961C921E92129715961C9274
:1053E0001E9214971796FC92EE9216971996DC92DD
:1053F000CE92189758961C922AA73BA70E949C50C1
:105400002AA53BA587E394E0F9019183808330933B
:10541000231420932214C9010E94057F4FC180915B
:105420002614882309F44CC171104AC18CE190E024
:105430000E94A8CF9C01DC0111961C930E93E7E01B
:10544000F0E01396FC93EE93129715961C921E9221
:1054500014971796FC92EE9216971996DC92CE92BC
:10546000189758961C922AA73BA70E949C502AA5E1
:105470003BA5D9012D923C923093251420932414FE
:10548000C9010E94A57F772473941AC180912914C1
:10549000882309F415C1811013C18CE190E00E94AA
:1054A000A8CF9C01FC011183008386E090E09383E8
:1054B000828315821482F782E682D186C086108E9E
:1054C000C9012AA73BA70E949C502AA53BA5D90148
:1054D0002D923C923093281420932714C9010E94E6
:1054E000A57F88248394ECC080912C14882309F430
:1054F000E7C06110E5C08CE190E00E94A8CF9C015C
:10550000FC011183008385E090E093838283158200
:105510001482F782E682D186C086108EC9012AA73E
:105520003BA70E949C502AA53BA5D9012D923C92F5
:1055300030932B1420932A14C9010E94A57F66245E
:105540006394BEC080912F14882309F4B9C0511010
:10555000B7C08CE190E00E94A8CF9C01FC011183B0
:10556000008384E090E09383828315821482F78223
:10557000E682D186C086108EC9012AA73BA70E9469
:105580009C502AA53BA5D9012D923C9230932E1414
:1055900020932D14C9010E94A57F5524539490C0D7
:1055A00080913214882309F48BC0911089C08CE15A
:1055B00090E00E94A8CF9C01FC011183008382E04F
:1055C00090E09383828315821482F782E682D186EB
:1055D000C086108EC9012AA73BA70E949C502AA50D
:1055E0003BA5D9012D923C92309331142093301475
:1055F000C9010E94A57F9924939462C080913514BB
:10560000882309F45DC041105BC08CE190E00E94EA
:10561000A8CF9C01FC011183008381E090E093837B
:10562000828315821482F782E682D186C086108E2C
:10563000C9012AA73BA70E949C502AA53BA5D901D6
:105640002D923C923093341420933314C9010E945C
:10565000A57F4424439434C080913814882381F179
:105660002DA121112DC08CE190E00E94A8CF9C01BA
:10567000DC0111961C930E9313961C921E921297A6
:1056800015961C921E9214971796FC92EE921697FE
:105690001996DC92CE92189758961C922AA73BA78F
:1056A0000E949C502AA53BA5F901318220823093AB
:1056B000371420933614C9010E94A57F21E02DA341
:1056C00083E0A80EB11C98E7A916B10409F010CD2B
:1056D000E1CC8091D812813059F480916B138823EA
:1056E00039F010926B1360E08EED91E00E946B72C6
:1056F0008091D812813059F480916813882339F051
:105700001092681360E08BED91E00E946B728091C3
:105710006813882359F080916B13882339F0109215
:105720006B1360E08EED91E00E946B7281E00E944D
:1057300084AB882339F082E00E9484AB882311F087
:105740001FA216C081E00E9484AB882329F082E06A
:105750000E9468AB81118AC78CE30E946659892B2D
:1057600009F075C78CE30E946659892B09F075C74B
:1057700086E0EEE3F3E1DE01549601900D928A9506
:10578000E1F78091371390914713B090381300914F
:10579000391310913A1370913B1360913C1350915F
:1057A0003D13409144132091451330914613A0912D
:1057B000AA07B091AB07BEA3ADA3E0918214F0910C
:1057C0008314F9A7E8A790906A1360906513E0909E
:1057D0005E13F0905F138090681370906713C09011
:1057E000C212D090C3125090C5124090C012309097
:1057F000C112FFA1FB8B8A8F9B8FBC8E0D8F1E8FDA
:105800007F8F68A359A34AA33CA32BA3F2E1AF2E39
:10581000FE017396DE01119601900D92AA94E1F7B4
:10582000EDE6FCE0F0931C07E0931B07AFA1A98312
:1058300088879987BA860B871C877D876E875F87E5
:10584000488B3A8B298B22E1FE013196ABE2B7E01F
:1058500001900D922A95E1F7992321F0863011F0FD
:10586000109233073092E9134092EA135092781461
:10587000D0927114C0927014609284147092751456
:1058800080927414F0927314E09272149092E81360
:1058900088A599A590937714809376148DA19EA1E5
:1058A00090931E0780931D0787E08093F60A10925D
:1058B000F70A61E00E94BF598CEE9AE00E944848C6
:1058C0001092F80A1092FB0A1092FA0A8091360799
:1058D000811102C01092370790913207911105C0D3
:1058E000811103C01092E10B98C08091DC0B909164
:1058F000DD0B0E94C2A181E08093E10B80912B0718
:10590000882359F1813071F08330C1F488E293E249
:1059100090932D0780932C0789E08093300780E1D6
:1059200097E217C088EB9BE090932D0780932C079C
:1059300083E08093300788E99AE30BC088E893E11D
:1059400090932D0780932C0786E08093300780EE9C
:105950009EE290932F0780932E0780913207882331
:10596000E9F1809136076091300770E08823C9F033
:10597000809138078823A9F080E090E00E94F6CB60
:105980009B01AC0160E070E088EC92E40E9417CECD
:1059900060931F077093200780932107909322073D
:1059A00025C080E090E00E94F6CB9B01AC0160E056
:1059B00070E088EC92E40E9417CE60931F0770930A
:1059C00020078093210790932207109216071092C8
:1059D000170710921807109219071FC010921F077F
:1059E0001092200710922107109222076091310730
:1059F00070E080E090E00E94F6CB9B01AC0160E09B
:105A000070E088EC92E40E9417CE609316077093C2
:105A10001707809318079093190710928A11109214
:105A2000230710921A07109224071092250710924C
:105A30002607109227070E9446835098589AE898A4
:105A4000809169008C7F809369008091EA1388239C
:105A500021F080916900826003C0809169008360B9
:105A6000809369006E98769AE8980E94028680E09A
:105A700090E040E09C0123573E4EF901E755FF4F6F
:105A80005081552331F0329720813181232B09F049
:105A90004F5F03968837910569F740933E07ABE463
:105AA000B7E020E030E084EC282E8EE9382E94E830
:105AB000492E91E6592E49E5642E41E6742E5CE6A6
:105AC000852E51E6952E67ECA62E6EE9B62E40E0A7
:105AD00055E909EC1EE976EDE72E7EE9F72EEAE4BA
:105AE000CE2EE4E9DE2EC90183579E4EFC01E75518
:105AF000FF4F6081662309F4B0C389559F4FFC01B5
:105B000080819181892B09F4A8C370E0FB01319752
:105B1000E53AF10508F0A1C38827E755FF4F8F4FFD
:105B20000C9491CF8EE59CE911969C938E9395C32E
:105B30008CE59CE911969C938E938FC38AE59CE932
:105B400011969C938E9389C382E59CE911969C9350
:105B50008E9383C38FE49CE911969C938E937DC3AF
:105B600089EB9BE911969C938E9377C383EC9BE919
:105B700011969C938E9371C38CE99BE911969C932B
:105B80008E936BC388E89BE911969C938E9365C3B3
:105B900089E79BE911969C938E935FC38DE19BE906
:105BA00011969C938E9359C384ED9AE911969C9318
:105BB0008E9353C387EC9AE911969C938E934DC3B1
:105BC0008AEB9AE911969C938E9347C388EB9AE9E6
:105BD00011969C938E9341C380EC91EA11969C930D
:105BE0008E933BC389EB91EA11969C938E9335C3B8
:105BF00082E891EA11969C938E932FC38AEA91EAE8
:105C000011969C938E9329C383EA91EA11969C93F3
:105C10008E9323C38BE791EA11969C938E931DC3B9
:105C200089E791EA11969C938E9317C387E791EACF
:105C300011969C938E9311C387E691EA11969C93DB
:105C40008E930BC385E691EA11969C938E9305C3C0
:105C500083E691EA11969C938E93FFC28CE591EABC
:105C600011969C938E93F9C28AE591EA11969C93C2
:105C70008E93F3C288E591EA11969C938E93EDC2C0
:105C800085EA9EE911969C938E93E7C283EA9EE98A
:105C900011969C938E93E1C281EA9EE911969C93A2
:105CA0008E93DBC284EF97E611969C938E93D5C2B8
:105CB00086E591EA11969C938E93CFC286E491EA91
:105CC00011969C938E93C9C280EC9FE911969C9388
:105CD0008E93C3C281EA9FE911969C938E93BDC2B5
:105CE00084E491EA11969C938E93B7C285E191EA80
:105CF00011969C938E93B1C28EE091EA11969C937B
:105D00008E93ABC28DED90EA11969C938E93A5C2B3
:105D100085E69CE911969C938E939FC28BED90EA49
:105D200011969C938E9399C289ED90EA11969C935B
:105D30008E9393C286ED90EA11969C938E938DC2BA
:105D400082EB90EA11969C938E9387C28EE890EA3C
:105D500011969C938E9381C283ED90EA11969C9349
:105D60008E937BC28FEA90EA11969C938E9375C2B4
:105D70008BE890EA11969C938E936FC280ED90EA27
:105D800011969C938E9369C28CEA90EA11969C932B
:105D90008E9363C288E890EA11969C938E935DC2BD
:105DA0008DEC90EA11969C938E9357C289EA90EA03
:105DB00011969C938E9351C285E890EA11969C931C
:105DC0008E934BC28AEC90EA11969C938E9345C2B7
:105DD00086EA90EA11969C938E933FC282E890EAFD
:105DE00011969C938E9339C287EC90EA11969C93FE
:105DF0008E9333C283EA90EA11969C938E932DC2C0
:105E00008FE790EA11969C938E9327C284EC90EAD8
:105E100011969C938E9321C280EA90EA11969C93EE
:105E20008E931BC28CE790EA11969C938E9315C2B9
:105E300081EC90EA11969C938E930FC28DE990EAC3
:105E400011969C938E9309C289E790EA11969C93D0
:105E50008E9303C28EEB90EA11969C938E93FDC1B4
:105E60008AE990EA11969C938E93F7C186E790EAAF
:105E700011969C938E93F1C18BEB90EA11969C93B3
:105E80008E93EBC187E990EA11969C938E93E5C1BE
:105E900083E790EA11969C938E93DFC188EB90EA9A
:105EA00011969C938E93D9C184E990EA11969C93A4
:105EB0008E93D3C180E790EA11969C938E93CDC1C7
:105EC00085EB90EA11969C938E93C7C181E990EA85
:105ED00011969C938E93C1C18DE690EA11969C9386
:105EE0008E93BBC183EE9EE911969C938E93B5C1B0
:105EF00089E690EA11969C938E93AFC185E690EA6D
:105F000011969C938E93A9C181E690EA11969C9379
:105F10008E93A3C18DE590EA11969C938E939DC1BB
:105F200089E590EA11969C938E9397C185E590EA56
:105F300011969C938E9391C181E590EA11969C9362
:105F40008E938BC18DE490EA11969C938E9385C1BC
:105F500084E490EA11969C938E937FC18FE99EE929
:105F600011969C938E9379C18DE99EE911969C932D
:105F70008E9373C18DE090EA11969C938E936DC1C0
:105F80008FE49FE911969C938E9367C18BE390EA0F
:105F900011969C938E9361C18BE99EE911969C9317
:105FA0008E935BC189E99EE911969C938E9355C1AE
:105FB0008FED9FE911969C938E934FC18DEF9EE9D3
:105FC00011969C938E9349C18BEE95E911969C9303
:105FD0008E9343C180EA95E911969C938E933DC1BF
:105FE00088EB91E611969C938E9337C184EA91E6F3
:105FF00011969C938E9331C180E991E611969C9302
:106000008E932BC18EEA9CE911969C938E9325C1A9
:1060100087EB96E911969C938E931FC18AEA96E9C5
:1060200011969C938E9319C180E996E911969C93E1
:106030008E9313C18EE696E911969C938E930DC1B3
:106040008EE896E911969C938E9307C180E796E9B6
:1060500011969C938E9301C188E394E911969C93C9
:106060008E93FBC08CEE93E911969C938E93F5C0B2
:106070008EE094E911969C938E93EFC08EEF93E996
:1060800011969C938E93E9C080E294E911969C93BB
:106090008E93E3C082EC93E911969C938E93DDC0BE
:1060A00082EB93E911969C938E93D7C084ED93E98C
:1060B00011969C938E93D1C084E995E911969C9397
:1060C0008E93CBC088E895E911969C938E93C5C0BA
:1060D0008CE795E911969C938E93BFC080E795E974
:1060E00011969C938E93B9C084E695E911969C9382
:1060F0008E93B3C088E595E911969C938E93ADC0BD
:106100008CE495E911969C938E93A7C086EB94E955
:1061100011969C938E93A1C084EA94E911969C9366
:106120008E939BC082E994E911969C938E9395C0BF
:1061300080E894E911969C938E938FC08EE694E943
:1061400011969C938E9389C08CE594E911969C934B
:106150008E9383C01196DC92CE927FC01196FC92F2
:10616000EE927BC011961C930E9377C086E295E960
:1061700011969C938E9371C011965C934E936DC053
:106180001196BC92AE9269C011969C928E9265C097
:1061900011967C926E9261C011965C924E925DC097
:1061A00011963C922E9259C0E1ECFEE91196FC93B7
:1061B000EE9353C088EB9EE911969C938E934DC04D
:1061C000E5EBFEE91196FC93EE9347C082EB9EE966
:1061D00011969C938E9341C0EFEAFEE91196FC93D1
:1061E000EE933BC08CEA9EE911969C938E9335C04A
:1061F000E4ECF6E91196FC93EE932FC08DEC96E952
:1062000011969C938E9329C0E6ECF6E91196FC93C7
:10621000EE9323C082EE94E911969C938E931DC059
:10622000E5EDF4E91196FC93EE9317C088EC94E940
:1062300011969C938E9311C0E9E4F6E91196FC93B4
:10624000EE930BC086E396E911969C938E9305C05E
:10625000ECE5F6E91196FC93EE932D5F3F4F129615
:106260002837310509F03FCC10923F078091430752
:10627000811114C080E090E0FC01EC5CFD4E2081B7
:106280003181245631092436310528F003968837A8
:10629000910591F703C081E080933F071092450775
:1062A00080914907811114C080E090E0FC01EC5C12
:1062B000FD4E20813181285C31092436310528F0DA
:1062C00003968837910591F703C081E080934507D5
:1062D0008091AA079091AB07DC01ED91FC91EE5AF9
:1062E000FF4F209111133091121340910F135091D1
:1062F00010130190F081E02D61E019958091AA07BB
:106300009091AB07DC01ED91FC91EE5AFF4F20918B
:1063100015133091161340911313509114130190DB
:10632000F081E02D62E019958091AA079091AB076A
:10633000DC01ED91FC91EE5AFF4F20911913309141
:106340001A1340911713509118130190F081E02D0A
:1063500063E019958091AA079091AB07DC01ED915C
:10636000FC91EE5AFF4F2091241330912513409158
:106370002213509123130190F081E02D64E01995D0
:106380008091AA079091AB07DC01ED91FC91EE5A48
:10639000FF4F2091281330912913409126135091DB
:1063A00027130190F081E02D65E019958091AA07EF
:1063B0009091AB07DC01ED91FC91EE5AFF4F2091DB
:1063C0002C1330912D1340912A1350912B130190CF
:1063D000F081E02D66E019958091AA079091AB07B6
:1063E000DC01ED91FC91EC5AFF4F0190F081E02D22
:1063F00040911B1361E019958091AA079091AB071A
:10640000DC01ED91FC91EC5AFF4F0190F081E02D01
:1064100040911C1362E019958091AA079091AB07F7
:10642000DC01ED91FC91EC5AFF4F0190F081E02DE1
:1064300040911D1363E019958091AA079091AB07D5
:10644000DC01ED91FC91EC5AFF4F0190F081E02DC1
:1064500040912E1364E019958091AA079091AB07A3
:10646000DC01ED91FC91EC5AFF4F0190F081E02DA1
:1064700040912F1365E019958091AA079091AB0781
:10648000DC01ED91FC91EC5AFF4F0190F081E02D81
:106490004091301366E019958091AA079091AB075F
:1064A000DC01ED91FC9102ACF3ADE02D60911F1386
:1064B00019958091AA079091AB07DC01ED91FC91B1
:1064C00006ACF7ADE02D6091341319958091AA07C1
:1064D0009091AB07DC01ED91FC9100A8F1A9E02DB2
:1064E0006091201319958091AA079091AB07DC0168
:1064F000ED91FC9106A8F7A9E02D60912113199563
:106500008091AA079091AB07DC01ED91FC91E65BCD
:10651000FF4F0190F081E02D4091351360E0199517
:106520008091AA079091AB07DC01ED91FC91E65BAD
:10653000FF4F0190F081E02D4091361361E01995F5
:1065400080E090E09C0123573E4EF901E755FF4F54
:106550004081423731F4329720813181232B09F079
:106560008BC003968837910569F70E94C39D80917F
:10657000AA079091AB07DC01ED91FC91EC59FF4F1C
:106580000190F081E02D40E06091311319958091E8
:10659000AA079091AB07DC01ED91FC91EC59FF4FFC
:1065A0000190F081E02D41E06091331319958091C5
:1065B000AA079091AB07DC01ED91FC91EC59FF4FDC
:1065C0000190F081E02D42E06091321319950E9414
:1065D000E8AC0E94FD866B017C0110E011110FC038
:1065E0008091AE07882359F02FEE34E940ED57E053
:1065F00060E070E08DE69CE00E94DA4D11E00E94C0
:106600008682882351F00E94D56A0E94DE620E9431
:106610005B6A0E9412820E94E6690E9433AA029776
:1066200011F00E94645E0E9409A60E9433AA02979C
:10663000A9F60E94FD86DC01CB018C199D09AE09EB
:10664000BF098C3B9240A105B10540F218C082E021
:106650000E9484AB81110DC085C882E00E9468ABA6
:10666000882309F485C8E3E0EFA382C8A1E0AFA3C3
:106670007FC8B2E0BFA37CC80E94B79D78CF0E94BC
:10668000B37D0E945B6A8091F50B811102C00E946C
:1066900085720E9406AA86E30E947F86BC01990F3C
:1066A000880B990B611571058105910511F00E9408
:1066B0006CCB62E086E30E94BF592DEA33E948EED5
:1066C00053E060E070E08DE69CE0AB960FB6F89486
:1066D000DEBF0FBECDBFDF91CF911F910F91FF9015
:1066E000EF90DF90CF90BF90AF909F908F907F9072
:1066F0006F905F904F903F902F900C94DA4D5F9287
:106700006F927F928F929F92AF92BF92CF92DF92C1
:10671000EF92FF920F931F93CF93DF9381E08093CB
:1067200026148093291480932C1480932F14809323
:106730003B1480933E149091F7129150963040F0A4
:106740008093F71261E070E08AE691E00E940F7199
:106750009091F7122DEF290F8091AC12233008F0A1
:1067600011C28A3079F03CF4883009F463C0893072
:1067700009F4C0C1B6C18B3009F4A4C08C3009F44F
:10678000E6C0AFC184E290E00E94A8CFFC018091F6
:106790006C1328E030E03383228388248394992487
:1067A0009A9495828482AA24AA94B12CB782A68254
:1067B00011861086108E93E8792E718E2BE9C22EE9
:1067C00028E0D22ED38EC28E37E6E32E34E0F32EAD
:1067D000F182E082C0E5D3E1D1A3C0A312A283A3DA
:1067E000F093A007E0939F07CF010E942C8E84E2D4
:1067F00090E00E94A8CFFC0180916C1329E030E06A
:106800003383228395828482B782A6821186108682
:10681000108E718ED38EC28EF182E082D1A3C0A37E
:1068200012A283A3F0939E07E0939D07CF010E94DD
:106830002C8E0EC380E290E00E94A8CFFC0188E07D
:1068400090E0938382838824839499249A949582F8
:106850008482AA24AA94B12CB782A68211861086BB
:10686000108EAAE0DA2ED18EBBE9EB2EB8E0FB2E1B
:10687000F38EE28ECFE4D4E0D183C083F093A007FF
:10688000E0939F07CF010E94CC8080E290E00E94BD
:10689000A8CFFC0189E090E0938382839582848273
:1068A000B782A68211861086108ED18EF38EE28E6C
:1068B000D183C083F0939E07E0939D07CF010E9490
:1068C000CC80C6C289E190E00E94A8CFFC0188E09C
:1068D00090E093838283CC24C394DD24DA94D58220
:1068E000C482EE24EA94F12CF782E68211861086A7
:1068F000108EC3E4D4E0D183C083F093A007E0936B
:106900009F07CF010E94CF7F10923B148091F71216
:10691000843009F09DC289E190E00E94A8CFFC017B
:1069200089E090E093838283D582C482F782E682F5
:1069300011861086108ED183C083F0939E07E0935A
:106940009D07CF010E94CF7F10923E1481C29430E8
:1069500009F04BC089E190E00E94A8CFEC0183E6EA
:10696000882E86E0982E9982888287E090E09B832B
:106970008A83AA24A394BB24BA94BD82AC82CC247B
:10698000CA94D12CDF82CE8219861886188ECE0149
:106990000E949C5037E3E32E34E0F32EF982E88224
:1069A000D093A007C0939F07CE010E94057F10924D
:1069B000261489E190E00E94A8CFEC019982888298
:1069C00086E090E09B838A83BD82AC82DF82CE82A8
:1069D00019861886188ECE010E949C50F982E88292
:1069E000D0939E07C0939D074DC0953009F050C0CD
:1069F00089E190E00E94A8CFEC01E3E68E2EE6E06C
:106A00009E2E9982888287E090E09B838A83AA24C5
:106A1000A394BB24BA94BD82AC82CC24CA94D12C5A
:106A2000DF82CE8219861886188ECE010E949C5075
:106A3000B7E3EB2EB4E0FB2EF982E882D0939E07F9
:106A4000C0939D07CE010E94057F1092261489E114
:106A500090E00E94A8CFEC019982888286E090E0C5
:106A60009B838A83BD82AC82DF82CE8219861886A0
:106A7000188ECE010E949C50F982E882D093A00724
:106A8000C0939F07CE010E94057F10922914E0C198
:106A900089E190E00E94A8CFEC0183E696E099831B
:106AA000888387E090E09B838A8381E09FEF9D83CA
:106AB0008C838FEF90E09F838E8319861886188EC3
:106AC000CE010E949C5087E394E099838883D09301
:106AD000A007C0939F07CE010E94057F1092261445
:106AE000B7C189E08093AC1269E070E08FE191E07A
:106AF0000E940F7180E290E00E94A8CFFC0188E024
:106B000090E0938382838824839499249A94958235
:106B10008482AA24AA94B12CB782A68211861086F8
:106B2000108E60E8D62ED18E7BE9E72E78E0F72E26
:106B3000F38EE28ECBE5D4E0D183C083F093A0073F
:106B4000E0939F07CF010E94D78D80E290E00E94E2
:106B5000A8CFFC0189E090E09383828395828482B0
:106B6000B782A68211861086108ED18EF38EE28EA9
:106B7000D183C083F0939E07E0939D07CF010E94CD
:106B8000D78D66C18A3009F458C03CF4883009F4C6
:106B9000A2C0893009F405C1FBC08B3009F4BEC026
:106BA0008C3009F0F5C089E190E00E94A8CFEC019B
:106BB00093E6892E96E0992E9982888287E090E06C
:106BC0009B838A83AA24A394BB24BA94BD82AC82FB
:106BD000CC24CA94D12CDF82CE8219861886188ED6
:106BE000CE010E949C5047E3E42E44E0F42EF9824B
:106BF000E882D093A207C093A10789E190E00E94A8
:106C0000A8CFEC019982888286E090E09B838A83FA
:106C1000BD82AC82DF82CE8219861886188ECE01A4
:106C20000E949C50F982E882D093A407C093A307E6
:106C30001092261410922914F5C084E290E00E946C
:106C4000A8CFFC0170906C136090031388E090E073
:106C5000938382838824839499249A94958284824E
:106C6000AA24AA94B12CB782A68211861086108E0F
:106C700093E8592E518E2BE9C22E28E0D22ED38EC6
:106C8000C28E37E6E32E34E0F32EF182E082C0E5D7
:106C9000D3E1D1A3C0A362A273A2F093A207E093B1
:106CA000A10784E290E00E94A8CFFC0189E090E077
:106CB0009383828395828482B782A682118610860E
:106CC000108E518ED38EC28EF182E082D1A3C0A3EA
:106CD00062A273A2A3C080E290E00E94A8CFFC0150
:106CE00088E090E0938382838824839499249A9403
:106CF00095828482AA24AA94B12CB782A682118696
:106D00001086108EBAE0DB2ED18ECBE9EC2EC8E0D7
:106D1000FC2EF38EE28ECFE4D4E065C089E190E0F2
:106D20000E94A8CFFC0188E090E093838283CC246A
:106D3000C394DD24DA94D582C482EE24EA94F12C43
:106D4000F782E68211861086108EC3E4D4E0D183E8
:106D5000C083F093A207E093A10789E190E00E942D
:106D6000A8CFFC0189E090E093838283D582C4821E
:106D7000F782E68211861086108ED183C083F0934D
:106D8000A407E093A30710923B1410923E144AC04C
:106D900089E08093AC1269E070E08FE191E00E949D
:106DA0000F7180E290E00E94A8CFFC0188E090E0A3
:106DB000938382838824839499249A9495828482ED
:106DC000AA24AA94B12CB782A68211861086108EAE
:106DD000D0E8DD2ED18E8BE9E82E88E0F82EF38EF8
:106DE000E28ECBE5D4E0D183C083F093A207E09399
:106DF000A10780E290E00E94A8CFFC0189E090E02A
:106E00009383828395828482B782A68211861086BC
:106E1000108ED18EF38EE28ED183C083F093A407BF
:106E2000E093A3078091A3079091A407DC01ED9163
:106E3000FC910280F381E02D19958091A10790913A
:106E4000A207DC01ED91FC910280F381E02D199500
:106E50008091F712833039F0823009F06CC0809154
:106E6000AC128C3051F189E190E00E94A8CFEC0186
:106E700083E696E09983888386E090E09B838A830B
:106E800081E09FEF9D838C838FEF90E09F838E83C3
:106E900019861886188ECE010E949C5087E394E0D4
:106EA00099838883D0939C07C0939B07CE010E944F
:106EB000057F10922914C6E029C089E190E00E9464
:106EC000A8CFEC0183E696E09983888384E090E084
:106ED0009B838A8381E09FEF9D838C838FEF90E07B
:106EE0009F838E8319861886188ECE010E949C502F
:106EF00087E394E099838883D0939C07C0939B0792
:106F0000CE010E94057F10922F14C4E06091BB1245
:106F10007091BC128C2F0E94B24F6091BD12709183
:106F2000BE128C2F0E94AD4F8091BF12E0919B0743
:106F3000F0919C07808FE091AD128E2FEE0F990B90
:106F4000AA0BBB0BFC013897E830F10508F0BBC079
:106F50008827E25BFE4F8F4F0C9491CF84E290E044
:106F60000E94A8CFFC0180916C1328E030E03383AD
:106F7000228321E03FEF358324832FEF30E03783F6
:106F8000268311861086108E94E8918F2BE938E0C5
:106F9000338F228F27E634E03183208320E533E1ED
:106FA00031A320A312A283A31EC080E290E00E941E
:106FB000A8CFFC0188E090E09383828381E09FEF7B
:106FC000958384838FEF90E0978386831186108664
:106FD000108E87E8818F8BE998E0938F828F8BE505
:106FE00094E091838083F093A907E093A80799C068
:106FF00080E290E00E94A8CFFC0188E090E09383BB
:10700000828381E09FEF958384838FEF90E0978365
:10701000868311861086108E8DE0818F8BE998E033
:10702000938F828F8FE494E0DCCF89E190E00E941F
:10703000A8CFFC0188E090E09383828381E09FEFFA
:10704000958384838FEF90E09783868311861086E3
:10705000108E83E494E091838083F093A907E093FA
:10706000A80710923B145DC08CE190E00E94A8CF6D
:10707000EC0183E696E09983888385E090E09B832A
:107080008A8381E09FEF9D838C838FEF90E09F83C5
:107090008E8319861886188ECE010E949C5087E533
:1070A00096E037C089E190E00E94A8CFFC011382EE
:1070B0001282158214821782168211861086108E13
:1070C0008FE194E08ECF8CE08093AD126CE070E0A5
:1070D00080E291E00E940F7189E190E00E94A8CFC8
:1070E000EC0183E696E09983888385E090E09B83BA
:1070F0008A8381E09FEF9D838C838FEF90E09F8355
:107100008E8319861886188ECE010E949C5087E3C4
:1071100094E099838883D093A907C093A80710921D
:107120002C148091A8079091A907DC01ED91FC91A6
:107130000280F381E02D19958091B512843658F4C0
:10714000853608F084E664E6681B8091A807909174
:10715000A9070E94D78E8091AD128C508230A8F47E
:107160006091B6127091B71285E00E94E34E609173
:10717000B8127091B91285E00E94C84E8091BA127F
:10718000E091A807F091A907808F2091AE12822F7D
:10719000022E000C990BAA0BBB0BFC013897E830B0
:1071A000F10508F089C08827EA5AFE4F8F4F0C94EA
:1071B00091CF84E290E00E94A8CFFC0180916C13F3
:1071C00029E030E03383228321E03FEF35832483BD
:1071D0002FEF30E03783268311861086108E94E8D7
:1071E000918F2BE938E0338F228F27E634E031830B
:1071F000208320E533E131A320A312A283A357C04B
:1072000080E290E00E94A8CFFC0189E090E09383A7
:10721000828381E09FEF958384838FEF90E0978353
:10722000868311861086108E87E8818F8BE998E01F
:10723000938F828F8BE594E038C080E290E00E94CB
:10724000A8CFFC0189E090E09383828381E09FEFE7
:10725000958384838FEF90E09783868311861086D1
:10726000108E8DE0818F8BE998E0938F828F8FE471
:1072700094E01BC08091F712823009F0F0C2809137
:10728000AC128C3009F0EBC21FC089E190E00E9483
:10729000A8CFFC01138212821582148217821682F3
:1072A00011861086108E8FE194E091838083F09395
:1072B000AD07E093AC075EC08091F712823061F5B4
:1072C0008091AC128C3041F58BE08093AE126BE074
:1072D00070E081E291E00E940F7189E190E00E94EC
:1072E000A8CFFC0189E090E09383828381E09FEF47
:1072F000958384838FEF90E0978386831186108631
:10730000108E83E494E091838083F093AD07E09343
:10731000AC0710923E142EC08CE08093AE126CE04D
:1073200070E081E291E00E940F7189E190E00E949B
:10733000A8CFEC0183E696E09983888384E090E00F
:107340009B838A8381E09FEF9D838C838FEF90E006
:107350009F838E8319861886188ECE010E949C50BA
:1073600087E394E099838883D093AD07C093AC07FB
:1073700010922F148091AC079091AD07DC01ED9134
:10738000FC910280F381E02D19958091B41284362E
:1073900058F4853608F084E664E6681B8091AC07F3
:1073A0009091AD070E94D78E8091AE128C508230A2
:1073B00000F56091AF127091B01284E00E94E34E2C
:1073C0006091B1127091B21284E00E94C84E809117
:1073D000B312E091AC07F091AD07808F8091AE12AF
:1073E0008D3039F48091B312E0918213F0918313C0
:1073F000808F8EE190E00E94A8CFEC01D090C41263
:10740000A090C812B090C9128090C6129090C71276
:1074100083E696E09983888383E090E09B838A8368
:1074200081E09FEF9D838C83EE24EA94F12CFF8210
:10743000EE8219861886188ECE010E949C508BE22F
:1074400094E0998388839A8E898EBC8EAB8EDD8E74
:10745000D0938314C09382146091CA127091CB129E
:1074600083E00E94E34E6091CC127091CD1283E0D4
:107470000E94C84E8091C412E0918214F09183144E
:10748000808F8091C4120E94DA7080918214909152
:107490008314DC01ED91FC910280F381E02D1995BC
:1074A0008091CF12882371F18EE390E00E94A8CFE3
:1074B000FC018091D9129091D8122091DE12309166
:1074C000DF124091DC125091DD126091DA1270915E
:1074D000DB12A091D412B091D512C091D212D091EA
:1074E000D312C090D012D090D11211821082F382A8
:1074F000E28215821482D4A2C3A2D6A3C5A3B0A7E8
:10750000A7A329C08EE390E00E94A8CFFC01809140
:10751000D9129091D8122091DE123091DF12409151
:10752000DC125091DD126091DA127091DB12A091A1
:10753000D212B091D312C091D012D091D112118237
:107540001082F382E28215821482D4A3C3A3B6A36D
:10755000A5A3F0A6E7A272A761A754A743A736A7E1
:1075600025A72BE938E030AB27A720E533E132AB84
:1075700021AB93AB84ABF0932A07E0932907C0912A
:107580002907D0912A076BA9613021F58BA19CA115
:10759000181619063CF4880F991F880F991F039637
:1075A0009CA38BA38DA19EA1181619063CF4880FED
:1075B000991F880F991F03969EA38DA38FA198A54D
:1075C000181619063CF4880F991F880F991F039607
:1075D00098A78FA32FA138A54BA15CA18DA19EA137
:1075E000421753071CF4821793077CF028173907BA
:1075F0001CF44817590764F0241735075CF4841706
:10760000950744F4142F052F05C0122F032F02C035
:10761000182F092F1F821E82188709871B861A863A
:107620001D861C861E870F87198A188A2DA53EA5E0
:1076300049A55AA58BA59CA5421753071CF4821790
:1076400093077CF0281739071CF44817590764F092
:10765000241735075CF48417950744F4142F052F7D
:1076600005C0122F032F02C0182F092F1B8A1A8A58
:107670001C8B0D8B1F8A1E8A198E188E1A8F0B8FEA
:107680001D8E1C8E1DAE1CAE8FE090E09AAF89AFB0
:107690001BAE18A21AA219A2613069F06230E9F09B
:1076A000611183C061E08CE20E94BF5910922D01EC
:1076B00010922C017AC061E08CE20E94BF591092B6
:1076C0002D0110922C0161E088E00E94BF5960E01A
:1076D00070E088E00E94FB5968C0E9A9FAA980819E
:1076E0009181A281B38181159649A105B10509F463
:1076F00057C040E056E960E070E08FA598A90E946D
:10770000E27764E170E080E090E00E94C386E9A93E
:10771000FAA980819181A281B38181152BE492071E
:10772000A105B105E9F068F4803629E09207A105CA
:10773000B105A1F080389542A105B105C1F442E040
:1077400012C0811521EE9207A105B10559F08115EE
:10775000924CA140B10559F445E005C041E003C099
:1077600043E001C046E06FE0CE010E946E4B8FA562
:1077700098A9DC01ED91FC910680F781E02D199527
:10778000E9A9FAA940815181628173818FA598A9E5
:107790000E94E27764E170E080E090E00E94C3869E
:1077A0004AE06EE0CE010E946E4B8091D912809328
:1077B000F40780913B148823F9F089E190E00E945E
:1077C000A8CFFC0188E090E0938382831582148225
:1077D0008FEF93E0978386838FEF91E09187808787
:1077E000108E83E494E091838083F0933A14E093C5
:1077F0003914CF010E94CF7F80913E14882309F471
:1078000077C089E190E00E94A8CFFC0189E090E078
:1078100093838283158214828FEF93E0978386830C
:107820008FEF91E091878087108E83E494E09183BD
:107830008083F0933D14E0933C14CF01DF91CF910E
:107840001F910F91FF90EF90DF90CF90BF90AF907E
:107850009F908F907F906F905F900C94CF7F2C3093
:1078600009F463CD8CE190E00E94A8CFEC0163E6BF
:10787000662E66E0762E7982688274E0872E912CDF
:107880009B828A82AA24A394BB24BA94BD82AC8230
:10789000CC24CA94D12CDF82CE8219861886188E09
:1078A0000E949C50A7E5EA2EA6E0FA2EF982E88213
:1078B000D093AD07C093AC078CE190E00E94A8CFB5
:1078C000EC01798268829B828A82BD82AC82DF82EF
:1078D000CE8219861886188E0E949C50F982E88202
:1078E000D0938313C0938213CE010E94A57F40CD15
:1078F000DF91CF911F910F91FF90EF90DF90CF908C
:10790000BF90AF909F908F907F906F905F90089501
:107910002F923F924F925F926F927F928F929F929F
:10792000AF92BF92CF92DF92EF92FF920F931F938D
:10793000CF93DF93CDB7DEB7CE5AD1090FB6F89407
:10794000DEBF0FBECDBFCDB6DEB6C455DF4F188249
:10795000CC5AD040C555DF4F1882CB5AD0408091C9
:10796000B20E8B3709F4E9C180F4873709F4D8C225
:1079700038F48F3109F446C5863709F4E1C108C6E9
:107980008937B9F008F4DBC234C0803809F473C415
:1079900038F48C3709F4E2C28E3709F42EC3F8C5E7
:1079A000823809F409C508F41EC5833809F4E7C410
:1079B000EFC50E94B0520E94FD862B013C010E943F
:1079C00033AA029709F429C50E94FD86DC01CB0188
:1079D00084199509A609B70980329340A105B1051C
:1079E00008F01BC50E94645E0E94B0520E946EA8FF
:1079F000E6CF0E9433AA029729F060E084E80E9453
:107A000023A98CC18091F60B823031F0833039F498
:107A100082E08093290F03C081E08093040F81E00E
:107A20008093BC0E8E0104551F4F2FE0AE014057CE
:107A30005F4F68E871E90E94ACA80E9406AA8930ED
:107A400058F0015011092FE0AE014F575F4F68E821
:107A500072E981E00E94ACA81092BB0E7724739467
:107A60000E941CAA882309F43DC1198222961FAEE8
:107A700022971091BB0E11110EC0BE0160577F4FAF
:107A8000CE018F5B9F4F0E94CCD1C455DF4F088140
:107A9000CC5AD04011C0113071F4BE016F577F4FE6
:107AA000CE018F5B9F4F0E94CCD1C555DF4F08811F
:107AB000CB5AD04001C000E0ADB6BEB68091F20B0B
:107AC000EDB7FEB722E0829FE019F10911240FB64D
:107AD000F894FEBF0FBEEDBF8DB79EB701967C0137
:107AE0006DE876E0CE018B559F4F0E94D655809170
:107AF000F60B823089F0833061F1813009F0A1C04A
:107B00004091F20B50E0B7018091C3149091C414DE
:107B10000E9463A710E039C02091F20B30E05FB7FC
:107B2000F89440E0842F90E08217930774F4880F54
:107B3000991FF701E80FF91FDC01AD51B14F8D918D
:107B40009C91918380834F5FEDCF5FBF1092030FB5
:107B50001CC02091F20B30E05FB7F89440E0842F16
:107B600090E08217930774F4880F991FF701E80FCC
:107B7000F91FDC01AE5BB04F8D919C9191838083A6
:107B80004F5FEDCF5FBF1092C0146DE270E0CE0189
:107B90008B559F4F0E94D4542091F20B293048F00E
:107BA000112321F0113021F418E004C028E001C0B5
:107BB00020E010E0121758F5F701E10FF11DE10F79
:107BC000F11D608171814AE0CE0181569F4FC355FE
:107BD000DF4F2883CD5AD0400E947D55BE016156AB
:107BE0007F4FCE018B559F4F0E94FB54CE01815693
:107BF0009F4F0E947855CE018B559F4F0E94447431
:107C00001F5FC355DF4F2881CD5AD040D3CF40E40A
:107C100050E0BE016F5F7F4FCE018B559F4F0E949A
:107C20003B74C755DF4F1881C95AD040CE018B55E0
:107C30009F4F0E9478550FB6F894BEBE0FBEADBEE2
:107C40000BC0CE018B559F4F0E9478550FB6F8940C
:107C5000BEBE0FBEADBE10E0BE016F5F7F4FCE0156
:107C60008F5B9F4F0E94CCD1010F10E0E1E4F0E068
:107C7000EC0FFD1FE00FF11F1082BE016F5B7F4F05
:107C80008091A4149091A5140E945757B801CE0179
:107C90008F5B9F4F0E948CA8BC018091A41490918F
:107CA000A5140E9400726AE08091A4149091A5141A
:107CB0000E946E568091A4149091A514DC01ED9160
:107CC000FC910680F781E02D19950E9406AA893063
:107CD00048F08091BB0E811103C07092BB0E02C0B0
:107CE0001092BB0E0E94B0520E946EA80E94138197
:107CF00081110E94883C8091B10E81110FC080914A
:107D0000BC0E882359F08091A614811107C0809180
:107D1000AF0E9091B00E0A970CF4A2CE8091F60BA4
:107D2000823039F0833009F033C481E08093290F29
:107D30002FC481E08093040F2BC41092BC0E5FC34C
:107D40001091B50E8FEF810F853028F060E089E843
:107D50000E9423A91DC4133079F018F41230F9F0F1
:107D600004C0143079F0153099F040E6442E49E013
:107D7000542E612C712C19C0412C3BE4532E612CE4
:107D8000712C13C0412C26E9522E612C712C0DC090
:107D9000412C92EC592E66246394712C06C080E825
:107DA000482E85E2582E612C712C00E0E12EF12C3A
:107DB0005701BFE8AB0EB11C1501E89427F8332436
:107DC000E6E9EE0EF11CE894E7F8FF24023091F0AA
:107DD00018F4013051F004C0033089F00430A1F0F0
:107DE00040E659E060E070E013C040E855E260E032
:107DF00070E00EC040E05BE460E070E009C040E08D
:107E000056E960E070E004C040E052EC61E070E0F0
:107E10008BE998E00E94E2778BE998E00E94DF53BB
:107E20000E94FD864B015C01F2E38F0E911CA11CA8
:107E3000B11C0E942EA80E94FD86681579058A054E
:107E40009B05B8F360E870E08BE998E00E94058339
:107E50006FE070E08BE998E00E940583612F8BE969
:107E600098E00E949853B1018BE998E00E94058345
:107E70000E94FD864B015C012AE0820E911CA11C30
:107E8000B11C0E942EA80E94FD86681579058A05FE
:107E90009B05B8F367E870E08BE998E00E940583E2
:107EA0006FE070E08BE998E00E940583612F8BE919
:107EB00098E00E949853B7018BE998E00E940583EF
:107EC0008BE998E00E94DF530E94FD864B015C0124
:107ED0003EE5830E31E0931EA11CB11C0E942EA82A
:107EE0000E94FD86681579058A059B05B8F30F5F2A
:107EF000053009F06BCFB301A2018BE998E00E9435
:107F0000E277409250135092511360925213709244
:107F10005313B301A20183EC91E00E9477746FC206
:107F200083E090E00E94A8CF2AE0DC012C932BE9AB
:107F300038E012963C932E9311976AE00CC083E0D0
:107F400090E00E94A8CF2DE0FC0120832BE938E0CF
:107F5000328321836DE00E948F6051C24091B50E43
:107F60005091B60E0091B70E1091B80E6091B30EFD
:107F70007091B40ECE010196C355DF4F4883CD5AA0
:107F8000D040C255DF4F5883CE5AD0400E941D4783
:107F9000C355DF4F4881CD5AD040C255DF4F58817D
:107FA000CE5AD040892BE9F08D81873050F485304E
:107FB00080F48130B0F0642F8B819C810E946B72C1
:107FC0000DC0893070F4B8018B819C810E94777458
:107FD00005C0BA018B819C810E940F710E94A0A9EB
:107FE00004C061E085E80E9423A98091AE0E811152
:107FF000CFC281E08093AE0ECBC2B090B30EE090C2
:10800000B40EC156DF4F1882CF59D0406DE876E0EC
:10801000CE018F579F4F0E94D6556B2D7E2DCE01DE
:1080200080579F4F0E941D47892B09F4BEC0CC5634
:10803000DF4FE881C459D0404E2F50E0FA0131970C
:10804000E830F10508F0B1C08827E25AFE4F8F4FA3
:108050000C9491CFCE56DF4F88819981C259D04080
:108060000E9425CD4AE0682FCE0101960E94A955B5
:108070001BC0CE56DF4F88819981C259D0400E94E3
:1080800025CD682F880F770B4AE00AC0CE56DF4F08
:1080900088819981C259D0400E9433CD4AE0BC0109
:1080A000CE0101960E947D55BE016F5F7F4FCE01CC
:1080B0008F579F4F0E949B54CE01019663C0CE56AE
:1080C000DF4F88819981C259D0400E9433CD2396D9
:1080D0001FAE1EAE239725961FAE1EAE2597279680
:1080E0001FAE1EAE27974AE0BE016F5F7F4F0E9412
:1080F000C7CB35C0CE56DF4F88819981C259D04059
:108100000E942DCD23961FAE1EAE239725961FAE3F
:108110001EAE259727961FAE1EAE27972AE0AE010A
:108120004F5F5F4F0E948BCB1AC0CE56DF4F8881C6
:108130009981C259D0400E942DCD23961FAE1EAE0C
:10814000239725961FAE1EAE259727961FAE1EAE0F
:1081500027972AE0AE014F5F5F4F0E949ACBBE0186
:108160006F5F7F4FCE018F5B9F4F0E945755BE01BF
:108170006F5B7F4FCE018F579F4F0E949B54CE0164
:108180008F5B9F4F0E9478554FE050E0BE016F5BC0
:108190007F4FCE018F579F4F0E943B74CB57DF4FCD
:1081A000F880C558D04011E002C0F12C10E0CE019B
:1081B0008F579F4F0E947855112309F4C7CD8E0128
:1081C00001561F4F20E4AE014F5F5F4F68E87B2DE3
:1081D0008E2D0E94ACA8BE016F5B7F4FCE01019631
:1081E0000E94CCD1C156DF4F8881CF59D040F80EC4
:1081F00081E08F0DC156DF4F8883CF59D040E1E039
:10820000F0E0EC0FFD1FEF0DF11D9CE79083E1E026
:10821000F0E0EC0FFD1FE80FF11D1082BE016F5F53
:108220007F4F8091A4149091A5140E945757C15676
:10823000DF4F6881CF59D04070E0CE0101960E9497
:108240008CA8BC018091A4149091A5140E94007286
:108250006AE08091A4149091A5140E946E568091BA
:10826000A4149091A514DC01ED91FC910680F78196
:10827000E02D19958DC18091B30E9091B40E803888
:10828000910509F085C18E0100571F4F20E4AE0112
:108290004F5F5F4F68E870E880E00E94ACA86BE633
:1082A00076E0CE018F579F4F0E94D655CE018F5753
:1082B0009F4F0E944474C057DF4F2881C059D0405F
:1082C000CB57DF4F88819981C558D040820F911DCF
:1082D000C057DF4F8883C059D04022961FAE2297E7
:1082E0004FE050E0BE016F5B7F4FCE018F579F4F35
:1082F0000E941874BE016F5B7F4FCE0101960E94F1
:10830000CCD1C057DF4F8881C059D040E1E0F0E0C8
:10831000EC0FFD1FE80FF11D1082BE016F5F7F4F54
:108320008091A4149091A5140E945757C057DF4F15
:108330006881C059D04070E0CE0101960E948CA89F
:10834000BC018091A4149091A5140E9400726AE06F
:108350008091A4149091A5140E946E568091A4144B
:108360009091A514DC01ED91FC910680F781E02D40
:108370001995CE018F579F4F0E94785509C1809162
:10838000B30E9091B40E8338910509F001C18E01AE
:1083900000571F4F20E4AE014F5F5F4F68E873E85E
:1083A00080E00E94ACA84AE06091AD0ECE018F57EC
:1083B0009F4F0E94A9557ACF8091B30E9091B40E31
:1083C0008238910509F0E4C08E0100571F4F20E468
:1083D000AE014F5F5F4F68E872E880E00E94ACA892
:1083E00063E876E05ECF8091B30E9091B40E813851
:1083F000910509F0CDC08091BC0E8111C9C00E94C9
:10840000A0A9C6C08091B30E9091B40E4F9709F009
:10841000BFC081E08093B10EBBC00E9433AA029717
:1084200019F060E084E894CC8091F50B811102C0D2
:108430000E9485720E9406AAF82E6DE876E0CE01B1
:1084400080579F4F0E94D655C156DF4F1882CF5993
:10845000D0408E0101561F4F20E4AE014F5F5F4FA9
:1084600068E879E780E00E94ACA8CF57DF4F198217
:108470001882C158D040CD57DF4F19821882C35897
:10848000D040CB57DF4F19821882C558D0406F2D8E
:1084900070E080E090E02AE0AE014F5B5F4F0E9409
:1084A0008BCBBE016F5B7F4FCE018F579F4F0E94DA
:1084B0005755BE016F577F4FCE0180579F4F0E9487
:1084C0009B54CE018F579F4F0E9478554FE050E04C
:1084D000BE016F5B7F4FCE0180579F4F0E94187483
:1084E000CC56DF4F1881C459D040BE016F5B7F4F1F
:1084F000CE0101960E94CCD1C156DF4F8881CF5961
:10850000D040810F91E0980FC156DF4F9883CF592B
:10851000D040E1E0F0E0EC0FFD1FE80FF11D8CE72B
:108520008083E1E0F0E0EC0FFD1FE90FF11D108208
:10853000BE016F5F7F4F8091A4149091A5140E949B
:108540005757C156DF4F6881CF59D04070E0CE01F8
:1085500001960E948CA8BC018091A4149091A5144E
:108560000E9400726AE08091A4149091A5140E9468
:108570006E568091A4149091A514DC01ED91FC91AC
:108580000680F781E02D1995CE0180579F4FF4CEDC
:108590000FB6F894DEBE0FBECDBEC255DF4F0FB68C
:1085A000F894DEBF0FBECDBFDF91CF911F910F9129
:1085B000FF90EF90DF90CF90BF90AF909F908F9003
:1085C0007F906F905F904F903F902F900895FC01A7
:1085D00012821382148215821682178212860895DF
:1085E00080E008950F931F93CF938C016DE87DE198
:1085F00085ED99E00E945957D8011896ED91FC91AC
:1086000019976081718185ED99E00E94826DC1E0CA
:10861000D8011A968C91C81710F568E87DE185EDB0
:1086200099E00E9459576C2F85ED99E00E943F70A8
:1086300065E87DE185ED99E00E945957F801908544
:108640008185E92FF82FEC0FF11DEC0FF11D6081F2
:10865000718185ED99E00E94826DCF5FD9CFCF9176
:108660001F910F910895CF93DF93CDB7DEB7A097F9
:108670000FB6F894DEBF0FBECDBF80310CF080E0A6
:108680002DE73DE13A83298326E73DE13C832B83B7
:1086900028E63DE13E832D832CE53DE138872F839D
:1086A00022E53DE13A87298728E43DE13C872B8795
:1086B00024E43DE13E872D872DE33DE1388B2F8774
:1086C00022E33DE13A8B298B25E23DE13C8B2B8B6C
:1086D0002AE13DE13E8B2D8B2EE03DE1388F2F8B43
:1086E0002CEF3CE13A8F298F2BEE3CE13C8F2B8F16
:1086F00026EE3CE13E8F2D8F29ED3CE138A32F8FF4
:10870000E82FEE0FFF0BEC0FFD1F81819281A096E9
:108710000FB6F894DEBF0FBECDBFDF91CF910895A5
:10872000AF92BF92CF92DF92EF92FF920F931F937F
:10873000CF93DF938FEB9EE07EE1D72ED80ECC2433
:10874000C39402E010E0C3E0D0E0E2E0BE2EEE24ED
:10875000E394F12C8091400F9091410FDC01ED9159
:10876000FC910084F185E02D1995892B09F4ADC0A9
:10877000A09030018091400F9091410FDC01ED916C
:10878000FC910284F385E02D199596B3B39A20915C
:10879000840030918500285A344E30938D00209308
:1087A0008C002A2D2C7119F010922A0F4BC093FBCC
:1087B000992790F9E0912A0FE11116C0992351F2FF
:1087C000803241F6C0922A0F8093BF0E8091BE1472
:1087D0009091BF14892B09F0BDCFF092BF14E092A5
:1087E000BE1410922C0FB6CF9111DECFE13041F4C0
:1087F000803409F0AFCFB0922A0F8093C00EE6CF3D
:1088000091E09E0F90932A0FF0E0E154F14F8083A6
:10881000903209F09FCF10922A0FEFEBFEE02FEF7E
:108820003FEF8191281B3109DE12FBCF4091DD0E15
:108830008091DE0E90E0982F8827840F911D2817D5
:10884000390729F0D093BF14C093BE1483CF809111
:10885000BE149091BF14019739F480912C0F8F5F53
:1088600080932C0F843020F01093BF140093BE141B
:1088700080912B0F8F5F80932B0F9091290F98176A
:1088800008F5C092C01420E030E0F901E154F14F46
:108890004281838190E0982F8827840F911DAC013D
:1088A0004F5E52404B3D554028F4F901EE5BF04FCE
:1088B000918380832E5F3F4F2C31310531F7109229
:1088C0002B0F48CF1092C01445CFDF91CF911F914D
:1088D0000F91FF90EF90DF90CF90BF90AF900895F1
:1088E000EF92FF920F931F93CF93DF9310928D110E
:1088F00082E080938E1168EE73E070939011609324
:108900008F1140ED57E050939211409391112CED4F
:1089100035E030939411209393118FE0809395115B
:108920001092961194E0909397117093991160931F
:10893000981150939B1140939A1130939D1120935D
:108940009C1180939E1110929F1193E09093A0111F
:108950007093A2116093A1115093A4114093A3119D
:108960003093A6112093A5118093A7111092A811FE
:1089700091E09093A9117093AB116093AA11509359
:10898000AD114093AC113093AF112093AE11809391
:10899000B0111092B111E2EBF1E1ABEBB1E180E08B
:1089A00008EE13E060ED77E04CED55E031E022E0B9
:1089B00095E0980F908312830183748363835683B9
:1089C0004583ED01229791E03883219628831C92FC
:1089D0008F5F3A961A968C3059F710922A1290931C
:1089E0002B1210922C1290932D128AE892E0909301
:1089F0002F1280932E1290933112809330128CE2BA
:108A000091E0909333128093321280E090E09C01C9
:108A100023573E4EF901E955FF4F118210823296DD
:108A2000108203968837910591F784E290E0909345
:108A300035128093341281E0809336122CE030E0BE
:108A4000309338122093371294E09093391221E238
:108A500030E030933B1220933A1227E020933C12EF
:108A600029E030E030933E1220933D1220E1209324
:108A70003F127AE07093AC122BE02093AD1220935A
:108A8000AE1248EE53E05093B0124093AF1220ED77
:108A900037E03093B2122093B1121092B31264E611
:108AA0006093B4126093B5125093B7124093B6120C
:108AB0003093B9122093B8121092BA125093BC128C
:108AC0004093BB123093BE122093BD121092BF127E
:108AD0001092C0128093C1121092C3121092C2124F
:108AE0008093C4128093C512E8ECF0E0F093C712B3
:108AF000E093C612E0E2F3E0F093C912E093C812EB
:108B00005093CB124093CA123093CD122093CC12C3
:108B10001092CE128093CF12E9E5F0E0F093D112DB
:108B2000E093D012E0E8F0E0F093D312E093D21299
:108B3000EFEFF0E0F093D512E093D412F093D71258
:108B4000E093D6121092D8121092D912F093DB1241
:108B5000E093DA12F093DD12E093DC12F093DF126F
:108B6000E093DE121092E0128093E1129093E212F1
:108B70001092E3128093E4129093E5121092E612A1
:108B80001092E7128093E8121092E9121092EA1202
:108B90008093EB121092EC1298E29093ED125093A6
:108BA000EF124093EE125093F1124093F012309373
:108BB000F3122093F2128093F41292E39093F51241
:108BC000E2E0E093F6128093F7126093F812E6E485
:108BD000E093F9129093FA121092FB121092FC1289
:108BE0001092FD121092FE121092FF1210920013BA
:108BF000EAEFF0E0F0930213E093011310920313F5
:108C000010920413609305136093061310920713D8
:108C1000109208139093091310920A1390930B1358
:108C2000EEE5F1E0F0930D13E0930C1310920E13A8
:108C3000ACEDB5E0B0931013A0930F1300EA1FE062
:108C400010931213009311133093141320931313E2
:108C5000C8E8D3E1D0931613C093151368EBE62E42
:108C60006BE0F62EF0921813E0921713E0E4FFE1A8
:108C7000F0931A13E093191310921B1310921C1304
:108C800010921D1369E160931E1380931F1380934C
:108C90002013809321135093231340932213309376
:108CA000251320932413F0922713E0922613109398
:108CB000291300932813D0932B13C0932A1320E772
:108CC00037E130932D1320932C1310922E13109212
:108CD0002F1310923013909331139093321390937B
:108CE000331310923413109235131092361380936D
:108CF00037131092381399E09093391310923A1366
:108D000010923B1310923C1310923D13B0933F13FB
:108D1000A0933E13F0934113E093401380934213CA
:108D2000709343131092441321E030E030934613C4
:108D3000209345131092471340E052EC61E070E03D
:108D4000409348135093491360934A1370934B1305
:108D500040934C1350934D1360934E1370934F13E5
:108D600040E056E960E070E0409350135093511397
:108D700060935213709353134093541350935513AD
:108D800060935613709357131092581320E039E1F3
:108D900030935A132093591310925B139EE19093D2
:108DA0005C1310925D132EE130E030935F1320933B
:108DB0005E133093611320936013309363132093F9
:108DC000621390936413909365138093661380935A
:108DD0006713109268139093691380936A1310922B
:108DE0006B139CE090936C1380936D1388EC9BE95C
:108DF000A0E0B0E080936E1390936F13A093701374
:108E0000B09371130DE811E1C0E0D0E0CE010E94F3
:108E100025CDF80161918F01861719F0CE010E94CE
:108E200039CD2196C53EF1E0DF0781F7DF91CF9183
:108E30001F910F91FF90EF9008954F925F926F9264
:108E40007F928F929F92AF92BF92CF92DF92EF92DA
:108E5000FF92CF93DF93EB01A091BD0EB091BE0EB8
:108E60009D012F5F3F4F45E0429F2001439F500CE3
:108E70001124052C000C66087708812C912C5401D4
:108E80002E34E1E03E07ECF446E15FEB61E077274A
:108E900075016401C40CD51CE61CF71C4C0D5D1D4E
:108EA0006E1D7F1D6BBFFA014791569165E0860EDE
:108EB000911CA11CB11CC417D50729F12F5F3F4F8E
:108EC000DFCF25E0822E912CA12CB12C21E030E0C7
:108ED000A217B30708F44CC046E15FEB61E07727C7
:108EE000480D591D6A1D7B1D6BBFFA0147915691B4
:108EF000F5E08F0E911CA11CB11CC417D50719F009
:108F00002F5F3F4FE5CF46E15FEB61E07727E5E07C
:108F1000E29F6001E39FD00C11240D2C000CEE08A1
:108F2000FF084E5F5F4F6F4F7F4F4C0D5D1D6E1DF5
:108F30007F1D6BBFFA0147915691FC015383428319
:108F400046E15FEB61E077274C5F5F4F6F4F7F4FEC
:108F5000C40ED51EE61EF71EEBBEF601C790FC013F
:108F6000C4823093BE0E2093BD0EC901019606C087
:108F70001092BE0E1092BD0E80E090E0DF91CF9176
:108F8000FF90EF90DF90CF90BF90AF909F908F9029
:108F90007F906F905F904F9008951F920F920FB641
:108FA0000F9211242F938F939F93109295001092FC
:108FB00094008091EA0B8F5F8093EA0B909191145B
:108FC000891784F01092EA0B2091EC0B80918F149A
:108FD00090919014820F911D27FD9A959093901473
:108FE00080938F148091E90B8F5F8093E90B9091B0
:108FF0009C14891784F01092E90B2091EB0B80915F
:109000009A1490919B14820F911D27FD9A9590932D
:109010009B1480939A149F918F912F910F900FBE64
:109020000F901F9018958091E80B811104C08091DA
:10903000E70B882321F080917100826003C080914A
:1090400071008D7F809371000895CF93DF93EC01C1
:10905000198618861F861E86198A188A1B8A1A8AFC
:109060000E94BF6C1EA61D86DF91CF910895CF93FD
:10907000DF93EC011F861E86198A188A1B8A1A8ABA
:109080000E94BF6C198618861C86DF91CF910895C7
:10909000FC018385882311F061E001C060E08285D6
:1090A0000C948F59FC018385882311F060E001C086
:1090B00061E082850C948F590F931F93CF93DF93B8
:1090C000CDB7DEB78C010E943748F801148A85E1DC
:1090D000FE013896D801559601900D928A95E1F7D8
:1090E000F80185899689938B828B8D8D8B3008F062
:1090F0008AE090E0F801918B808BC8010E94524871
:10910000C8010E94BF6C81E0F8018487DF91CF9194
:109110001F910F910895CF92DF92EF92FF920F93DC
:109120001F93CF93DF93CDB7DEB765970FB6F89453
:10913000DEBF0FBECDBF8C01FC0185858823E1F029
:1091400082899389892B09F44EC10E94FD86F8011A
:10915000C080D180E280F380AB01BC014C195D0975
:109160006E097F0982899389A0E0B0E08417950792
:10917000A607B70728F137C1F80180859185892BAB
:1091800009F494C00E94FD86F801C480D580E68071
:10919000F780AB01BC014C195D096E097F09808520
:1091A0009185A0E0B0E084179507A607B70708F0FF
:1091B0007DC0C8010E944848C8010E943748B9C014
:1091C000F8018685978501969787868760897189DA
:1091D0008617970768F580E090E00E94F6CB9B0128
:1091E000AC016BED7FE089E490E40E9417CEF801BA
:1091F00022A533A544A555A50E94ABCDF80162A7D1
:1092000073A784A795A70E94C4CE20E030E04FEF5B
:1092100052E40E9457CC20E030E04FEF52E40E942D
:10922000ABCD0E9489CEF80182850E94FB5970C0A7
:10923000F8018585823021F4C8010E94484879C030
:10924000F80186A5882309F474C0C8010E94254846
:1092500082E390E09A83898388E290E09C838B8309
:109260008EE690E09E838D8384EF91E098878F83D4
:109270001D8A84E08F938DB79EB745970FB6F894FB
:109280009EBF0FBE8DBFADB7BEB7119685E1FE0183
:10929000319601900D928A95E1F7C8010E945C48D1
:1092A0000FB6F894DEBF0FBECDBF9DC0F801828916
:1092B0009389892B09F497C00E94FD86F801C0802C
:1092C000D180E280F380AB01BC014C195D096E09CD
:1092D0007F0982899389A0E0B0E084179507A607EB
:1092E000B70708F080C0F8018685978501969787B3
:1092F0008687208931898217930708F053C080FF41
:1093000029C0C8010E944848F8018489882331F1A6
:10931000C80165960FB6F894DEBF0FBECDBFDF91D2
:10932000CF911F910F91FF90EF90DF90CF900C9411
:10933000BF6CC80165960FB6F894DEBF0FBECDBFF7
:10934000DF91CF911F910F91FF90EF90DF90CF9021
:109350000C942548C8010E945248D6CF868597852F
:109360008B309105A0F0C8010E944848C80165965D
:109370000FB6F894DEBF0FBECDBFDF91CF911F9126
:109380000F91FF90EF90DF90CF900C943748880FAB
:10939000991FF801E80FF91F85899689F801938BC9
:1093A000828BB6CFF80181A5882351F085899689F3
:1093B000938B828B17861686C8010E945248A8CFCD
:1093C000F80186A5882379F216A682E08587C80170
:1093D0000E94374884E690E0F801918B808B87A546
:1093E00090A9938B828B65960FB6F894DEBF0FBE63
:1093F000CDBFDF91CF911F910F91FF90EF90DF9044
:10940000CF900895CF93DF93EC018C85882331F0C2
:10941000CE010E944848CE010E9437488D8588239E
:1094200019F0CE010E942548CE01DF91CF910C9416
:1094300048488F929F92AF92BF92CF92DF92EF9265
:10944000FF920F931F93DC0114968D919C911597B9
:109450005696CD90DC9057976817790709F455C058
:109460009096FC9090974C01092E000CAA08BB081E
:109470008B01072E000C220B330B861797073CF449
:109480001296ED91FC911397FF2031F014C0ED91ED
:10949000FC911197FF2079F00D2C000CEE08FF08CD
:1094A000A9019801281939094A095B0954966D9157
:1094B0007C9155970EC00D2C000CEE08FF08A901F9
:1094C0009801281939094A095B0952966D917C91D6
:1094D0005397CB01770FAA0BBB0BBC01CD016C19C5
:1094E0007D098E099F090E9459CF8F01FF0F220B22
:1094F000330BA9019801281939094A095B090E940F
:1095000047CDC20ED31EE41EF51EC6011F910F915A
:10951000FF90EF90DF90CF90BF90AF909F908F9093
:109520000895482F50E095E1899FF0011124E753F9
:10953000FF4E2181328180859185280F391F8381DB
:1095400094818217930728F085819681281739071F
:10955000E8F485E1849FF001859FF00D1124E75325
:10956000FF4E858196812817390728F52581368198
:1095700085E1849FF001859FF00D1124E753FF4E94
:109580008285823019F411861086128685E1849FC7
:10959000F001859FF00D1124E753FF4E32832183A4
:1095A0008091840090918500280F391F30938900A5
:1095B0002093880008958381948182179307C0F6D1
:1095C00023813481D5CF4F925F926F927F928F9299
:1095D0009F92AF92BF92CF92DF92EF92FF920F9342
:1095E0001F93CF93DF936C01A4ECCA1AADEFDA0A94
:1095F000D601ED91FC917E970CF05DC0FC01E8581E
:10960000FF4F812C912CA191B191AB2B21F421150D
:10961000310549F450C0BFEF8B1A9B0AAEE18A16A0
:10962000910489F748C0EC015401AA0CBB1CAA0C98
:10963000BB1CAC0EBD1EF501EC54FF4F40835183A3
:10964000628373837401EE0CFF1CEC0EFD1EF701A8
:10965000E858FF4F31832083EC54FF4F1183008380
:10966000BE01680D791DFB01EC55FE4F81E0808342
:109670000E94FD86F5016083718382839383C65CBB
:10968000DD4F88819981F701E250FE4F91838083FD
:10969000D6012D913C9111972F5F3F4F2D933C9315
:1096A0009C012F5F3F4F1216130614F021E030E0AB
:1096B0003983288302C08FEF9FEFDF91CF911F91F5
:1096C0000F91FF90EF90DF90CF90BF90AF909F9061
:1096D0008F907F906F905F904F9008950F931F939E
:1096E000CF93DF938C01C62FD42F65E870E0DC01A7
:1096F0009F968D919C91D0970E940583F80187A534
:1097000090A9DC01ED91FC910190F081E02D6C2F8E
:109710001995F80187A590A9DC01ED91FC910190C4
:10972000F081E02D6D2F19952C2F30E0B9016B578A
:109730007F4F6D0F711D6F777727F80187A590A96F
:10974000DF91CF911F910F910C940583262F2B7FD2
:10975000A9F49A014F3F510519F014F02FEF30E0B2
:10976000A90141302FEF520714F441E05FEF57FF9A
:1097700003C05195419551090C946E4B0895CF93B8
:10978000DF93EC018CAD9DAD892B11F01DAE1CAEAD
:10979000CE010E94BA778BA9813029F0823069F01E
:1097A000811119C005C060E070E088E00E94FB599B
:1097B00010922D0110922C010AC040E064E0CE010D
:1097C0000E946E4B40E060E0CE010E946E4B1AA2F8
:1097D00019A21F8E1E8E0E94FD866DAB7EAB8FABD5
:1097E00098AFDF91CF910895EF92FF920F931F935F
:1097F000CF93DF93EC018B017A018BA9813069F063
:10980000823099F081111FC070932D0160932C015B
:109810007AA369A37F8F6E8F16C088E00E94FB59E0
:10982000F0922D01E0922C010AC0AB0164E0CE0160
:109830000E94A64BA70160E0CE010E94A64B1AA38E
:1098400009A3FF8EEE8E0E94FD866DAB7EAB8FABC3
:1098500098AFDF91CF911F910F91FF90EF900895F6
:109860008F929F92AF92BF92CF92DF92EF92FF9230
:109870000F931F93DC0114968D919C9115971A9666
:10988000CD90DC901B976817790709F455C0909626
:10989000FC9090974C01092E000CAA08BB088B0184
:1098A000072E000C220B330B861797073CF41296F9
:1098B000ED91FC911397FF2031F014C0ED91FC91D4
:1098C0001197FF2079F00D2C000CEE08FF08A9017C
:1098D0009801281939094A095B0918966D917C91FC
:1098E00019970EC00D2C000CEE08FF08A901980175
:1098F000281939094A095B0916966D917C911797C9
:10990000CB01770FAA0BBB0BBC01CD016C197D09F4
:109910008E099F090E9459CF8F01FF0F220B330B35
:10992000A9019801281939094A095B090E9447CD04
:10993000C20ED31EE41EF51EC6011F910F91FF90AB
:10994000EF90DF90CF90BF90AF909F908F90089551
:10995000EF92FF920F931F93CF93DF93EC018CADA7
:109960009DAD8230910509F45BC0892B11F01DAECD
:109970001CAE8BA98130A9F0823069F181114AC0F7
:1099800077FF03C0719561957109CE010E94304C3B
:1099900090932D0180932C019AA389A39F8F8E8F82
:1099A00039C0062F172F17FF03C011950195110914
:1099B000B801CE010E94304C7C01B801CE010E945A
:1099C000194A8C01B70188E00E94FB5910932D01C0
:1099D00000932C011BC0062F172F17FF03C01195F2
:1099E00001951109B801CE010E94304C7C01B801EB
:1099F000CE010E94194A8C01A70164E0CE010E94A9
:109A0000A64BA80160E0CE010E94A64BFAA2E9A2F3
:109A10001F8F0E8F0E94FD866DAB7EAB8FAB98AF14
:109A2000DF91CF911F910F91FF90EF900895CF9309
:109A3000DF93EC018CAD9DAD8230910519F1892B3E
:109A400011F01DAE1CAE2FA138A58DA19EA19F8344
:109A50008E83398728879B878A872DA53EA58BA56E
:109A60009CA59B8B8A8B3D8B2C8B9F8B8E8B60E078
:109A700070E0CE010E94A84C0E94FD866DAB7EABCB
:109A80008FAB98AFDF91CF910895CF93DF93EC0127
:109A90008CAD9DAD8230910519F1892B11F01DAE71
:109AA0001CAE2FA138A58BA19CA19F838E833987E3
:109AB00028879B878A872DA53EA589A59AA59B8B7C
:109AC0008A8B3D8B2C8B9F8B8E8B60E070E0CE0160
:109AD0000E94A84C0E94FD866DAB7EAB8FAB98AF09
:109AE000DF91CF910895DC01A250BE4F20E030E01D
:109AF0004D915D914617570739F4280F391FF90129
:109B0000EC55FE4F808108952F5F3F4F2E31310578
:109B100079F780E00895CF93DF93EC01C45CDD4FCB
:109B2000A881B981109709F442C0FC01E250FE4FB0
:109B300020E030E0419151914617570799F5A9016E
:109B4000440F551F480F591FFA01E858FF4F608115
:109B50007181672B61F111821082FC01E20FF31F0A
:109B6000EC55FE4F1082FA01EE53FE4F1182108227
:109B7000235D3F4F220F331F220F331FFC01E20FE3
:109B8000F31F1082118212821382FA01E859FE4FEC
:109B900011821082EA56FF4F118210821197B98309
:109BA000A88305C02F5F3F4F2E31310519F6DF9195
:109BB000CF9108950F931F9301E010E00E94E34AB4
:109BC0001F910F9108950F931F9300E010E00E94E2
:109BD000E34A1F910F9108952F923F924F925F9207
:109BE0006F927F928F929F92AF92BF92CF92DF92AD
:109BF000EF92FF920F931F93CF93DF9300D000D08B
:109C0000CDB7DEB78C010E94FD8698012E533E4FE2
:109C10003C832B831E830D83D801AC55BE4FBA8382
:109C2000A9831801B2E02B1ABEEF3B0AF901AA245E
:109C3000A394B12C32E0832E912C118210829F01CB
:109C40002A543140D9012D913C91232B09F44DC068
:109C5000AD81BE812D913D914D915C9113977D0118
:109C6000B4EBEB0EF11CD701CD90DD90ED90FC90A4
:109C70002B013C01421A530A640A750A4C145D0414
:109C80006E047F0490F1C20ED31EE41EF51EAD815A
:109C9000BE81CD92DD92ED92FC921397A981BA819B
:109CA0002C91222311F19F0126593109D9012D91BF
:109CB0003C912115310519F4B182A08216C07F01B3
:109CC000BAE5EB1AF108D7014D915C911197421753
:109CD00053075CF4B182A0824F5F5F4F4D935C935A
:109CE0004217530714F09182808232962D813E8173
:109CF0002C5F3F4F3E832D83A981BA811196BA8391
:109D0000A983E215F30509F098CFEB81FC818191DD
:109D10009191FC83EB8381309105A1F00297D1F4FE
:109D2000EB81FC81EC54F1400190F081E02D19951C
:109D3000AB81BC81DA966D917C91DB97C8010E9462
:109D40008B4D08C0EB81FC81EC54F1400190F08117
:109D5000E02D19952B813C8122153305B1F626960D
:109D60000FB6F894DEBF0FBECDBFDF91CF911F912C
:109D70000F91FF90EF90DF90CF90BF90AF909F90AA
:109D80008F907F906F905F904F903F902F900895AD
:109D90006E3E22E0720738F06B3C98E0790728F0BD
:109DA0006AEC78E002C06EEE72E0660F771F9FB734
:109DB000F89425E1829FF0011124E753FF4E74834C
:109DC00063839FBF08956E3E22E0720738F06B3CBC
:109DD00098E0790728F06AEC78E002C06EEE72E055
:109DE000660F771F9FB7F89425E1829FF001112439
:109DF000E753FF4E768365839FBF0895660F771FF5
:109E0000282F30E095E1899FF0011124E753FF4EA0
:109E1000858196816817790718F46581768107C076
:109E2000838194818617970710F4638174818FB7BB
:109E3000F89495E1929FF001939FF00D1124E75360
:109E4000FF4E728361838FBF0895982F8FB7F89468
:109E500025E1929FF0011124E753FF4E21E0278373
:109E60008FBF41B121E030E0B90102C0660F771F1A
:109E70009A95E2F7CB01842B81B908958A3058F482
:109E80009FB7F89425E1829FF0011124E753FF4E1C
:109E9000118610869FBF08951F93CF93DF9325E10E
:109EA000829FC0011124EC01C753DF4E8A858111C6
:109EB0000FC01FB7F89481E08A8789899A899A83AD
:109EC00089830E94FD866B877C878D879E871FBF55
:109ED000DF91CF911F910895CF93DF938A30D0F512
:109EE0006233710538F061369DE6790728F060E647
:109EF0007DE602C062E370E0D42FC82F80E090E0DE
:109F00000E94F6CB20E030E04AE754E40E9417CEEE
:109F100020E030E04CE852E40E9457CC9B01AC01B9
:109F200060E070E08AEF94E40E9417CE0E9489CE30
:109F30009B01DD2321F022273327261B370B8FB708
:109F4000F89495E1C99FF0011124E753FF4E318742
:109F500020878FBFDF91CF9108958A3010F40C9441
:109F6000C84E08958A3010F40C94E34E08958A3058
:109F700058F495E1899FF0011124E753FF4E818148
:109F8000928196958795089580E090E008958A30B3
:109F900010F40C94FE4E08951F920F920FB60F927C
:109FA00011240BB60F920F931F932F933F934F9350
:109FB0005F936F937F938F939F93AF93BF93CF9351
:109FC000EF93FF938091260F893048F01092260F6F
:109FD00080917811882399F0809171110DC0E091E2
:109FE000260FE15025E1E29FF0011124E753FF4ED7
:109FF0008781882321F0808192B1892782B9E091FD
:10A00000260F85E1E89FF0011124E753FF4E878179
:10A01000882321F0808192B1892B82B9E091260FAB
:10A02000C5E1CE9FF0011124E753FF4E8085918555
:10A03000892B09F04DC0E091260FCE9FF00111242D
:10A04000E753FF4E8285813009F061C00E94FD8692
:10A05000E091260FCE9FF0011124E753FF4E0385B8
:10A06000148525853685E091260FCE9FF0011124B9
:10A07000E753FF4E0784F089E02DAB01BC01401B84
:10A08000510B620B730BCF01A0E0B0E08417950772
:10A09000A607B707E0F5E091260FA091260FCA9F0B
:10A0A000D0011124A753BF4E53968D919C91549784
:10A0B000CE9FF0011124E753FF4E91878087E091F6
:10A0C000260FCE9FF0011124E753FF4E82E08287D6
:10A0D0008091260F0E94914A8091260F8F5F809376
:10A0E000260FFF91EF91CF91BF91AF919F918F91EB
:10A0F0007F916F915F914F913F912F911F910F91A0
:10A100000F900BBE0F900FBE0F901F901895E0910F
:10A11000260F809184009091850025E1E29FF00157
:10A120001124E753FF4E21813281820F931F9093B8
:10A13000890080938800D0CF1F93CF93DF938091C5
:10A14000250F811173C01092260F9FB7F89485E1F7
:10A1500028EB3BE04CED55E064E971E1A1E0B0E0B3
:10A16000E091260FE93008F052C0E091260F8E9F53
:10A17000F0011124E753FF4E32832183E091260F33
:10A180008E9FF0011124E753FF4E56834583E091E3
:10A19000260F8E9FF0011124E753FF4E74836383D3
:10A1A000E091260FF091260FED0101C0CC0FFA953A
:10A1B000EAF78E9FF0011124E753FF4EC083E09130
:10A1C000260F8E9FF0011124E753FF4E1782E09176
:10A1D000260F8E9FF0011124E753FF4E1186108643
:10A1E000E091260F8E9FF0011124E753FF4E128657
:10A1F000E091260F8E9FF0011124E753FF4E148A41
:10A20000138AE091260FEF5FE093260FA9CF9FBF3F
:10A210008FB7F89420EA3FE03093731120937211C6
:10A22000109271118FBF81E08093250FDF91CF9144
:10A230001F9108950F931F93CF93DF938C01C62F27
:10A24000D42FDC0111968D919C911297DC01ED9138
:10A25000FC910190F081E02DD8016C911995F801E5
:10A2600081819281DC01ED91FC910190F081E02DE2
:10A270006C2F1995F80181819281DC01ED91FC919F
:10A280000190F081E02D6D2F1995F80180816C2FE0
:10A2900070E0680F711D6D0F711D6F7777278181D9
:10A2A0009281DF91CF911F910F910C9405830F93B1
:10A2B0001F93CF93DF938C01C62FD42FDC0111960F
:10A2C0008D919C911297DC01ED91FC910190F081B0
:10A2D000E02DD8016C911995F80181819281DC0102
:10A2E000ED91FC910190F081E02D6C2F1995F80112
:10A2F00081819281DC01ED91FC910190F081E02D52
:10A300006D2F1995F80180816C2F70E0680F711D19
:10A310006D0F711D6F77772781819281DF91CF91CA
:10A320001F910F910C9405834F925F926F927F92D1
:10A33000AF92BF92CF92DF92EF92FF921F93CF9393
:10A34000DF93DD24D39445E0C42EC2E0D0E053E097
:10A35000E52EF12CAA24A394B12C8091090F9091A1
:10A360000A0FDC01ED91FC910084F185E02D199537
:10A37000892B09F4D1C0109130018091090F90917F
:10A380000A0FDC01ED91FC910284F385E02D199513
:10A3900096B3B39A20918400309185002059384EAD
:10A3A00030938D0020938C00212F2C7119F0109286
:10A3B000240F2AC093FB992790F9E091240FE11113
:10A3C00016C0992351F28F3041F6D092240F80931A
:10A3D0000B0F8091070F9091080F892B09F0BDCFCB
:10A3E000B092080FA092070F1092060FB6CF9923D4
:10A3F00081F01092240F1092060F8091070F909118
:10A40000080F029709F0A9CFF092080FE092070F0A
:10A41000A4CF91E09E0F9093240FF0E0E55FF04F02
:10A420008083993109F099CF811173C08091220FF7
:10A4300082FF05C0F092080FE092070F6AC083FD0B
:10A44000F9CF8091070F9091080F019761F48091E7
:10A45000060F8F5F8093060F843058F0D093080F5B
:10A46000C093070F06C0D093080FC093070F109238
:10A47000060F8091050F8F5F8093050F9091040F59
:10A48000981708F044C0D092030FA3EEBEE0ECE0B2
:10A49000FFE040E050E0BA0110E0CF01FC011B30CA
:10A4A00098F401964080512C612C712C012E04C02F
:10A4B000440C551C661C771C0A94D2F74429552974
:10A4C00066297729185FEACF9A013770205E3340FA
:10A4D000C29EC001C39E900D112497FD079623E0F4
:10A4E000959587952A95E1F784529A4F8D939D9380
:10A4F0001B503BE076956795579547953A95D1F770
:10A500008FE0A330B80749F61092050F02C01092F1
:10A51000030F1092240F21CFDF91CF911F91FF9055
:10A52000EF90DF90CF90BF90AF907F906F905F9053
:10A530004F9008958091F60B833031F48091E10EB5
:10A540009091E20E0C94904308958091F60B823026
:10A5500031F48091DF0E9091E00E0C9494510895A7
:10A560000E94A5520C949A521092A2101092AC1014
:10A570001092B6101092C01010924A1080E090E035
:10A58000FC01E35BFF4E1182079684359105C1F70C
:10A5900008950895CF92DF92EF92FF920F931F9349
:10A5A000CF93DF936C017A018B01C0E0D0E0CE1530
:10A5B000DF0589F0D8016D918D01D601ED91FC91F7
:10A5C0000190F081E02DC6011995892B11F47E01CF
:10A5D00002C02196ECCFC701DF91CF911F910F915F
:10A5E000FF90EF90DF90CF900895FC01A089B18992
:10A5F0008C91A689B78982FD0FC09C91818D8F5F58
:10A600008F73228D821749F0218DDF01A20FB11DBA
:10A610005D969C93818F08958C910895089580E0B4
:10A6200090E00895FC01538D448D252F30E0842F58
:10A6300090E0821B930B541710F0CF96089501976A
:10A640000895FC01918D828D981761F0828DDF0154
:10A65000A80FB11D5D968C91928D9F5F9F73928F15
:10A6600090E008958FEF9FEF0895FC01918D828D0A
:10A67000981731F0828DE80FF11D858D90E00895D7
:10A680008FEF9FEF0895FC01918D228D892F90E02F
:10A69000805C9F4F821B91098F73992708958EEFDD
:10A6A00097E00E94435321E0892B09F420E0822F98
:10A6B00008958BE998E00E94435321E0892B09F427
:10A6C00020E0822F089588E399E00E94435321E01F
:10A6D000892B09F420E0822F089585ED99E00E94EE
:10A6E000435321E0892B09F420E0822F0895FC01D7
:10A6F000848DDF01A80FB11DA35ABF4F2C91848D0B
:10A7000090E001968F739927848FA689B7892C933F
:10A71000A089B1898C9180648C93938D848D9813DA
:10A7200006C00288F389E02D80818F7D80830895A3
:10A73000EF92FF920F931F93CF93DF93EC0181E091
:10A74000888F9B8D8C8D981305C0E889F98980814D
:10A7500085FD24C0F62E0B8D10E00F5F1F4F0F7389
:10A760001127E02E8C8DE8120CC00FB607FCFACF33
:10A77000E889F989808185FFF5CFCE010E94775362
:10A78000F1CF8B8DFE01E80FF11DE35AFF4FF082F0
:10A790000B8FEA89FB898081806207C0EE89FF897F
:10A7A0006083E889F98980818064808381E090E01A
:10A7B000DF91CF911F910F91FF90EF900895CF936C
:10A7C000DF93EC01888D8823C9F0EA89FB898081B9
:10A7D00085FD05C0A889B9898C9186FD0FC00FB68B
:10A7E00007FCF5CF808185FFF2CFA889B9898C91CC
:10A7F00085FFEDCFCE010E947753E7CFDF91CF9158
:10A80000089580E090E0892B21F00E946D53811122
:10A8100019C080E090E0892B21F00E9463538111E0
:10A8200014C080E090E0892B21F00E9459538111DF
:10A830000FC080E090E0892B81F00E944F5381117E
:10A840000AC008950E940000E4CF0E940000E9CFF2
:10A850000E940000EECF0C940000089590E0FC01EF
:10A860003197E231F10508F04EC08827EA59FE4FD2
:10A870008F4F0C9491CF809180008F7703C080918F
:10A8800080008F7D80938000089580918000877F75
:10A89000F9CF84B58F7702C084B58F7D84BD0895CC
:10A8A0008091B0008F7703C08091B0008F7D80933E
:10A8B000B0000895809190008F7707C0809190003C
:10A8C0008F7D03C080919000877F809390000895D2
:10A8D0008091A0008F7707C08091A0008F7D03C07A
:10A8E0008091A000877F8093A0000895809120012F
:10A8F0008F7707C0809120018F7D03C08091200158
:10A90000877F8093200108950E94BED16115710553
:10A9100079F0FB0101900020E9F73197AF01461B68
:10A92000570BDC01ED91FC910280F381E02D19942D
:10A9300080E090E008950F931F93CF93DF938C01F5
:10A94000EB01FC01808191810097B1F068817981F0
:10A950006115710579F0428153812C813D81421747
:10A96000530740F00E94D7D18C819D81F8019583D7
:10A97000848313C00E943DD088819981F80191831E
:10A9800080838A819B81938382838C819D8195833F
:10A990008483198218821B821A821D821C82DF9195
:10A9A000CF911F910F9108950F931F93CF93DF9332
:10A9B000EC0188819981009729F02A813B81261733
:10A9C000370788F48B016F5F7F4F0E94D5D00097C7
:10A9D00061F0998388831B830A832C813D81232B1B
:10A9E00011F4FC01108281E001C080E0DF91CF9181
:10A9F0001F910F910895EF92FF920F931F93CF93A2
:10AA0000DF93FB0124813581E080F180FC0104812A
:10AA10001581E114F10411F480E017C0211531050E
:10AA200099F0EC01020F131FB8010E94D45488233F
:10AA300099F3288139818C819D81B701820F931F01
:10AA40000E94D7D11D830C8381E0DF91CF911F91AC
:10AA50000F91FF90EF900895EF92FF920F931F9345
:10AA6000CF93DF93EC017B018A01BA010E94D45499
:10AA70002881398181110DC02115310519F0C901D5
:10AA80000E943DD0198218821D821C821B821A826C
:10AA900006C01D830C83B701C9010E94D7D1CE0126
:10AAA000DF91CF911F910F91FF90EF900895CF9379
:10AAB000DF93EC016115710559F0FB010190002055
:10AAC000E9F73197AF01461B570B0E942C550CC07C
:10AAD00088819981009711F00E943DD019821882D7
:10AAE0001D821C821B821A82CE01DF91CF910895B4
:10AAF000FC01808191810C943DD00F931F93CF93E3
:10AB0000DF93CDB7DEB762970FB6F894DEBF0FBE06
:10AB1000CDBF8C01CB01F801118210821382128209
:10AB20001582148250E0BE016F5F7F4F0E9475CB8B
:10AB3000BE016F5F7F4FC8010E94575562960FB6E6
:10AB4000F894DEBF0FBECDBFDF91CF911F910F9163
:10AB500008950F931F93CF93DF93CDB7DEB7299757
:10AB60000FB6F894DEBF0FBECDBF8C01862FF80163
:10AB700011821082138212821582148250E0BE016B
:10AB80006F5F7F4F90E00E94BCCBBE016F5F7F4F35
:10AB9000C8010E94575529960FB6F894DEBF0FBE24
:10ABA000CDBFDF91CF911F910F910895FC011182CC
:10ABB000108213821282158214826115710551F080
:10ABC000FB0101900020E9F73197AF01461B570BBD
:10ABD0000C942C550895CF93DF9300D01F92CDB7DE
:10ABE000DEB7611571058105910579F09B01AC0116
:10ABF00069833A834B835C830E9468CB29813A81C5
:10AC00004B815C810E9447CD03C060E070E0CB01C6
:10AC10000F900F900F900F90DF91CF9108954F926A
:10AC20005F926F927F92EF92FF920F931F93CF9359
:10AC3000DF93CDB7DEB7A1970FB6F894DEBF0FBE96
:10AC4000CDBF7C01FA01CB0119A2223008F42AE021
:10AC50008E010F5D1F4F422E512C612C712CBF01B4
:10AC6000A30192010E9479CDF901CA010150110995
:10AC70006A3014F4605D01C0695CD8016C93232BC9
:10AC8000242B252B61F7B801C7010E948654A19699
:10AC90000FB6F894DEBF0FBECDBFDF91CF911F91ED
:10ACA0000F91FF90EF907F906F905F904F9008957D
:10ACB0006BE876E00C9486540F931F93CF93DF9349
:10ACC000EC010E9486548C01CE010E945856800FE0
:10ACD000911FDF91CF911F910F910895DC01ED91AC
:10ACE000FC910190F081E02D19944F925F926F9248
:10ACF0007F928F929F92AF92BF92CF92DF92EF920C
:10AD0000FF92CF93DF93EC016A017B01B22E9A018F
:10AD1000AB01C701B6010E94CCCE882319F06EE8C2
:10AD200076E027C026013701E89477F82FEF3FEF50
:10AD30004FE75FE7C301B2010E94CCCE81110DC085
:10AD40002FEF3FEF4FE75FE7C301B2010E94F1CB66
:10AD500018161CF462E976E00CC02FEF3FEF4FE7C6
:10AD60005FE4C701B6010E94BFCE18169CF466E9E5
:10AD700076E0CE01DF91CF91FF90EF90DF90CF9002
:10AD8000BF90AF909F908F907F906F905F904F900B
:10AD90000C9486542FEF3FEF4FE75FECC701B601ED
:10ADA0000E94F1CB87FDE3CF20E030E0A901C7018D
:10ADB000B6010E94F1CB87FF0AC06DE2CE010E946E
:10ADC0006E564C01F7FAF094F7F8F09402C0812C1B
:10ADD000912CA12C60E070E080E09FE3AB1441F087
:10ADE00020E030E040E251E40E9417CEA394F6CF79
:10ADF0009B01AC01C701B6010E94ABCD2B013C0108
:10AE00000E9490CE6B017C010E94F6CB9B01AC01AD
:10AE1000C301B2010E94AACD2B013C012AE0B70177
:10AE2000A601CE010E940F567C01E80CF91CBB2044
:10AE300031F06EE2CE010E946E56E80EF91EDB2C58
:10AE4000DD2029F120E030E040E251E4C301B2010D
:10AE50000E9457CC2B013C010E9490CE4B01A12CAB
:10AE6000B12C2AE0B501A401CE010E940F56E80ED4
:10AE7000F91EC501B4010E94F6CB9B01AC01C301D0
:10AE8000B2010E94AACD2B013C01DA94D9CFC701AF
:10AE9000DF91CF91FF90EF90DF90CF90BF90AF9078
:10AEA0009F908F907F906F905F904F9008950C943B
:10AEB0008654EF92FF920F931F93CF93DF938C01F1
:10AEC0007B01C0E0D0E0F701EC0FFD1F6491662329
:10AED00061F0D801ED91FC910190F081E02DC80165
:10AEE0001995892B11F02196EECFCE01DF91CF91EC
:10AEF0001F910F91FF90EF9008950F931F93CF93A1
:10AF0000DF93EC010E9459578C01CE010E945856E4
:10AF1000800F911FDF91CF911F910F9108951F9284
:10AF20000F920FB60F9211240BB60F922F933F93EF
:10AF30004F935F936F937F938F939F93AF93BF9341
:10AF4000EF93FF938EEF97E00E947753FF91EF917D
:10AF5000BF91AF919F918F917F916F915F914F9131
:10AF60003F912F910F900BBE0F900FBE0F901F902F
:10AF700018951F920F920FB60F9211240BB60F92D5
:10AF80002F933F934F935F936F937F938F939F93F1
:10AF9000AF93BF93EF93FF938EEF97E00E94F5522C
:10AFA000FF91EF91BF91AF919F918F917F916F91A1
:10AFB0005F914F913F912F910F900BBE0F900FBE5D
:10AFC0000F901F9018951F920F920FB60F92112499
:10AFD0000BB60F922F933F934F935F936F937F9393
:10AFE0008F939F93AF93BF93EF93FF938BE998E079
:10AFF0000E947753FF91EF91BF91AF919F918F91F5
:10B000007F916F915F914F913F912F910F900BBE68
:10B010000F900FBE0F901F9018951F920F920FB6B2
:10B020000F9211240BB60F922F933F934F935F9380
:10B030006F937F938F939F93AF93BF93EF93FF9300
:10B040008BE998E00E94F552FF91EF91BF91AF918B
:10B050009F918F917F916F915F914F913F912F9130
:10B060000F900BBE0F900FBE0F901F9018951F9260
:10B070000F920FB60F9211240BB60F922F933F939E
:10B080004F935F936F937F938F939F93AF93BF93F0
:10B09000EF93FF9388E399E00E947753FF91EF913C
:10B0A000BF91AF919F918F917F916F915F914F91E0
:10B0B0003F912F910F900BBE0F900FBE0F901F90DE
:10B0C00018951F920F920FB60F9211240BB60F9284
:10B0D0002F933F934F935F936F937F938F939F93A0
:10B0E000AF93BF93EF93FF9388E399E00E94F552EB
:10B0F000FF91EF91BF91AF919F918F917F916F9150
:10B100005F914F913F912F910F900BBE0F900FBE0B
:10B110000F901F9018951F920F920FB60F92112447
:10B120000BB60F922F933F934F935F936F937F9341
:10B130008F939F93AF93BF93EF93FF9385ED99E028
:10B140000E947753FF91EF91BF91AF919F918F91A3
:10B150007F916F915F914F913F912F910F900BBE17
:10B160000F900FBE0F901F9018951F920F920FB661
:10B170000F9211240BB60F922F933F934F935F932F
:10B180006F937F938F939F93AF93BF93EF93FF93AF
:10B1900085ED99E00E94F552FF91EF91BF91AF913B
:10B1A0009F918F917F916F915F914F913F912F91DF
:10B1B0000F900BBE0F900FBE0F901F901895CF935E
:10B1C000DF93EC01E881F9810680F781E02D199584
:10B1D000EA89FB8980818F7E8083EA89FB8980816F
:10B1E000877F8083EA89FB8980818F778083EA89E2
:10B1F000FB8980818F7D80838A8D898FDF91CF91BC
:10B200000895CF92DF92EF92FF921F93CF93DF9337
:10B21000EC016A017B01122FE889F98982E08083C1
:10B220004115514E61057105B1F060E079E08DE3A3
:10B2300090E0A70196010E9479CDDA01C90101973A
:10B24000A109B109B695A79597958795AC014115C8
:10B2500080E15807A8F0E889F989108260E874E86D
:10B260008EE190E0A70196010E9479CDBA01A90173
:10B270004150510961097109769567955795479530
:10B28000EC85FD855083EE85FF854083188EEC8923
:10B29000FD891083EA89FB89808180618083EA8946
:10B2A000FB89808188608083EA89FB89808180684E
:10B2B0008083EA89FB8980818F7D8083DF91CF91B4
:10B2C0001F91FF90EF90DF90CF900895CF93DF9381
:10B2D000282F30E0F901E359F14E8491F901E95D3D
:10B2E000F14ED491F901EF51F24EC491CC2391F07B
:10B2F00081110E942E54EC2FF0E0EE0FFF1FE95356
:10B30000F24EA591B491EC91ED2381E090E021F40F
:10B3100080E002C080E090E0DF91CF9108951F931C
:10B32000CF93DF93282F30E0F901E359F14E849158
:10B33000F901E95DF14ED491F901EF51F24EC4915A
:10B34000CC23C9F0162F81110E942E54EC2FF0E06F
:10B35000EE0FFF1FE355F24EA591B4918FB7F8940D
:10B36000111105C09C91ED2FE095E92302C0EC91ED
:10B37000ED2BEC938FBFDF91CF911F910895CF9369
:10B38000DF9390E0FC01E95DF14E2491FC01EF5167
:10B39000F24E8491882361F190E0880F991FFC019F
:10B3A000ED56F24EC591D491FC01E355F24EA591B4
:10B3B000B491611109C09FB7F894888120958223C8
:10B3C0008883EC912E230BC0623061F49FB7F89410
:10B3D0003881822F809583238883EC912E2B2C93A8
:10B3E0009FBF06C08FB7F894E8812E2B28838FBFAC
:10B3F000DF91CF9108951F93CF93DF93182FEB0127
:10B4000061E00E94BF59209711F460E004C0CF3F73
:10B41000D10539F461E0812FDF91CF911F910C9418
:10B420008F59E12FF0E0E359F14EE4914E2F50E0B7
:10B43000FA013197E231F10508F09DC08827E858FC
:10B44000FE4F8F4F0C9491CF84B5806884BDC7BDEB
:10B4500097C084B5806284BDC8BD92C080918000D1
:10B46000806880938000D0938900C093880088C052
:10B4700080918000806280938000D0938B00C09385
:10B480008A007EC080918000886080938000D09385
:10B490008D00C0938C0074C08091B0008068809350
:10B4A000B000C093B3006CC08091B0008062809304
:10B4B000B000C093B40064C0809190008068809315
:10B4C0009000D0939900C09398005AC0809190004A
:10B4D000806280939000D0939B00C0939A0050C0EC
:10B4E00080919000886080939000D0939D00C093DD
:10B4F0009C0046C08091A00080688093A00080914D
:10B50000A0008F7B8093A000D093A900C093A800D7
:10B5100037C08091A00080628093A000D093AB00E0
:10B52000C093AA002DC08091A00088608093A000E5
:10B53000D093AD00C093AC0023C0809120018068FF
:10B5400080932001D0932901C093280119C08091D4
:10B550002001806280932001D0932B01C0932A01A7
:10B560000FC080912001886080932001D0932D012D
:10B57000C0932C0105C0C038D1050CF04BCF45CF8E
:10B58000DF91CF911F91089581E08093ED0B089595
:10B5900081E08093EE0B089581E08093EF0B089596
:10B5A0002F923F924F925F926F927F928F929F92D3
:10B5B000AF92BF92CF92DF92EF92FF920F931F93C1
:10B5C000CF93DF9300D000D0CDB7DEB74DB65EB6D7
:10B5D0000E94A5520E949A520E9433AA029709F033
:10B5E000EFC20E941CAA882309F4E4C2C090BA14D6
:10B5F000D090BB14E090B814F090B914B601C70114
:10B600000E94734D8823F1F0F701E250FE4F00E0F5
:10B6100010E0819191918C159D0571F40E94FD8639
:10B62000000F111F000F111FF701E00FF11F6083C2
:10B6300071838283938308C00F5F1F4F0E31110502
:10B6400041F702C00E9409AB1092F00BEDB6FEB6B6
:10B650004091F30B5091F40BCA01880F991FADB6BE
:10B66000BEB6A81AB90A0FB6F894BEBE0FBEADBEDC
:10B670000DB71EB70F5F1F4F8091F60B823069F038
:10B68000833029F1813009F071C0B8018091C31471
:10B690009091C4140E9463A733C03FB7F89420E090
:10B6A000822F90E08417950774F4880F991FF80192
:10B6B000E80FF91FDC01AD51B14F8D919C91918341
:10B6C00080832F5FEDCF3FBF1092030F19C03FB7AC
:10B6D000F89420E0822F90E08417950774F4880F87
:10B6E000991FF801E80FF91FDC01AE5BB04F8D9197
:10B6F0009C91918380832F5FEDCF3FBF1092C01448
:10B7000020E06AE071E0822F90E04091F30B5091CD
:10B71000F40B8417950754F5689FF001699FF00DAD
:10B720001124E855F04FA085B1858C918823E1F074
:10B73000A081B1813C91C801830F911D830F911DA0
:10B74000DC0112978D919C91A281B3814D915C9106
:10B7500011970480F581E02D4817590711F41082E4
:10B7600003C070838D939C932F5FCDCF0FB6F89459
:10B77000FEBE0FBEEDBE8091A210882321F081EAAB
:10B7800090E10E9451AA8091AC10882321F08BEAAD
:10B7900090E10E9451AA8091B610882321F085EB98
:10B7A00090E10E9451AA8091C010882321F08FEB74
:10B7B00090E10E9451AA8091F10B882309F465C0A1
:10B7C0008091B610811105C08091C010882309F4C2
:10B7D00050C08091B9109091BA10E091BD10F091D5
:10B7E000BE10238134812817390724F48085811104
:10B7F00009C00EC0218132818217930734F48085FD
:10B80000811106C088E090E005C080E190E002C0B0
:10B8100080E290E02091C3103091C410E091C710F5
:10B82000F091C810438154814217530724F42085B6
:10B83000222349F00AC041815281241735073CF484
:10B840002085222311F0816003C0846001C08260E2
:10B8500020914810309149102817390719F4109297
:10B860004A1007C0909349108093481081E080935C
:10B870004A108091481090914910429709F4A4C150
:10B8800081E08093C2108093B810AEE4B0E161E52E
:10B8900070E188EE682E83E0782E22242394FD0147
:10B8A00031978081882309F47CC11496CD90DC9077
:10B8B0001597DE82CD82F6018781882309F471C154
:10B8C0008C91882309F46DC111964D915C9112976A
:10B8D00030847301E41AF50A1E141F042CF07A0157
:10B8E000F8EEEF1AF3E0FF0A20E030E001E010E0AC
:10B8F000EFE0F7E290E0832C912CA32CB12CC12C2B
:10B90000D12CA982BA82CB82DC82650182E0C81A7E
:10B91000D108081519050CF04AC08BE0C816D104EF
:10B92000E0F5F6018827E657FE4F8F4F0C9491CF34
:10B93000F901E15BF94F27C0F901E75BF94F23C03B
:10B94000F901EF5BF94F1FC0F901E95CF94F1BC02A
:10B95000F901E55DF94F17C0F901E35EF94F13C036
:10B96000F901E35FF94F0FC0F901E550FA4F0BC041
:10B97000F901E951FA4F07C0F901EF52FA4F03C03C
:10B98000F901E754FA4F0280F381E02DE41BF50B37
:10B99000F7FF03C0F195E195F109EE15FF0514F4E9
:10B9A000902F7F010F5F1F4F2E5F3F4FB2CF9F5FE2
:10B9B000ED81FE818185882309F4EAC0032D10E022
:10B9C000F8013297EB30F10508F0E2C08827EB561A
:10B9D000FE4F8F4F0C9491CF913009F0ACC0C3C093
:10B9E000913009F4D4C0933009F0D2C0A4C0913092
:10B9F00009F4CBC0923009F4CAC0933009F4B3C043
:10BA0000943009F0C5C097C0913009F4BCC09230A1
:10BA100009F4BBC0943009F4A6C0953009F0B8C051
:10BA20008AC0913009F4ADC0923009F4ACC09330B3
:10BA300009F4ABC0943009F4AAC0953009F493C05E
:10BA4000963009F0A5C077C0913009F498C09230C3
:10BA500009F497C0933009F496C0953009F497C063
:10BA6000963009F480C0973009F092C064C09130DC
:10BA700009F483C0923009F482C0933009F481C084
:10BA8000943009F480C0953009F47FC0963009F4F1
:10BA90007EC0973009F467C0983009F079C04BC078
:10BAA000913009F468C0923009F467C0933009F40A
:10BAB00066C0943009F465C0963009F466C09730CA
:10BAC00009F465C0983009F44EC0993009F060C09F
:10BAD00032C0913009F44DC0923009F44CC093301B
:10BAE00009F44BC0943009F44AC0953009F449C0B8
:10BAF000963009F448C0973009F447C0983009F4EB
:10BB000046C0993081F19A3009F042C014C091309A
:10BB100071F1923071F1933071F1943071F195308F
:10BB200071F1973081F1983081F1993081F19A303B
:10BB3000D1F09B3069F591E02BC09130B1F092309B
:10BB4000B1F09330B1F09430B1F09530B1F096305F
:10BB5000B1F09730B1F09830B1F09930B1F09A303F
:10BB6000B1F09B30A9F492E013C09CE011C09BE0BF
:10BB70000FC09AE00DC099E00BC098E009C097E0B3
:10BB800007C096E005C095E003C094E001C093E0D3
:10BB9000FB018081891302C01C9203C02C92FB011F
:10BBA00090831796695F7F4FF0E1A23ABF0709F0D3
:10BBB00076CE04C00E94B4520E9409AB81E066C0F8
:10BBC0000E94B45280E062C0E0904B10F0904C10A4
:10BBD0001E141F040CF055C08091B7100091B814CA
:10BBE0001091B9146091610F7091620F8823B1F0C8
:10BBF00081E08093B810C8010E94734D811115C077
:10BC0000A701FF0C660B770B23E03AEAC8010E94FC
:10BC1000DA4D9093620F8093610F07C0C8010E94B4
:10BC2000734D811102C01092B8108091C110009123
:10BC3000B8141091B91460915F0F7091600F882350
:10BC4000D1F081E08093C210C8010E94734D811130
:10BC50001CCE40914B1050914C10052E000C660BE1
:10BC6000770B20E03AEAC8010E94DA4D9093600F0A
:10BC700080935F0F0ACEC8010E94734D811105CEDB
:10BC800002C01092B8101092C210FFCD0FB6F894F7
:10BC90005EBE0FBE4DBE26960FB6F894DEBF0FBE39
:10BCA000CDBFDF91CF911F910F91FF90EF90DF906B
:10BCB000CF90BF90AF909F908F907F906F905F904C
:10BCC0004F903F902F900895CF9380915E0FC09139
:10BCD0000A02811101C1C23009F450C0C33009F415
:10BCE0009DC0C13009F028C18091EF0B811124C1A2
:10BCF00081E090E00E94A8CF9093C4148093C31475
:10BD000062E083E00E94BF5910923F0F1092BD1471
:10BD10001092BC141092C11480E090E0FC01EE0F70
:10BD2000FF1FE35DF04F118210820196883091056C
:10BD3000A9F710923E0F10923D0F80916A008C601F
:10BD400080936A00ED9A8FB7F89420918400309127
:10BD500085003093280F2093270F8FBF2CEC3AE5F6
:10BD60004AEF50E060E070E08091B8149091B9140F
:10BD70000E94DA4D81E080935E0FDEC08091EE0B71
:10BD80008111DAC081E090E00E94A8CF9093E00E8C
:10BD90008093DF0E809104018E7F80930401809157
:10BDA00005018160809305018EEF97E090930A0F63
:10BDB0008093090F2EE240EA56E861E070E00E94AD
:10BDC0000159809165008B7F809365001092350149
:10BDD00089E0809334018EE2809332018CEF80936E
:10BDE000300180E9809331011092080F1092070F03
:10BDF0001092060F1092050F1092030FE3EEFEE073
:10BE00008CED95E0819391932FE0E330F207D1F729
:10BE1000C1E0C093040F28EC3AE551C08091ED0BCE
:10BE200081118AC081E090E00E94A8CF9093E20E39
:10BE30008093E10E809104018E7F809304018091B4
:10BE400005018160809305018EEF97E09093410F8B
:10BE50008093400F26E040E052EC61E070E00E94E9
:10BE60000159809165008B7F8093650010923501A8
:10BE700080E18093340186E0809332018EEF8093DD
:10BE8000300180E9809331011092BF141092BE14EA
:10BE900010922C0F10922B0F1092C014E2E4FFE0CE
:10BEA0008CED95E0819391932FE0EE35F207D1F779
:10BEB00010922A0FC1E0C093290F24EC3AE54AEF13
:10BEC00050E060E070E08091B8149091B9140E9445
:10BED000DA4DC0935E0F30C0C23069F0C330D1F08C
:10BEE000C13051F58091EF0B811126C08091BC14B7
:10BEF0009091BD141DC08091EE0B81111DC08091E9
:10BF0000DF0E9091E00E0E9494518091070F909166
:10BF1000080F0EC08091ED0B81110EC08091E10ED3
:10BF20009091E20E0E9490438091BE149091BF14B4
:10BF3000029711F4C093F60B80910A028230A1F1AE
:10BF4000833009F454C0813009F074C08091EF0B44
:10BF5000882309F46FC0ED98E59A10923F0F109274
:10BF6000C2141092BD141092BC141092C11480E03F
:10BF700090E0FC01EE0FFF1FE35DF04F1182108295
:10BF8000019688309105A9F710923E0F10923D0F4F
:10BF90008091C3149091C4140E943DD010925E0F02
:10BFA0001092EE0B82E044C08091EE0B882309F4DE
:10BFB00041C08091090F90910A0F0E94DF58809133
:10BFC00031018F7780933101809131018F7E809391
:10BFD0003101109230018091DF0E9091E00E0E94AD
:10BFE0003DD010925E0F1092ED0B83E021C0809146
:10BFF000ED0B8823F9F08091400F9091410F0E9442
:10C00000DF58809131018F77809331018091310128
:10C010008F7E80933101109230018091E10E9091DA
:10C02000E20E0E943DD010925E0F1092EF0B81E065
:10C0300080930A028091B8149091B914CF910C9416
:10C04000EC4DAF92BF92CF92DF92EF92FF920F939F
:10C050001F93CF93DF937C016B015A01D0E0C0E0C6
:10C060008D2F90E0F701A181B2818A159B05D0F454
:10C07000F601E80FF91F60810CE915EC21E0332788
:10C08000C6270C0F111D211D311D2BBFF801C791B3
:10C09000ED91FC9111970190F081E02DCD01199562
:10C0A000DF5FDECFED91FC9111970190F081E02DE3
:10C0B0006C2FCD01DF91CF911F910F91FF90EF90E9
:10C0C000DF90CF90BF90AF901994CF93DF9300D0C3
:10C0D0001F921F92CDB7DEB7FE01319625E0DF013A
:10C0E0001D922A95E9F724E8298325E52C832AE285
:10C0F0002D836A834B8345E050E0BF010E9421609D
:10C1000065E070E080E090E00E94C38680E00F90E0
:10C110000F900F900F900F90DF91CF910895EF92B5
:10C12000FF921F93CF93DF931F92CDB7DEB77C01B1
:10C13000162FFC01618172810E944D7165E070E0F3
:10C1400080E090E00E94C38642E462E4C7010E945E
:10C150006560412F60E0C7010E946560811170C079
:10C1600040E061E0C7010E946560811169C040E064
:10C1700062E0C7010E946560811162C046E062E032
:10C18000C7010E94656081115BC040E063E0C701A8
:10C190000E946560811154C040E064E0C7010E94C4
:10C1A000656011E0811110E040E065E0C7010E9488
:10C1B0006560811101C01F5F40E066E0C7010E9419
:10C1C0006560811101C01F5F40E067E0C7010E9408
:10C1D0006560811101C01F5F40E068E0C7010E94F7
:10C1E0006560811101C01F5F40E069E0C7010E94E6
:10C1F0006560811101C01F5F44E06AE0C7010E94D1
:10C200006560811101C01F5F44E06AE0C7010E94C0
:10C210006560811101C01F5F62E370E080E090E023
:10C220000E94C38682E8898341E050E0BE016F5FCF
:10C230007F4FC7010E94216081E0183011F0111179
:10C2400080E00F90DF91CF911F91FF90EF900895C4
:10C25000CF93DF9300D01F92CDB7DEB72AEA2983B0
:10C26000FC0120812A836B834C8344E050E0BE01B3
:10C270006F5F7F4F0E9421600F900F900F900F9083
:10C28000DF91CF9108958091AA079091AB07DC01CF
:10C29000ED91FC910084F185E02D19958091AA071C
:10C2A0009091AB07DC01ED91FC910480F581E02DCC
:10C2B000199480911307882371F0109213078091CD
:10C2C0007913882341F06EE370E2809177139091A7
:10C2D00078130C947D5708958091F712833099F06C
:10C2E0008091130781110FC081E080931307809123
:10C2F0007913882341F069E270E28091771390917D
:10C3000078130C947D57089580911307882321F0AA
:10C3100080E090E00C94596180E090E00C946C61B6
:10C3200080911207833079F083E080931207809127
:10C330007913882341F068E170E28091771390913E
:10C3400078130C947D57089580911207823079F00C
:10C3500082E08093120780917913882341F067E08F
:10C3600070E280917713909178130C947D57089523
:10C3700080911207813079F081E0809312078091DB
:10C380007913882341F066EF7FE1809177139091D4
:10C3900078130C947D5708958091070180FF1BC08E
:10C3A00080917913882351F08BE39CE00E944FAC7D
:10C3B000811108C08091470C811104C08BE39CE07F
:10C3C0000C94024A67E970E2809177139091781398
:10C3D0000E947D57F3CF08958091070181FF1BC014
:10C3E00080917913882351F08AE09CE00E944FAC41
:10C3F000811108C08091160C811104C08AE09CE074
:10C400000C94024A6AE670E2809177139091781357
:10C410000E947D57F3CF08958091070180FF17C0D8
:10C4200080917913882331F08BE39CE00E944FAC1C
:10C43000882321F08BE39CE00C9463AC61E870E20C
:10C4400080917713909178130E947D57F3CF0895D0
:10C450008091070181FF17C080917913882331F003
:10C460008AE09CE00E944FAC882321F08AE09CE0A7
:10C470000C9463AC64E570E280917713909178132B
:10C480000E947D57F3CF089580917B13882371F02C
:10C490000E94467080917913882341F066EB7FE11A
:10C4A00080917713909178130C947D570895CF93D2
:10C4B000DF938091070181FD2AC0C0914007D09190
:10C4C000410780914407882371F08FE30E947F86A3
:10C4D000813092402CF010924107109240070AC020
:10C4E00081E090E003C08FE30E947F869093410734
:10C4F0008093400780914007909141078C179D07DA
:10C5000019F41092420703C081E080934207DF9143
:10C51000CF9108958091F712833059F02CF4813037
:10C52000E9F08230D9F030C0863044F08630B1F086
:10C530002BC080919F079091A0071FC080919F07FB
:10C540009091A007DC01ED91FC910480F581E02D34
:10C55000199580919D0790919E070FC08091A30728
:10C560009091A407DC01ED91FC910480F581E02D10
:10C5700019958091A1079091A207DC01ED91FC91A2
:10C580000480F581E02D19958091AA079091AB0761
:10C59000DC01ED91FC91E25BFF4F0190F081E02D19
:10C5A00019958091AA079091AB07DC01ED91FC9160
:10C5B0000484F585E02D60E070E019940E948A62A1
:10C5C0000E94C68880917B1381110E9446708091E1
:10C5D000AC079091AD07DC01ED91FC910480F581F1
:10C5E000E02D19958091A8079091A907DC01ED91A4
:10C5F000FC910480F581E02D19958091CF1288235C
:10C6000031F08091290790912A070C94BF4B08952F
:10C6100080917B13882339F180917213882319F15B
:10C62000109272130E94099E80918B11882319F039
:10C6300010928B110CC08091AA079091AB07DC017E
:10C64000ED91FC910288F389E02D60E019958091CD
:10C650007913882341F06FED7FE1809177139091FA
:10C6600078130E947D57109272130895CF93909182
:10C670007B139923D1F19091E00B911136C09091E9
:10C680007213911132C0C82F81E080937213809190
:10C690007D0F882331F081E00E945C9E10927D0F17
:10C6A00002C00E94189E80918B11882319F010926D
:10C6B0008B110CC08091AA079091AB07DC01ED9122
:10C6C000FC910288F389E02D61E01995809179133E
:10C6D000882359F0CC2349F06BEC7FE180917713EC
:10C6E00090917813CF910C947D57CF91089510922B
:10C6F0008C110E94686B81E00C943663CF93DF93BA
:10C70000C0917B0FD0917C0FBE018DE69CE00E9412
:10C71000734D882329F0BE018DE69CE00E948B4D6D
:10C7200010927C0F10927B0FDF91CF910895CF92E2
:10C73000DF92EF92FF920F931F93CF93DF93C090FE
:10C74000FC12D090FD12E090FE12F090FF121C142B
:10C750001D041E041F040CF041C080917B1388232C
:10C7600099F100917B0F10917C0FB8018DE69CE050
:10C770000E94734D8823D9F0EBE6FEE0C0E0D0E0E4
:10C78000819191918017910769F40E94FD86CC0FE9
:10C79000DD1FCC0FDD1FC359D34F688379838A8394
:10C7A0009B831CC02196CE31D10551F717C024E4DC
:10C7B00032E6B701A6018DE69CE00E94DA4D909327
:10C7C0007C0F80937B0F0AC0DF91CF911F910F9157
:10C7D000FF90EF90DF90CF900C947E63DF91CF912C
:10C7E0001F910F91FF90EF90DF90CF9008950F93DE
:10C7F0001F938091100281111EC00E94FD8600913E
:10C80000770F1091780F2091790F30917A0FAB014B
:10C81000BC01401B510B620B730B8091F012909185
:10C82000F112A0E0B0E0481759076A077B0718F03B
:10C8300081E0809310021F910F9108958091F01272
:10C840009091F112892B89F080911002882381F058
:10C850000E94FD866093770F7093780F8093790F15
:10C8600090937A0F10921002089581E08093100245
:10C870000895CF92DF92EF92FF92CF93DF93809152
:10C88000E00B811190C18091A707823040F0809128
:10C890007913882309F487C164E77FE193C080910D
:10C8A000D812882309F49AC08091F407882309F4E8
:10C8B00095C080917A13811191C08091E0128823F4
:10C8C00059F18091861190918711A0918811B091B2
:10C8D0008911892B8A2B8B2BF9F00E94FD86C09041
:10C8E0008611D0908711E0908811F09089119B01FA
:10C8F000AC012C193D094E095F0969017A012091AB
:10C90000E01230E0A8EEB3E00E949BCDC616D70639
:10C91000E806F90608F462C0C0912907D0912A07F9
:10C920008CAD9DAD892B11F01DAE1CAE8BA9813055
:10C9300009F073C08C899D8990932D0180932C01FF
:10C940008C899D899F8F8E8F0E94FD866DAB7EABFB
:10C950008FAB98AF8091AA079091AB07DC01ED9166
:10C96000FC910284F385E02D199581E080937A1380
:10C970002091F40730E0A8EEB3E00E949BCDAB011C
:10C98000BC0129E334E68DE69CE00E94DA4D9093E9
:10C9900076138093751380917913882309F403C16A
:10C9A00062E47FE180917713909178130E94595748
:10C9B0006091F40780917713909178130E943F70F3
:10C9C00069E37FE18091771390917813DF91CF91A4
:10C9D000FF90EF90DF90CF900C947D570E94F7630B
:10C9E00080911002882309F4DEC080917B138111AD
:10C9F000DAC081E080937B13809310020E941E6452
:10CA0000809179138823A1F06FEE7EE180917713F6
:10CA1000909178130E947D570BC0823009F094CF1B
:10CA20004FEF60E0CE010E946E4B8FEF90E08ACF17
:10CA300080917A13811137C08091D812882399F19F
:10CA40008091F407882379F18091E012882359F1CD
:10CA50008091861190918711A0918811B0918911D0
:10CA6000892B8A2B8B2BF9F00E94FD86C0908611B2
:10CA7000D0908711E0908811F09089119B01AC0152
:10CA80002C193D094E095F0969017A012091E012D4
:10CA900030E0A8EEB3E00E949BCDC616D706E806AC
:10CAA000F90608F44CC010927A1380917313909198
:10CAB0007413806190937413809373138091AA0709
:10CAC0009091AB07DC01ED91FC910280F381E02DA8
:10CAD000199580915D1381110E94086B8091A707C1
:10CAE000811125C04091F2125091F3124115510568
:10CAF000B1F0C1E0C0938B1160E070E027E733E64E
:10CB00008DE69CE00E94DA4DC0938C1180916B13EE
:10CB100081110E94496980E00E945C9E08C081E00A
:10CB200080938B1180937D0F80E00E943663DF91AC
:10CB3000CF91FF90EF90DF90CF900C94976364E2D9
:10CB40007FE180917713909178130E9459570E944A
:10CB5000FD86C0908611D0908711E0908811F090EA
:10CB600089116C197D098E099F0928EE33E040E098
:10CB700050E00E9479CDBA01A90121E0809177139C
:10CB8000909178130E940F566EEF7EE1809177139B
:10CB9000909178130E945957809177139091781350
:10CBA0000E94585680CFDF91CF91FF90EF90DF9099
:10CBB000CF900895AF92BF92CF92DF92EF92FF9203
:10CBC0000F931F93CF93DF9390916F0F91110BC031
:10CBD0002091B3073091B40730936E0F20936D0FFF
:10CBE00091E090936F0F9091650F91110BC0209180
:10CBF000B1073091B2073093640F2093630F91E037
:10CC00009093650FA0906D0FB0906E0F0091630F21
:10CC10001091640FD0917913843608F047C0C82F63
:10CC2000682F70E080E090E00E94F6CB20E030E0DA
:10CC300048EC52E40E9417CE6B017C01B501BB0C9D
:10CC4000880B990B0E94F8CB9B01AC01C701B60180
:10CC50000E9457CC0E9489CE7093B4076093B307AB
:10CC6000B801110F880B990B0E94F8CB9B01AC0106
:10CC7000C701B6010E9457CC0E9489CE7093B207BB
:10CC80006093B107DD2371F16EEC7EE18091771343
:10CC9000909178130E9459576C2F8091771390913F
:10CCA00078130E943F706CEC7EE10CC0B092B40728
:10CCB000A092B3071093B2070093B107DD2391F060
:10CCC00060EE7EE18091771390917813DF91CF91A0
:10CCD0001F910F91FF90EF90DF90CF90BF90AF909A
:10CCE0000C947D57DF91CF911F910F91FF90EF90A2
:10CCF000DF90CF90BF90AF900895CF93823069F4CA
:10CD00009091EB122091E8123091EC124091E912CF
:10CD10005091EA126091E7120CC09091E5122091B7
:10CD2000E2123091E6124091E3125091E4126091C8
:10CD3000E11260939614509393144093941430939B
:10CD40009214209395149093971490910002891750
:10CD5000B9F08093000290917913992389F0C82F3C
:10CD600063EB7EE180917713909178130E9459577D
:10CD70006C2F8091771390917813CF910C94287039
:10CD8000CF91089560E089E30E948F5960E08AE3C3
:10CD90000E948F5960E085E30E948F5960E085E032
:10CDA0000E948F5960E084E00E948F5960E087E024
:10CDB0000E948F5959980895CF93C0910F026C2FFC
:10CDC00089E30E948F5981E0C8276C2F8AE30E9473
:10CDD0008F59C0930F02CF910895CF93DF93C091E5
:10CDE0000E026C2F89E30E948F59D1E0DC276D2F52
:10CDF0008AE30E948F596C2F85E30E948F596D2F13
:10CE000085E00E948F596D2F84E00E948F596C2F0E
:10CE100087E00E948F59CC2311F0599801C0599A8C
:10CE200090910E0281E0892780930E02DF91CF91CD
:10CE30000895CF93DF938091980F81110DC01092C8
:10CE4000970F1092960F81E090E09093950F80934A
:10CE5000940F8093980F36C08091960F9091970F02
:10CE6000863191057CF18F38910534F48091940FCF
:10CE70009091950F019609C08D3521E0920754F4E9
:10CE80008091940F9091950F02969093950F8093B7
:10CE9000940F18C0863222E0920734F48091940FE8
:10CEA0009091950F0496F1CF883E93403CF4809189
:10CEB000940F9091950F8A5B9F4FE7CF1092950F3B
:10CEC0001092940F0E94ED66C091960FD091970F2B
:10CED000C93E83E0D8075CF01092980F0E94C266AA
:10CEE00023E937E648EE53E060E070E007C029E14F
:10CEF00037E6AE010D2E000C660B770B8DE69CE03D
:10CF00000E94DA4D9093930F8093920F8091940F2B
:10CF10009091950F8C0F9D1F9093970F8093960F74
:10CF2000DF91CF910895CF93DF938091B00788234D
:10CF300021F0DF91CF910C941967C091920FD0919D
:10CF4000930FBE018DE69CE00E94734D882329F06B
:10CF5000BE018DE69CE00E948B4DDF91CF910C9439
:10CF6000C266CF93C0918F0F6C2F70E088E00E9453
:10CF7000FB5989E180938E0F90910D02992311F056
:10CF8000CD5F01C0C350C0938F0F80918F0F873941
:10CF900070F0992321F08FEF80938F0F08C08D3DA3
:10CFA00030F086E980938F0F88E780938E0F809111
:10CFB0008F0F8F3F19F410920D0205C08A3118F4BB
:10CFC00081E080930D0240918E0F50E060E070E0B0
:10CFD00021EB37E68DE69CE00E94DA4D9093D41465
:10CFE0008093D314CF910895CF93DF93EC01BC01CC
:10CFF00088E00E94FB599E01A4E6B0E00E949BCD10
:10D000002FEF33E040E050E00E9447CD8091641361
:10D01000821320936413DF91CF910895CF93609191
:10D02000880F653FE0F5CAE0C60FC093880F809176
:10D03000870F882329F06C2F70E088E00E94FB594D
:10D040008091860F8823E1F08091A507882319F04D
:10D050006C2F70E012C080918B14882389F0A0910E
:10D060007E0F2C2F30E0B0E00E949BCD2FEF30E000
:10D0700040E050E00E9447CDB90184E00E94FB5996
:10D080002EE038E64FE050E060E070E08DE69CE096
:10D090000E94DA4D9093850F8093840F35C01092D3
:10D0A000880F6091840F7091850F1616170624F46F
:10D0B0008DE69CE00E948B4D8091870F882339F08C
:10D0C00061E088E00E948F5981E080938C14809108
:10D0D000860F8823A9F08091A507882311F061E0CD
:10D0E0000CC080918B14882339F060917E0F70E022
:10D0F00084E00E94FB5904C060E084E00E948F59E4
:10D100001092870F1092860FCF910895CF93DF93DF
:10D1100010928C14C091D314D091D414BE018DE61A
:10D120009CE00E94734D882329F0BE018DE69CE0AF
:10D130000E948B4D60E088E00E948F5980917913A6
:10D140008823D1F08091D514882319F068E871E222
:10D150000DC08091D214882319F06FE671E206C0E9
:10D1600080918113811108C060E671E2809177138C
:10D17000909178130E947D571092D5141092D2147A
:10D18000DF91CF91089581E080938C1461E088E075
:10D190000E948F5980917913882361F08091D51472
:10D1A000811108C062E571E2809177139091781344
:10D1B0000C947D5708958091D514811111C00E945F
:10D1C000866881E08093D51480917913882341F09B
:10D1D00067EB71E280917713909178130E947D57ED
:10D1E00080918D0F882329F060E088E00E948F599C
:10D1F00002C00E94C36890918D0F81E089278093BF
:10D200008D0F882329F0409160135091611304C061
:10D21000409162135091631360E070E02BED38E6AB
:10D220008DE69CE00E94DA4D9093D4148093D31441
:10D230000895CF9380918C0F81110FC081E080936E
:10D240008C0F80917913882341F060E271E2809124
:10D250007713909178130E947D57C0918B0F6C2F9C
:10D2600085E00E948F594091691350E060E070E0C2
:10D2700029E139E68DE69CE00E94DA4D90938A0F11
:10D280008093890F81E06C2F682760938B0FCF917B
:10D290000895CF938091870F811116C08091860FDA
:10D2A000811112C080918C14882319F081E0809341
:10D2B000870F8091A507811104C080918B1488236A
:10D2C00019F081E08093860F8091870F811105C04E
:10D2D0008091860F882309F477C00E9468CB22E8EA
:10D2E00030E040E050E00E9447CD665A6093880FDE
:10D2F0008091830F70E0681B71099B0177FF04C068
:10D3000022273327261B370B2D3331053CF077FFBF
:10D3100002C08C5301C0845C8093880FC091880F39
:10D32000C093830F8091870F882329F06C2F70E0C2
:10D3300088E00E94FB598091860F8823E1F080915C
:10D34000A507882319F06C2F70E012C080918B1410
:10D35000882389F0A0917E0F2C2F30E0B0E00E944E
:10D360009BCD2FEF30E040E050E00E9447CDB90167
:10D3700084E00E94FB59C63978F40E9468CB20E50E
:10D3800030E040E050E00E9447CDAB01BC01485D79
:10D390005F4F6F4F7F4F0EC00E9468CB22E330E09B
:10D3A00040E050E00E9447CDAB01BC01425E5F4FC0
:10D3B0006F4F7F4F29E439E68DE69CE00E94DA4DFD
:10D3C0009093850F8093840FCF9108956091900F73
:10D3D0007091910F8DE69CE00E94734D81112EC0DB
:10D3E00060E089E30E948F5960E08AE30E948F59D0
:10D3F00060E085E30E948F5960E085E00E948F59CC
:10D4000060E084E00E948F5960E087E00E948F59BD
:10D41000599880916613882319F02DEE36E602C0E4
:10D420002CED36E642E350E060E070E08DE69CE0F3
:10D430000E94E34D9093910F8093900F089560E0C8
:10D440008AE30C948F5961E08AE30C948F590F930F
:10D450001F93CF93DF938C01C1E0D0E00C171D0721
:10D46000ACF00E94236A64E670E080E090E00E94E5
:10D47000C3860E941F6AC017D10734F46AE570E0C2
:10D4800080E090E00E94C3862196E8CFDF91CF91A3
:10D490001F910F91089583E090E00C94276A82E039
:10D4A00090E00C94276A81E090E00C94276A60E099
:10D4B00089E30C948F5961E089E30C948F590F93A1
:10D4C0001F93CF93DF938C01C1E0D0E00C171D07B1
:10D4D000ACF00E945B6A64E670E080E090E00E943D
:10D4E000C3860E94576AC017D10734F46AE570E01A
:10D4F00080E090E00E94C3862196E8CFDF91CF9133
:10D500001F910F91089583E090E00C945F6A82E090
:10D5100090E00C945F6A81E090E00C945F6A109256
:10D520008C146091641370E088E00E94FB59809134
:10D530007913882341F061EA71E280917713909129
:10D5400078130C947D57089510928B148091A50741
:10D55000811104C060E084E00E948F5980917913AA
:10D56000882341F06FE371E28091771390917813F3
:10D570000C947D57089581E080938B148091A507CA
:10D58000811106C060917E0F70E084E00E94FB591B
:10D5900080917913882341F06DE271E280917713D5
:10D5A000909178130C947D570895CF93DF93C09199
:10D5B000900FD091910FBE018DE69CE00E94734DBB
:10D5C000882359F0BE018DE69CE00E948B4D10929D
:10D5D000910F1092900F0E94C26680915B13882376
:10D5E00021F0DF91CF910C94BB6ADF91CF91089528
:10D5F0001092A50780918B14811104C060E084E033
:10D600000C948F5960917E0F70E084E00C94FB596C
:10D6100081E08093A50761E084E00C948F59CF935B
:10D62000DF9360E085E00E948F5980918C0F81111B
:10D630000BC08091AA079091AB07DC01ED91FC91A2
:10D6400004ACF5ADE02D1995C091890FD0918A0FEA
:10D65000BE018DE69CE00E94734D882329F0BE0137
:10D660008DE69CE00E948B4D80917913882379F0A0
:10D6700020918C0F8091771390917813222319F0C9
:10D6800064E171E202C068E071E20E947D5710928D
:10D690008C0FDF91CF91089561E085E00E948F5952
:10D6A0008091AA079091AB07DC01ED91FC9104AC4D
:10D6B000F5ADE02D199580917913882341F06DEF38
:10D6C00070E280917713909178130C947D570895B0
:10D6D0006091840F7091850F1616170624F48DE65D
:10D6E0009CE00E948B4D84E68093880F0C940E681A
:10D6F00060E085E30E948F5910928A148091AA07F6
:10D700009091AB07DC01ED91FC9100ACF1ADE02D07
:10D71000199580917913882341F061EF70E280912F
:10D720007713909178130C947D57089561E085E309
:10D730000E948F5981E080938A148091AA0790916A
:10D74000AB07DC01ED91FC9100ACF1ADE02D19953A
:10D7500080917913882341F066EE70E2809177130F
:10D76000909178130C947D5708958F929F92AF9269
:10D77000BF92CF92DF92EF92FF9285E40E947F8664
:10D78000BC01990F880B990B0E94F8CB20E030E088
:10D7900040E85AE30E9457CC20E030E040EA50E4F1
:10D7A0000E9457CC6B017C0180910C02882351F0C0
:10D7B000C0927F0FD092800FE092810FF092820F83
:10D7C00010920C0226E636E646E65FE360917F0F94
:10D7D0007091800F8091810F9091820F0E9457CCA1
:10D7E0004B015C0120ED3CEC4CEC5DE3C701B60164
:10D7F0000E9457CC9B01AC01C501B4010E94ABCD86
:10D8000060937F0F7093800F8093810F9093820FAE
:10D810002DE33CE248E450E40E9457CC2AE939E980
:10D8200049E95EE30E94ABCDFF90EF90DF90CF908F
:10D83000BF90AF909F908F90089580910B028823A6
:10D8400059F00E94B56B20E030E040E050E40E94C7
:10D85000F1CB87FF3BC008950E94B56B20E030E01C
:10D860004AE754E40E9457CC0E9490CE209159136D
:10D8700030915A134091B0076217730710F4442394
:10D8800059F1442309F447C00E94B56B20E030E011
:10D890004AE754E40E9457CC0E9490CE209159133D
:10D8A00030915A1362177307B0F11092B00781E0FC
:10D8B0008093AF0780917913882369F16EEA70E253
:10D8C00080917713909178130C947D5710920B02EE
:10D8D00081E08093AF07089581E08093B0071092B4
:10D8E000AF0780917913882391F06DEC70E28091FD
:10D8F0007713909178130E9459570E94B9AC6AEC43
:10D9000070E280917713909178130E947D570E9466
:10D91000DE620C9493670895CF93DF9380910701A3
:10D9200080FD2AC0C0914607D091470780914A07E1
:10D93000882371F08EE30E947F86813092402CF024
:10D9400010924707109246070AC081E090E003C09A
:10D950008EE30E947F8690934707809346078091CD
:10D960004607909147078C179D0719F410924807B6
:10D9700003C081E080934807DF91CF910895CF9352
:10D98000DF93EC010E94FD86688379838A839B8301
:10D99000CE01DF91CF910895EF92FF921F93CF9325
:10D9A000DF93CDB7DEB765970FB6F894DEBF0FBE35
:10D9B000CDBF182F7B018CEE9AE00E94254881E0B4
:10D9C00080931A0B84E690E09093FD0A8093FC0A02
:10D9D00084E6E816F10418F484E6E82EF12CC70179
:10D9E00064E670E00E9469CF70931C0B60931B0B80
:10D9F0007093FF0A6093FE0A1093F90A8FEF810F6C
:10DA0000823010F41230D1F08CEE9AE00E94484837
:10DA10008091F70A882329F083EC95EFA8ECBFE307
:10DA200004C084EB98ECA6E9B0E48093160B9093C5
:10DA3000170BA093180BB093190B55C08091F70AE0
:10DA4000882329F084EB98ECA6E9B0E404C083ECC9
:10DA500095EFA8ECBFE38093160B9093170BA09360
:10DA6000180BB093190B8CEE9AE00E9452488091EB
:10DA70001A0B8823C1F11092F90A8EE690E09A837E
:10DA8000898388E290E09C838B838CE390E09E8383
:10DA90008D831D8A83E08F938DB79EB745970FB610
:10DAA000F8949EBF0FBE8DBFADB7BEB7119685E18E
:10DAB000FE01319601900D928A95E1F78CEE9AE085
:10DAC0000E945C480FB6F894DEBF0FBECDBF6596CE
:10DAD0000FB6F894DEBF0FBECDBFDF91CF911F917F
:10DAE000FF90EF9008958CEE9AE065960FB6F8944B
:10DAF000DEBF0FBECDBFDF91CF911F91FF90EF90A2
:10DB00000C94BF6C0F931F93CF93DF93EC01AB0189
:10DB100060E070E02AE00E940F568C01CE010E9466
:10DB20005856800F911FDF91CF911F910F9108954B
:10DB30008F929F92AF92BF92CF92DF92EF92FF921D
:10DB40000F931F93CF93DF931F921F92CDB7DEB732
:10DB5000082E000C990BAA0BBB0BFC013197EF3080
:10DB6000F10508F066C28827E056FE4F8F4F0C94EF
:10DB700091CF84E08093DB0A82E38093DC0A86E223
:10DB80008093DE0A81E08093E10A8093E20A809329
:10DB9000E00A4DE352E220E030E08091DB0A90E0C1
:10DBA000281739070CF08CC1FA0185919491A0E0F7
:10DBB000B0E0880F991FAA1FBB1FF901EE0FFF1FCE
:10DBC000EE0FFF1FEE58F54F80839183A283B3833E
:10DBD0002F5F3F4F4E5F5F4FE0CF84E08093DB0AC3
:10DBE00082E38093DC0A86E28093DE0A81E0809300
:10DBF000E10A8093E20A82E08093E00A45E352E280
:10DC000020E030E08091DB0A90E0281739070CF023
:10DC100057C1FA0185919491A0E0B0E0880F991F57
:10DC2000AA1FBB1FF901EE0FFF1FEE0FFF1FEE58DB
:10DC3000F54F80839183A283B3832F5F3F4F4E5F65
:10DC40005F4FE0CF84E08093DC0A85E28093DE0AB8
:10DC500081E08093E10A88E08093E20A83E0809388
:10DC6000E00A80E090E0FC01E35DFD4DE491DC0121
:10DC7000AD51B54FEC93019688309105A1F70E9404
:10DC8000B3901EC188E08093DB0A86E08093DC0AB3
:10DC900086E28093DE0A81E08093E10A8093E20AC3
:10DCA00084E08093E00A4DE152E220E030E0809190
:10DCB000DB0A90E0281739070CF002C1FA018591C0
:10DCC0009491A0E0B0E0880F991FAA1FBB1FF90133
:10DCD000EE0FFF1FEE0FFF1FEE58F54F808391836D
:10DCE000A283B3832F5F3F4F4E5F5F4FE0CF88E04B
:10DCF0008093DB0A81E08093DC0A97E29093DE0A4E
:10DD00008093E10A8093E20A85E08093E00A4DE087
:10DD100052E220E030E08091DB0A90E028173907DA
:10DD20000CF0CEC0FA0185919491A0E0B0E0880F8C
:10DD3000991FAA1FBB1FF901EE0FFF1FEE0FFF1F58
:10DD4000EE58F54F80839183A283B3832F5F3F4FBB
:10DD50004E5F5F4FE0CF82E18093DB0A81E08093EA
:10DD6000DC0A97E29093DE0A8093E10A8093E20A4C
:10DD70008FE08093E00A49EE51E220E030E08091AC
:10DD8000DB0A90E0281739070CF09AC0FA01859158
:10DD90009491A0E0B0E0880F991FAA1FBB1FF90162
:10DDA000EE0FFF1FEE0FFF1FEE58F54F808391839C
:10DDB000A283B3832F5F3F4F4E5F5F4FE0CFE09171
:10DDC000460BF091470B74978081918140E550E0BC
:10DDD00060E070E08A5B944F0E940B922AC182E15E
:10DDE0008093DB0A85E08093DC0A82E28093DE0A7E
:10DDF00081E08093E10A8093E20A87E08093E00A61
:10DE000080E993E3A0E0B0E08093720A9093730AF4
:10DE1000A093740AB093750AF2E08F2E912C01E062
:10DE200010E080E090E0A0E0BBE54CE454E060E06E
:10DE300070E024EEC22E2CE0D22EE12CF12C9801C1
:10DE4000220F331F220F331F5401AA0CBB1CAA0C34
:10DE5000BB1C2E58354FF901B7FF0DC0C082D182CF
:10DE6000E282F38295012E58354FF90140835183A8
:10DE7000628373830CC040835183628373839501F3
:10DE80002E58354FF901C082D182E282F382880F89
:10DE9000991FAA1FBB1F0E5F1F4FF2E08F0E911C30
:10DEA00022E18216910459F688E79FEFA0E0B0E0E6
:10DEB0008093B60A9093B70AA093B80AB093B90AB0
:10DEC0000E942291B6C0CE0101960E949F9023E04D
:10DED00040E150E060E070E072C084E08093DB0AD3
:10DEE00082E38093DC0A86E28093DE0A81E08093FD
:10DEF000E10A8093E20A8AE08093E00A41EE51E26F
:10DF000020E030E08091DB0A90E028173907C4F662
:10DF1000FA0185919491A0E0B0E0880F991FAA1FA3
:10DF2000BB1FF901EE0FFF1FEE0FFF1FEE58F54F5D
:10DF300080839183A283B3832F5F3F4F4E5F5F4FF8
:10DF4000E1CF84E08093DB0A80E28093DC0A86E202
:10DF50008093DE0A81E08093E10A8093E20A8BE0FD
:10DF60008093E00A49ED51E220E030E08091DB0A45
:10DF700090E0281739070CF0A3CFFA01859194910E
:10DF8000A0E0B0E0880F991FAA1FBB1FF901EE0F98
:10DF9000FF1FEE0FFF1FEE58F54F80839183A28382
:10DFA000B3832F5F3F4F4E5F5F4FE0CFCE010196AF
:10DFB0000E949F9021E040E154E060E070E0CE01DB
:10DFC00001960E947E9135C084E08093DB0A83E055
:10DFD0008093DC0A86E28093DE0A81E08093E10A86
:10DFE0008093E20A8DE08093E00A41ED51E220E067
:10DFF00030E08091DB0A90E0281739070CF060CF01
:10E00000FA0185919491A0E0B0E0880F991FAA1FB2
:10E01000BB1FF901EE0FFF1FEE0FFF1FEE58F54F6C
:10E0200080839183A283B3832F5F3F4F4E5F5F4F07
:10E03000E0CF0F900F90DF91CF911F910F91FF9044
:10E04000EF90DF90CF90BF90AF909F908F9008950A
:10E050000F931F93CF93DF93EC01462F50E060E0C6
:10E0600070E02AE00E940F568C01CE010E945856A3
:10E07000800F911FDF91CF911F910F910895462F2F
:10E0800050E060E070E02AE00C940F568091E00BC5
:10E0900081118FC00E94F76380911002882321F0C4
:10E0A00080917B13811105C080917A13882309F434
:10E0B00080C010927B1381E0809310020E941E6446
:10E0C000809179138823D1F06AE976E08091771303
:10E0D000909178130E94575780917A13882341F0CA
:10E0E0006AEA76E080917713909178130E945757EF
:10E0F00080917713909178130E94585680917A13EB
:10E10000882369F0609175137091761316161706BF
:10E1100024F48DE69CE00E948B4D10927A1380913E
:10E12000731390917413806290937413809373139C
:10E1300080917213882311F081E001C080E00E9479
:10E14000279E80916B13882359F08091F212909151
:10E15000F312892B29F080918C1181110E94686B38
:10E1600081E080938B110E94086380910E138111CE
:10E170000FC080918A11882359F023E431E644E6E8
:10E1800050E060E070E08DE69CE00E94DA4D02C055
:10E190000E9443610E948A620E9497630E94FD86EA
:10E1A00060938611709387118093881190938911E1
:10E1B000089508952FB7F894882381F080910B116A
:10E1C00090910C1190931A118093191180911B1149
:10E1D00090911C1118161906ACF00FC080910D110A
:10E1E00090910E1190931A118093191180911B1127
:10E1F00090911C11181619062CF480911B11909106
:10E200001C1107C080911B1190911C119195819553
:10E21000910990931C1180931B112FBF0895AF9209
:10E22000BF92CF92DF92EF92FF920F931F93CF9303
:10E23000DF931F921F92CDB7DEB78C017A8369837B
:10E24000CE0101966C01580192E0A90EB11CE12C9F
:10E25000F12CC8010E9425CDF60161916F0186174E
:10E2600031F0C8010E9439CDFFEFEF1AFF0A0F5FAE
:10E270001F4F0A151B0569F781E0EF2809F480E0BC
:10E280000F900F90DF91CF911F910F91FF90EF9022
:10E29000DF90CF90BF90AF900895EF92FF920F93D1
:10E2A0001F93CF93DF931F921F92CDB7DEB78C01E0
:10E2B0007B018AEA8A8341E050E0BE016E5F7F4FB6
:10E2C000C8010E942160D701ED91FC910680F78181
:10E2D000E02DC701199582E8898341E050E0BE0135
:10E2E0006F5F7F4FC8010E9421600F900F90DF91F8
:10E2F000CF911F910F91FF90EF900895CF92DF92F1
:10E30000EF92FF920F931F930E94FD866B017C0199
:10E3100060937D1370937E1380937F13909380138B
:10E320008091F70B0E94665980937C139091F90BB2
:10E33000992329F091E0811190E090937C138091D2
:10E34000010C9091020CA091030CB091040C970168
:10E350008601081B190B2A0B3B0B4091050C5091B1
:10E36000060C6091070C7091080C9091FA0B041741
:10E3700015072607370760F4C092FD0BD092FE0BFD
:10E38000E092FF0BF092000C1092FC0B892F1EC044
:10E390009093FB0B80917C138093FA0BC092FD0B42
:10E3A000D092FE0BE092FF0BF092000C891761F007
:10E3B000C092010CD092020CE092030CF092040C7B
:10E3C00091E09093FC0B02C01092FC0B1F910F91F7
:10E3D000FF90EF90DF90CF9008950F931F93CF930E
:10E3E000DF93EC012AE00E940F568C01CE010E94BF
:10E3F0005856800F911FDF91CF911F910F91089573
:10E40000CF92DF92EF92FF920F931F93CF93DF9300
:10E410006B01770FEE08FF08F7FE1BC0EC016DE201
:10E420000E946E568C0144275527BA014C195D098C
:10E430006E097F092AE0CE010E940F56800F911FBE
:10E44000DF91CF911F910F91FF90EF90DF90CF90D0
:10E4500008952AE0B701A601DF91CF911F910F9196
:10E46000FF90EF90DF90CF900C940F56CF92DF92F9
:10E47000EF92FF920F931F93CF93DF938C016B0169
:10E48000770FEE08FF08F7FE12C06DE20E946E568D
:10E49000EC0144275527BA014C195D096E097F0923
:10E4A0002AE0C8010E940F56C80FD91F06C02AE0F3
:10E4B000B701A6010E940F56EC01C8010E945856F0
:10E4C0008C0F9D1FDF91CF911F910F91FF90EF90C7
:10E4D000DF90CF9008950F931F93CF93DF931F92F8
:10E4E000CDB7DEB78C0169830E9425CD698186177F
:10E4F00029F0C8010E9439CD81E001C080E00F9071
:10E50000DF91CF911F910F910895CF930E9406AA9A
:10E5100084E090E09093F40B8093F30B1092A110A1
:10E520001092AB101092B5101092BF10EDE4F0E114
:10E53000DF011C92179680E1A13AB807D1F78EE867
:10E5400091E19093AA108093A9101092A410809149
:10E55000F20B90918E11891718F091E09093A11011
:10E5600027E931E13093B4102093B3101092AE102C
:10E5700090919711891718F091E09093AB1020EAD1
:10E5800031E13093BE102093BD101092B8109091DD
:10E59000A011891718F091E09093B51029EA31E1A4
:10E5A0003093C8102093C7101092C2109091A911F7
:10E5B000891718F091E09093BF101092F10B20E0B2
:10E5C00030E0D901AC5CBD4E4D915C914150510998
:10E5D0004432510520F491E09093F10B05C02D5F7A
:10E5E0003F4F2837310569F79091F10B992341F19D
:10E5F0002091A1113091A2112D5D3F4F3093A211B6
:10E600002093A1112091A3113091A411235231091B
:10E610003093A4112093A3112091AA113091AB1132
:10E620002D5D3F4F3093AB112093AA112091AC1177
:10E630003091AD11235231093093AD112093AC11BB
:10E640009091AD129F3049F49091AE129F3029F411
:10E6500010924C1010924B1008C020910C13309166
:10E660000D1330934C1020934B1022E130E0309387
:10E670004910209348102091F30B3091F40BA2EB3A
:10E68000B1E141E0B683A5839C91992329F08917D4
:10E6900018F040832F5F3F4F1A96379690E1E13A8A
:10E6A000F90781F73093F40B2093F30B21313105F7
:10E6B00034F080E190E09093F40B8093F30B0E9490
:10E6C000B45285EA90E19093AB0F8093AA0F8091AA
:10E6D000A9109091AA109093A90F8093A80F82EA95
:10E6E00090E19093AD0F8093AC0F83EA90E190930B
:10E6F000AF0F8093AE0F81EA90E19093B10F8093BA
:10E70000B00F8FEA90E19093B50F8093B40F809192
:10E71000B3109091B4109093B30F8093B20F8CEA22
:10E7200090E19093B70F8093B60F8DEA90E19093AC
:10E73000B90F8093B80F8BEA90E19093BB0F809351
:10E74000BA0F89EB90E19093BF0F8093BE0F809139
:10E75000BD109091BE109093BD0F8093BC0F86EBBF
:10E7600090E19093C10F8093C00F87EB90E190935D
:10E77000C30F8093C20F85EB90E19093C50F8093F8
:10E78000C40F83EC90E19093C90F8093C80F8091E0
:10E79000C7109091C8109093C70F8093C60F80EC5C
:10E7A00090E19093CB0F8093CA0F81EC90E190930E
:10E7B000CD0F8093CC0F8FEB90E19093CF0F809390
:10E7C000CE0F2091F30B3091F40B2450310960E00F
:10E7D0007AE0C7E0462F50E04217530724F5CA01FC
:10E7E0000496789FF001799FF00D1124E855F04FC1
:10E7F000C49FC001C59F900D1124AC01415B5F4EC9
:10E8000053834283DC01A35BBF4E15964D915C910F
:10E81000169751834083825B9F4E95838483B18793
:10E82000A0876F5FD7CF81E08093F50BCF910895DC
:10E830000F931F93CF93DF93FC0124813581211522
:10E84000310519F4FB01108211C0EA0121972C1740
:10E850003D0708F4E9018B01FC0160817181AE0183
:10E86000C8010E94DED1C00FD11F1882DF91CF9165
:10E870001F910F9108954115510529F061157105FA
:10E8800011F00C9418740895EF92FF920F931F9358
:10E89000CF93DF931F921F92CDB7DEB78C018CE729
:10E8A00089831A82F801E480F580FFEFEF1AFF0AEE
:10E8B000B701C8010E94D454882381F0F801208157
:10E8C000318184819581BE016F5F7F4F820F931FDD
:10E8D0000E94D7D1F801F582E48281E00F900F9079
:10E8E000DF91CF911F910F91FF90EF900895AF921C
:10E8F000BF92CF92DF92EF92FF920F931F93CF932D
:10E90000DF9300D01F92CDB7DEB78C0149835A83C5
:10E910006B837C83CE0101966C01580194E0A90EB3
:10E92000B11CE12CF12CC8010E9425CDF6016191AA
:10E930006F01861731F0C8010E9439CDFFEFEF1A41
:10E94000FF0A0F5F1F4F0A151B0569F781E0EF28CB
:10E9500009F480E00F900F900F900F90DF91CF910E
:10E960001F910F91FF90EF90DF90CF90BF90AF90ED
:10E970000895CF92DF92EF92FF920F931F93CF9360
:10E98000DF93EC010091990FE0E0F0E020E030E04F
:10E99000A90110E0CE17DF071CF1309711F40D32FA
:10E9A000E1F0DF01A756B04FFC9080ED8F0D8A306B
:10E9B000A8F4AAE0B0E00E9466CD2F2DFF0C330B27
:10E9C000205331096901330FEE08FF089B01AC01A8
:10E9D0002C0D3D1D4E1D5F1D01C011E03196DACF9B
:10E9E000CA01B901112339F0909580957095619510
:10E9F0007F4F8F4F9F4FDF91CF911F910F91FF90CE
:10EA0000EF90DF90CF9008958091FA0B811105C0AF
:10EA100081E09091FC0B911101C080E00895089570
:10EA20000895089508950895623039F0633041F0F3
:10EA3000613041F440935314089540935214089563
:10EA4000409351140895623069F06330A1F0613051
:10EA5000D1F450935B1440935A1430935D14209377
:10EA60005C140895509362144093611430936414BD
:10EA700020936314089550936B1440936A14309359
:10EA80006D1420936C140895FC01858108950895F8
:10EA900008950895089520916F14211102C0FC017A
:10EAA0006283089520916F14211102C0FC016483D8
:10EAB000089520916F14211102C0FC016383089511
:10EAC0000895089580916F14811102C00C945D9790
:10EAD0000895089580E0089508950895089508958B
:10EAE0000895089580916F14811104C08FE090E023
:10EAF0000C947698089520916F14211108C0FC01A0
:10EB00008481882321F082E090E00C947698089527
:10EB100020916F14211108C0FC018381882321F00A
:10EB200081E090E00C947698089580916F148111A3
:10EB300004C08BE090E00C947698089580916F1457
:10EB4000811105C060E080E190E00C94D6980895B2
:10EB500080916F14811105C060E08FE090E00C940B
:10EB6000D698089580916F14811127C06330A1F069
:10EB700028F4613049F0623059F008956530A1F011
:10EB800078F06630A9F0089560E089E090E013C065
:10EB900060E08AE090E00FC060E08BE090E00BC0A6
:10EBA00060E08CE090E007C060E08DE090E003C0A2
:10EBB00060E08EE090E00C94D698089580916F14F8
:10EBC000811127C06330A1F028F4613049F0623030
:10EBD00059F008956530A1F078F06630A9F00895F5
:10EBE00061E089E090E013C061E08AE090E00FC04E
:10EBF00061E08BE090E00BC061E08CE090E007C04A
:10EC000061E08DE090E003C061E08EE090E00C9464
:10EC1000D698089520916F14211109C0FC018281BA
:10EC2000882329F061E088E090E00C94D69808955C
:10EC300020916F14211109C0FC018481882329F0DF
:10EC400061E082E090E00C94D698089520916F14D2
:10EC5000211109C0FC018381882329F061E081E052
:10EC600090E00C94D698089580916F14811105C09E
:10EC700061E086E090E00C94D698089580916F143E
:10EC8000811105C060E08BE090E00C94D698089567
:10EC900080916F14811105C061E087E090E00C94D1
:10ECA000D698089580916F14811105C061E085E0C8
:10ECB00090E00C94D698089580916F14811105C04E
:10ECC00061E08AE090E00C94D6980895CF93DF93AA
:10ECD000FC0125812223A1F1EC0180916F148111A7
:10ECE0002EC06091581470915914809168149091BD
:10ECF00069140E948B4D10925E1480916F148111E3
:10ED00000CC060915F1470916014809168149091B0
:10ED100069140E948B4D1092651480916F148111BB
:10ED20000CC0609166147091671480916814909182
:10ED300069140E948B4D10926E14109250141D8213
:10ED4000DF91CF910895CF93DF93FC0125812111AD
:10ED50003DC0EC0180916F14811136C08091501438
:10ED6000811132C080915314882349F080915E1440
:10ED7000811105C081E080935E140E94E499809126
:10ED80005214882369F080916F14811109C0809119
:10ED90006514811105C081E0809365140E94A299D9
:10EDA00080915114882369F080916F14811109C0FA
:10EDB00080916E14811105C081E080936E140E94D1
:10EDC000609981E08093501481E08D83DF91CF9131
:10EDD0000895862F90916F14911102C00C94B598EC
:10EDE0000895CF93C1E080916F14811103C08C2FDF
:10EDF0000E94B598CF5FC730B1F7CF910895809149
:10EE00006F14882329F06CED75E081E00C94FE4EC0
:10EE100084E090E00C94769880916F14882329F018
:10EE200068EE73E081E00C94FE4E60E084E090E0D8
:10EE30000C94D6986CED75E080E00C94FE4E24EFB7
:10EE400031E0DB010E94A1CF2FEF30E040E050E045
:10EE50000E9447CDCA01B90164527A4F8F4F9F4F2C
:10EE600080E00C94FE4E80916F14882339F060EDA1
:10EE700077E081E00E94FE4E0C94269A61E083E0E8
:10EE800090E00C94D69880916F1481111BC08091F2
:10EE900057148823B9F068EE73E081E00E94FE4EBB
:10EEA000109257142DE537E948E95AE360E070E025
:10EEB00080916814909169140E94DA4D90935614D1
:10EEC00080935514089520916F14211109C0209149
:10EED0005414222329F002960E94399A1092541455
:10EEE000089520916F14222389F06FE676E080E088
:10EEF0000E94FE4E24E637E942E350E060E070E015
:10EF000080916814909169140C94DA4D20915414F6
:10EF1000211106C002960E94399A81E08093541410
:10EF2000089580E00E94254F81E00E94254F809146
:10EF30006F14811103C082E00E94254F6CED75E0D3
:10EF400080E00E94FE4E6CED75E081E00E94FE4E76
:10EF500080916F1481110DC08CE996ECA1E0BB2764
:10EF6000ABBFFC016791769182E00E94FE4E0C944B
:10EF700046970895FC0184859585978386838685C9
:10EF80009785918780878089918993878287808DF3
:10EF9000918D938B828B828D938D958B848B848DB9
:10EFA000958D978B868B0895FC0180899189938735
:10EFB00082878289938995878487848995899787B1
:10EFC0008687089526E00C9401592F923F924F9224
:10EFD0005F926F927F928F929F92AF92BF92CF92E9
:10EFE000DF92EF92FF920F931F93CF93DF9300D0A6
:10EFF0001F92CDB7DEB75C010E94DE620E941F6ADD
:10F000000E945B6A80917713909178130E94585602
:10F010000E941E9724E0A216B10409F49CC00CF0D3
:10F020004FC0A3E0AA16B10409F03CC18CE190E006
:10F030000E94A8CF9C838B8383E696E0AB81BC8142
:10F0400011969C938E931396BC92AE92129781E088
:10F050009FEF15969C938E9314978FEF90E01796E1
:10F060009C938E93169719961C921E9218975896F9
:10F070001C925897CD010E949C5087E596E0EB8149
:10F08000FC8191838083E0918214F0918314D08C71
:10F0900000910D1110910E1116950795E0900B112E
:10F0A000F0900C11F694E7946AE673E2809177137E
:10F0B000909178130E947D57812C9924939412C1CA
:10F0C000B5E0AB16B10409F4A6C0E6E0AE16B10493
:10F0D00009F0E8C08CE190E00E94A8CF9C838B836C
:10F0E00083E696E0AB81BC8111969C938E93139638
:10F0F000BC92AE92129781E09FEF15969C938E93EF
:10F1000014978FEF90E017969C938E93169719960D
:10F110001C921E92189758961C925897CD010E94E7
:10F120009C5087E596E0EB81FC8191838083E091A0
:10F130009B07F0919C07D08C00914C1110914D11C0
:10F1400016950795E0904A11F0904B11F694E794CC
:10F150006DE973E2A0C08CE190E00E94A8CF9C838F
:10F160008B8383E696E0AB81BC8111969C938E9352
:10F170001396BC92AE92129781E09FEF15969C93E6
:10F180008E9314978FEF90E017969C938E9316971B
:10F1900019961C921E92189758961C925897CD015A
:10F1A0000E949C5087E596E0EB81FC8191838083EF
:10F1B000009122111091231116950795E0902011CE
:10F1C000F0902111F694E7948091AE128C50823029
:10F1D00040F4E091AC07F091AD07D08C6DED73E297
:10F1E0005AC08091F712823009F07AC08091AC1237
:10F1F0008C3009F075C0E0919B07F0919C07D08C92
:10F200006DEB73E280917713909178130E947D5794
:10F210008824839466C08CE190E00E94A8CF9C83F0
:10F220008B8383E696E0AB81BC8111969C938E9391
:10F230001396BC92AE92129781E09FEF15969C9325
:10F240008E9314978FEF90E017969C938E9316975A
:10F2500019961C921E92189758961C925897CD0199
:10F260000E949C5087E596E0EB81FC81918380832E
:10F27000E091A807F091A907D08C00913711109167
:10F28000381116950795E0903511F0903611F694E7
:10F29000E7946DE773E280917713909178130E9461
:10F2A0007D571EC061E573E28091771390917813CA
:10F2B0000F900F900F900F90DF91CF911F910F91B2
:10F2C000FF90EF90DF90CF90BF90AF909F908F9086
:10F2D0007F906F905F904F903F902F900C947D5750
:10F2E000812C912C0E941E9764E473E28091771325
:10F2F000909178130E947D5768E373E280917713B1
:10F30000909178130E945957B8018091771390918A
:10F3100078130E9436726CE273E2809177139091B9
:10F3200078130E945957B701809177139091781301
:10F330000E94367260E273E28091771390917813A5
:10F340000E9459578D2D0E94F496809177139091C9
:10F3500078130E945856AB81BC81ED91FC911197B6
:10F360000280F381E02DCD011995CA2C8A2D0E94CF
:10F37000B74F8D3D9540A8F464E378E08A2D0E9454
:10F38000AD4FEB81FC81F78AE68AB70182810E944A
:10F39000C74F6CED75E08A2D0E94B24FDD20C1F0A1
:10F3A0001AC064E873E08A2D0E94B24FAB81BC8121
:10F3B00057961C930E935697B80112968C910E9403
:10F3C000C74F6CED75E08A2D0E94AD4FDD2019F01E
:10F3D0003324339401C0312C21E02983212C2A834A
:10F3E0000E94D05A8091B610882359F1AB81BC811C
:10F3F000ED91FC9111976091BB107091BC10019040
:10F40000F081E02DCD0119958C2D0E94B74F8D3DD7
:10F41000B5E09B075CF48438E3E09E0784F08C0140
:10F420008D3D954074F00CED15E00BC07C018533EB
:10F4300098403CF064E3E62E68E0F62E02C004E853
:10F4400013E02A8121111FC08091AC108823C9F1DB
:10F45000E091B310F091B410858196814091AF1086
:10F460005091B0109C0121533109421753074CF1C0
:10F47000C196841795072CF10E94FD8664157505C9
:10F4800086059705F0F08091AC108823C1F040917B
:10F49000AF105091B010E091B310F091B41085818D
:10F4A00096819C01285C3109421753072CF0885340
:10F4B0009F4F841795071CF481E0382605C021E092
:10F4C0002A83222009F47CC0332009F445C0DD20C2
:10F4D000F9F064E873E08C2D0E94B24F992009F492
:10F4E00058C06091C8127091C91241E08C2D0E94E1
:10F4F0006C4F0E9409A6AB81BC8112968C910E9430
:10F50000B74F08171907ACF38C2D0E943E4F41C02E
:10F5100064E378E08C2D0E94AD4F9920B1F06091AA
:10F52000C8127091C91240E08C2D0E946C4F0E944D
:10F5300009A6AB81BC8112968C910E94B74F8E15A3
:10F540009F05ACF38C2D0E943E4FEB81FC81F78A26
:10F55000E68AB701828110C0DD20B1F064E378E073
:10F560008C2D0E94AD4FAB81BC815796FC92EE92E0
:10F570005697B70112968C910E94C74F6CED75E0BB
:10F580008C2D0E94B24F12C064E873E08C2D0E9453
:10F59000B24FEB81FC81178B068BB80182810E94F0
:10F5A000C74F6CED75E08C2D0E94AD4F0E94FD861B
:10F5B0002B013C01F8EC4F0E511C611C711C1A828E
:10F5C00029812223D9F18091A2108823A9F14091A9
:10F5D000A5105091A610E091A910F091AA10858174
:10F5E00096819C01285C3109421753072CF08853FF
:10F5F0009F4F8417950704F581E0D82680917713F3
:10F6000090917813DD2039F061E173E20E947D571B
:10F6100082E090E006C06FEF72E20E947D5781E0C9
:10F6200090E00E94276A0E94FD86AB81BC815896BB
:10F63000DC922224239403C0212C1EC0212C809113
:10F64000A210882309F48AC2E091A910F091AA10AF
:10F65000858196814091A5105091A6109C0121535F
:10F660003109421753070CF479C2C19621E029836E
:10F67000841795070CF472C20E94B0520E947E71EA
:10F680008DE69CE00E94EC4D8091FA0B882309F4F2
:10F69000A7CE8091FC0B882309F4A2CE0E947E7134
:10F6A0000E9404758823D1F384E0A816B104D9F12F
:10F6B00034F4B3E0AB16B10409F438C1C4C1E5E0D9
:10F6C000AE16B10409F4CDC0F6E0AF16B10409F0EE
:10F6D000BAC11093BC120093BB12F092BE12E0921A
:10F6E000BD12D092BF12B8018EE291E00E940F715C
:10F6F000B70180E391E00E940F716D2D82E391E0EC
:10F700000E946B72B80186E00E94E34EB70186E06A
:10F710000E94C84EE0919B07F0919C07D08E6CED43
:10F7200075E086E091C08820C1F01093BC12009370
:10F73000BB12F092BE12E092BD12D092BF12B8017D
:10F740008EE291E00E940F71B70180E391E00E9488
:10F750000F716D2D82E391E017C01093B0120093EA
:10F76000AF12F092B212E092B112D092B312B8017D
:10F7700082E291E00E940F71B70184E291E00E9461
:10F780000F716D2D86E291E00E946B72B80184E0EA
:10F790000E94E34EB70184E00E94C84E882049F0E1
:10F7A000E0919B07F0919C07D08E6CED75E084E0B2
:10F7B0004BC0E091AC07F091AD07D08E8091AE12B6
:10F7C0008D3029F4E0918213F0918313D08E6CED8B
:10F7D00075E084E00E94C74F66E970E080E090E049
:10F7E0000E94C3868091AE128D3011F584E00E9494
:10F7F000B74FA091AC07B091AD078D3D95404CF04F
:10F80000ED91FC9111970190F081E02D6FEF7FEF6A
:10F8100008C0ED91FC9111970190F081E02D61E01D
:10F8200070E0CD0119958091AC079091AD076FC044
:10F830008091AC079091AD07DC01ED91FC910480C3
:10F84000F581E02D1995FFC00E94C74F66E970E071
:10F8500080E090E00E94C38680919B0790919C0776
:10F86000EBCF1093B7120093B612F092B912E09258
:10F87000B812D092BA12B80189E291E00E940F71D9
:10F88000B7018BE291E00E940F716D2D8DE291E046
:10F890000E946B72B80185E00E94E34EB70185E0DB
:10F8A0000E94C84EE091A807F091A907D08E6CED98
:10F8B00075E085E00E94C74F66E970E080E090E067
:10F8C0000E94C3868091AD128D3059F585E00E946B
:10F8D000B74FA091A807B091A9078D3D95404CF076
:10F8E000ED91FC9111970190F081E02D6FEF7FEF8A
:10F8F00008C0ED91FC9111970190F081E02D61E03D
:10F9000070E0CD0119958091A8079091A907DC01BD
:10F91000ED91FC910190F081E02D60E070E019958F
:10F9200092C08091A8079091A90786CF1093CB121F
:10F930000093CA12F092CD12E092CC12D092C4126F
:10F94000B8018DE391E00E940F71B7018FE391E060
:10F950000E940F716D2D87E391E00E946B72B801D8
:10F9600083E00E94E34EB70183E00E94C84E80917D
:10F97000C412E0918214F0918314808F8091C4129C
:10F980000E94DA7083E00E94B74F2091C4122223B4
:10F9900069F1B9E0BC1538F020910D1130910E11CC
:10F9A0003695279502C02EEE32E08217930709F4B0
:10F9B0004AC06091C8127091C91241E083E00E9470
:10F9C0006C4F0E9409A6EB81FC8182810E94B74F97
:10F9D00008171907B4F383E00E943E4FAB81BC8146
:10F9E00057961C930E935697B80129C0A9E0AC1501
:10F9F00008F4B6C020910B1130910C113695279563
:10FA00008217930701F16091C8127091C91240E00A
:10FA100083E00E946C4F0E9409A6EB81FC818281E9
:10FA20000E94B74F8E159F05B4F383E00E943E4FAE
:10FA3000AB81BC815796FC92EE925697B701129615
:10FA40008C910E94C74F80917713909178130E94F8
:10FA500058560E941E97B4E0AB16B10499F03CF4DE
:10FA6000F3E0AF16B10449F563E872E220C025E087
:10FA7000A216B104D1F086E0A816B104F1F463EB4C
:10FA800072E215C08091AE128C50823018F465EE8F
:10FA900072E20DC08091F712823079F48091AC123D
:10FAA0008C3059F46CEC72E202C06AE972E2809127
:10FAB0007713909178130E947D570E941E9768E7F4
:10FAC00072E280917713909178130E947D576CE6D3
:10FAD00072E280917713909178130E945957B80180
:10FAE00080917713909178130E94367260E672E2EB
:10FAF00080917713909178130E945957B7018091A4
:10FB00007713909178130E94367264E572E28091C7
:10FB10007713909178130E9459578D2D0E94F49677
:10FB200080917713909178130E9458560F900F9000
:10FB30000F900F90DF91CF911F910F91FF90EF9059
:10FB4000DF90CF90BF90AF909F908F907F906F90FD
:10FB50005F904F903F902F900C94576A19828CCDF4
:10FB60002AEC38E04DCFCF93DF93CDB7DEB728979F
:10FB70000FB6F894DEBF0FBECDBF809181138823EE
:10FB8000E1F1109281130E94D56A81E08093030213
:10FB90008091AE07882389F165E472E28091771342
:10FBA000909178130E945957E091F60BE4300CF0D5
:10FBB000E0E08EE191E19A8389838AE191E19C837F
:10FBC0008B8385E191E19E838D8380E191E198872C
:10FBD0008F83EE0FFF0BEC0FFD1F6181728180910F
:10FBE00077139091781328960FB6F894DEBF0FBE66
:10FBF000CDBFDF91CF910C947D5728960FB6F89426
:10FC0000DEBF0FBECDBFDF91CF9108950895089557
:10FC1000FC01828193818830910529F410922B0197
:10FC200010922A010895099721F410922901109247
:10FC300028010895FC01178A168A6CED75E082810F
:10FC40000C94C74FCF93DF93EC011F8A1E8A8A81E1
:10FC50000E943E4F8B8D882331F08A810E94B74FDE
:10FC60009A8F898F1B8EDF91CF910895DF92EF924B
:10FC7000FF920F931F93CF93DF93EC018A8189301A
:10FC800010F40E94254FDD8C6B8D7C8D098D1A8DB3
:10FC9000EA80FB8089E08E1508F466C00F301105FC
:10FCA00038F001369DE6190728F000E61DE602C08F
:10FCB0000FE010E06F30710538F061368DE678079F
:10FCC00028F060E67DE602C06FE070E080E090E042
:10FCD0000E94F6CB20E030E04AE754E40E9417CEC1
:10FCE00020E030E04CE852E40E9457CC9B01AC018C
:10FCF00060E070E08AEF94E40E9417CE0E9489CE03
:10FD0000FF2425E12E9DF0012F9DF00D1124E753D6
:10FD1000FF4EDD2071F023813481AB0177FF04C0F9
:10FD200044275527461B570B88279927841B950B7B
:10FD30000AC025813681AB0177FF04C044275527CF
:10FD4000461B570BCA014FB7F89455E15E9DF00171
:10FD50005F9DF00D1124E753FF4E108B0787328B08
:10FD6000218B948B838B4FBF9D8D6B8D7C8D8A8176
:10FD70009923F9F08A3058F495E1899FF001112414
:10FD8000E753FF4E058116811695079502C00EEECA
:10FD900012E041E00E946C4F61E070E080E090E092
:10FDA0000E94C3868A810E94B74F08171907A0F3E3
:10FDB0001EC08A3058F495E1899FF0011124E75361
:10FDC000FF4E038114811695079502C00AEC18E0D6
:10FDD00040E00E946C4F61E070E080E090E00E94A3
:10FDE000C3868A810E94B74F80179107A0F38A814A
:10FDF0000E943E4FB8018A81DF91CF911F910F91F0
:10FE0000FF90EF90DF900C94C74FCF93DF93EC01FE
:10FE10008A81893010F40E94254F48EE53E05B87B9
:10FE20004A8720ED37E03D872C878CED95E09F8752
:10FE30008E87598B488B3B8B2A8B9D8B8C8BDF91CC
:10FE4000CF910895CF93DF93EC017F8B6E8B8885E4
:10FE500099856817790769F48A810E943E4F8B8DD6
:10FE6000882329F18A810E94B74F9A8F898F1B8E30
:10FE70001EC0CE010E94688FEA81EA30B0F49C0176
:10FE8000C39714F022E330E02E3C8FEF380714F4D0
:10FE90002EEC3FEF8FB7F89495E1E99FF001112424
:10FEA000E753FF4E318720878FBF81E08B8FDF9133
:10FEB000CF9108950F931F93CF93DF938C01FC0193
:10FEC000778B668B0E94688FEC01F80182819381A9
:10FED00088309105D1F4D7FF06C060E08AE00E9427
:10FEE0008F5961E005C061E08AE00E948F5960E0AF
:10FEF00086E00E948F59D7FF03C0D195C195D109E3
:10FF0000D0932B01C0932A011BC00997C9F4D7FFD6
:10FF100006C060E08DE00E948F5961E005C061E09D
:10FF20008DE00E948F5960E08BE00E948F59D7FFCF
:10FF300003C0D195C195D109D0932901C09328015F
:10FF4000DF91CF911F910F910895CF93DF93EC0133
:10FF50008A81893010F40E94254F2EEC3FEF3B87B9
:10FF60002A8782E390E09D878C871F861E86398BC7
:10FF7000288B9B8B8A8B1D8A1C8A6EEE72E08A818D
:10FF80000E94B24F6AEC78E08A810E94AD4F8CEDFE
:10FF900095E09A8F898F1B8EDF91CF910895CF9333
:10FFA000DF93EC0121E03FEF3B872A878FEF90E062
:10FFB0009D878C871F861E86398B288B9B8B8A8B0F
:10FFC0001D8A1C8A61E08AE00E94BF5961E086E0D8
:10FFD0000E94BF5961E08DE20E94BF5961E08DE04F
:10FFE0000E94BF5961E08BE00E94BF5961E08EE240
:10FFF0000E94BF598A819B818830910529F4109213
:020000021000EC
:100000002B0110922A0106C0099721F410922901B0
:1000100010922801DF91CF9108950F931F93CF93F2
:10002000DF938C01FC01178A168AEC01699640E087
:1000300068E0CE010E9428614FE766E0CE010E9491
:10004000286140E06CE0CE010E9428614FE767E044
:10005000CE010E9428610E94FD86F801648F758F91
:10006000868F978FDF91CF911F910F910895EF9217
:10007000FF920F931F93CF93DF938C01FC01778B3B
:10008000668B0E94688FEC01F80182819381883031
:10009000910531F57801F9E1EF0EF11CD7FF06C0AB
:1000A0006AE0C1388FEFD80754F001C068E02C2F08
:1000B0009D2FC038D1052CF02FE790E002C021E839
:1000C0009FEF422F592F57FF03C05195419551097A
:1000D000C7010E942861CD2B69F54FE766E027C074
:1000E000099741F57801E9E1EE0EF11CD7FF06C052
:1000F0006EE0C138FFEFDF0754F001C06CE02C2F39
:100100009D2FC038D1052CF02FE790E002C021E8E8
:100110009FEF422F592F57FF03C051954195510929
:10012000C7010E942861CD2B29F44FE767E0C70182
:100130000E9428610E94FD86F801648F758F868F6A
:10014000978FDF91CF911F910F91FF90EF900895BE
:100150000F931F93CF93DF93EC010E94FD860C8DCC
:100160001D8D2E8D3F8DDC01CB01801B910BA20BD1
:10017000B30B853F9140A105B10548F06E897F8999
:10018000CE01DF91CF911F910F910C943780DF91B9
:10019000CF911F910F910895CF93DF93EC01809140
:1001A0008513811109C06A8D7B8DCE0149960E940D
:1001B0004D7181E08093851321E83FEF3B872A87CB
:1001C0008FE790E09D878C871F861E86398B288B52
:1001D0009B8B8A8B1D8A1C8ADF91CF9108950F9388
:1001E0001F93CF93DF93EC010E94FD860C8D1D8D34
:1001F0002E8D3F8DDC01CB01801B910BA20BB30B2D
:10020000853F9140A105B10548F06E897F89CE01F7
:10021000DF91CF911F910F910C94E18FDF91CF91DE
:100220001F910F9108956F927F928F929F92AF923C
:10023000BF92CF92DF92EF92FF920F931F93CF93D3
:10024000DF938091A4149091A514DC01ED91FC91B1
:100250000084F185E02D1995B12C181619060CF0C3
:10026000D1C0AA24A3948091A4149091A514DC0178
:10027000ED91FC910084F185E02D1995892B09F40D
:10028000C1C0C091E71381E08C0F8093E713809188
:10029000A4149091A514DC01ED91FC910284F385E6
:1002A000E02D1995EC2FF0E0E955FC4E80838A3063
:1002B000D1F6E090E713F12C1092BA0E1092B90E1D
:1002C0001092B50E1092B60E1092B70E1092B80E94
:1002D0001092B40E1092B30E1092B20E87EAC82E8E
:1002E00083E1D82E00E010E0D0E0C0E00E151F053D
:1002F0000CF06CC0F60191916F019D3009F463C060
:100300009C3789F19A3009F052C0D33009F059C0B6
:10031000CC2309F456C06C2E712CC30101970E94A6
:10032000B9747093BA0E6093B90E0E94FD86609303
:10033000A7147093A8148093A9149093AA14809181
:100340008413882309F45BC08090B90E9090BA0E94
:10035000B8016619770987EA93E10E948CA888168C
:10036000990679F54CC08C2F90E0FC01E756F04FD0
:100370001082D13099F068F0D230B1F40E94B97493
:100380006093B50E7093B60E8093B70E9093B80E2F
:100390000BC00E94B9746093B20E06C00E94B9747B
:1003A0007093B40E6093B30EDF5FC0E00CC00F33E8
:1003B00011053CF4EC2FF0E0E756F04F9083CF5F4F
:1003C00002C01092A6130F5F1F4F90CF8091A6130B
:1003D00081110EC08091AF0E9091B00E0196909356
:1003E000B00E8093AF0E60E087E80E9423A902C0A0
:1003F000BB24B3941092A7131092E71334CFA092AA
:10040000A613E1CF8B2DDF91CF911F910F91FF901C
:10041000EF90DF90CF90BF90AF909F908F907F90A4
:100420006F900895CF931092B10E1092AE0E10926D
:10043000B00E1092AF0E61E089E30E948F590E94C6
:100440002EA88091A4149091A514DC01ED91FC914B
:100450000084F185E02D1995892B61F08091A41419
:100460009091A514DC01ED91FC910284F385E02DBF
:100470001995E7CF0E94A0A98091A4149091A5148A
:10048000DC01ED91FC910680F781E02D1995109229
:10049000A6140E94FD866093A7147093A8148093FD
:1004A000A9149093AA14C1E00E94138181110E94A3
:1004B000883C0E946EA80E94B0528091AF0E90912D
:1004C000B00E0A9724F48091A614882331F060E0DE
:1004D0008AE80E9423A9C093B10E8091B10E8823AF
:1004E00019F38091AE0E882341F045EE51E060E0B3
:1004F00070E08DE891E10E9415CD60E089E30E94F3
:100500008F5960E08AE3CF910C948F59EF92FF925C
:100510000F931F93CF93DF9300D000D0CDB7DEB7FA
:1005200067EC76E0CE0101960E94D6550D811E81C2
:10053000F02EEE24E3948091A4149091A514DC0194
:10054000ED91FC910084F185E02D1995892B21F125
:100550008091A4149091A514DC01ED91FC9102848A
:10056000F385E02D19958F3439F4E092A51380932B
:100570009613E0929513DFCF9091A5139923D9F2AA
:10058000E091951391E09E0F90939513F0E0EA5659
:10059000FC4E80839F1578F2809195138F1510F48F
:1005A000F12C21C04FE050E066E873E1CE010196E6
:1005B0000E941874A6E9B3E1E7ECF6E0FF24F39497
:1005C0001127CF01875C96408017910734F49D91E5
:1005D00081919817B1F3F12CF4CF109296131092E9
:1005E000A51310929513CE0101960E9478558F2D78
:1005F00026960FB6F894DEBF0FBECDBFDF91CF9128
:100600001F910F91FF90EF900895DC01ED91FC9107
:100610000190F081E02D1994CF93DF93EC017F8B53
:100620006E8B0E94688FBC018A81DF91CF910C9400
:10063000C74F80911102882311F0599801C0599A2F
:100640009091110281E08927809311020895109200
:100650008A111092230710921A0710922407109201
:100660002507109226071092270781E08093DE0B62
:1006700040912E0750912F0760E070E026E433E8A8
:1006800080911B0790911C070C94DA4D8091E10B2F
:10069000882361F18091DF0A81111CC01092210B27
:1006A0001092220B1092230B1092240B1092250B08
:1006B0001092260B1092290B8091DC0B9091DD0B90
:1006C000DC01ED91FC910190F081E02D19951092E3
:1006D000DE0B089526E433E845E050E060E070E08A
:1006E00080911B0790911C070C94DA4D089560913E
:1006F000F5137091F61380911B0790911C070E94CF
:10070000734D882319F081E08093F413089560E01D
:1007100087E00E948F591092DF0B089561E087E017
:100720000E948F5981E08093DF0B0895CF93DF9370
:1007300080910214811110C084EF91E09093011414
:10074000809300148BE290E09093FF138093FE134C
:1007500081E08093021420C08091FE139091FF13DA
:100760008532910514F0049709C08331910514F086
:10077000029704C0823091052CF001979093FF13EB
:100780008093FE138091FE139091FF1397FF04C096
:100790001092FF131092FE13C091FD13CC2319F099
:1007A0000E94878302C00E948E8381E08C27809301
:1007B000FD13C0910014D09101141C161D065CF0AD
:1007C000109202140E94878329E034E84AEF50E037
:1007D00060E070E007C026E933E8AE010D2E000CA2
:1007E000660B770B80911B0790911C070E94DA4DD6
:1007F0009093FC138093FB138091FE139091FF1351
:10080000C81BD90BD0930114C0930014DF91CF9172
:1008100008950F931F93CF93DF938091E00B88236C
:1008200031F0DF91CF911F910F910C94968300913D
:10083000FB131091FC13C0911B07D0911C07B8014A
:10084000CE010E94734D882321F0B801CE010E9491
:100850008B4DDF91CF911F910F910C948783CF9295
:10086000DF92EF92FF921092E00B20911F073091E0
:100870002007409121075091220760912407709131
:10088000250780912607909127070E94AACD6B012A
:100890007C0120E030E0A9010E94F1CB87FD09C076
:1008A000C0922407D0922507E0922607F0922707EE
:1008B00008C0109224071092250710922607109264
:1008C0002707FF90EF90DF90CF900C940984EF9270
:1008D000FF921F93CF93DF9300D0CDB7DEB784E6AE
:1008E00089838CE38A8388E28B831091F71313301A
:1008F000F8F4E12EF12C10FF03C00E94878302C0A0
:100900000E948E83E1E0F0E0EC0FFD1FEE0DFF1D75
:10091000408150E060E070E027E634E880911B07FA
:1009200090911C070E94DA4D1F5F1093F71304C0CB
:100930000E9487831092F7130F900F900F90DF9112
:10094000CF911F91FF90EF9008958091DF0B882346
:1009500019F00E94878302C00E948E839091DF0B62
:1009600081E089278093DF0B08950F931F93CF9326
:10097000DF939091FA1380918A1191112BC08823F3
:1009800009F451C00091F8131091F913C0911B079D
:10099000D0911C07B801CE010E94734D882321F02D
:1009A000B801CE010E948B4D0E948E8325EB34E866
:1009B00042EC51E060E070E080911B0790911C07D1
:1009C0000E94E34D9093F9138093F81381E0809394
:1009D000FA1355C0882331F0DF91CF911F910F9109
:1009E0000C94A5848091DF0B8823B1F36091F813F8
:1009F0007091F91380911B0790911C070E948B4DF9
:100A000025EB34E844E150E060E070E080911B07A2
:100A100090911C070E94E34D9093F9138093F81373
:100A20001092FA132CC0C0911202D0911302229797
:100A3000D0931302C09312021C161D0674F4BE015B
:100A4000772787E00E94FB59CC2321F081E0809337
:100A5000DF0B15C01092DF0B12C06091F81370917C
:100A6000F91380911B0790911C070E948B4D0E94E7
:100A700087838FEF90E09093130280931202DF91AF
:100A8000CF911F910F9108950F931F93CF93DF93F1
:100A90000091F0131091F113C091F213D091F31360
:100AA000C00FD11FD093F313C093F213BE01772769
:100AB00087E00E94FB59CC2321F081E08093DF0B7B
:100AC00002C01092DF0B10161106ECF58091EE13A8
:100AD0009091EF13C817D9070CF487C08091F413D5
:100AE000882371F01092EF131092EE138CEF9FEFAA
:100AF0009093F1138093F01381E08093ED1375C010
:100B000068E770E080E090E00E94EB55DC01CB01EB
:100B10000A96A11DB11D9093EF138093EE1368E226
:100B200070E080E090E00E94EB55DC01CB010A967A
:100B3000A11DB11D66277727681B790B7093F113F0
:100B40006093F01352C0012B09F44FC08091EE1353
:100B50009091EF138C179D070CF447C08091ED1313
:100B6000882321F10091F5131091F613C0911B0712
:100B7000D0911C07B801CE010E94734D8823A9F1C2
:100B8000B801CE010E948B4D0E9487831092F3130F
:100B90001092F2131092ED1380918A11882329F19B
:100BA000DF91CF911F910F910C94B58469E670E0AD
:100BB00080E090E00E94EB55DC01CB018A569F4F0C
:100BC000AF4FBF4F9093EF138093EE1368E270E046
:100BD00080E090E00E94EB55DC01CB010A96A11D5C
:100BE000B11D9093F1138093F013DF91CF911F917A
:100BF0000F91089560E088E00C948F5961E089E2DC
:100C00000C948F590F931F93CF93DF9360E08BE287
:100C10000E948F590091EB131091EC13C0911B07A8
:100C2000D0911C07B801CE010E94734D882341F07A
:100C3000B801CE01DF91CF911F910F910C948B4D94
:100C4000DF91CF911F910F910895809137078823ED
:100C500069F08091E10B882349F081E08093DE0BFD
:100C6000809136070E94986D0C9446830895CF9327
:100C7000DF93CDB7DEB765970FB6F894DEBF0FBE32
:100C8000CDBF81E08093E20B8091E813882371F15E
:100C900082E390E09A83898388E290E09C838B834F
:100CA0008EE690E09E838D8384EF91E098878F831A
:100CB0001D8A84E08F938DB79EB745970FB6F89441
:100CC0009EBF0FBE8DBFADB7BEB7119685E1FE01C9
:100CD000319601900D928A95E1F78CEE9AE00E9490
:100CE0005C480FB6F894DEBF0FBECDBF65960FB659
:100CF000F894DEBF0FBECDBFDF91CF91089586334C
:100D000008F0865390917B00282F2870977F922BB4
:100D100090937B008770806480937C0080917A0040
:100D2000806480937A0080917A0086FDFCCF809168
:100D300078002091790090E0922B08953FB7F894C5
:100D40008091081490910914A0910A14B0910B1489
:100D500026B5A89B05C02F3F19F00196A11DB11D16
:100D60003FBFBA2FA92F982F8827820F911DA11D51
:100D7000B11DBC01CD0142E0660F771F881F991F8E
:100D80004A95D1F708958F929F92AF92BF92CF92DA
:100D9000DF92EF92FF926B017C010E949E864B01D5
:100DA0005C01C114D104E104F104F1F00E949E86BB
:100DB000DC01CB0188199909AA09BB09883E934037
:100DC000A105B10570F321E0C21AD108E108F108CC
:100DD00088EE880E83E0981EA11CB11CC114D104BA
:100DE000E104F10419F7DDCFFF90EF90DF90CF9091
:100DF000BF90AF909F908F9008952FB7F894609117
:100E000004147091051480910614909107142FBF5B
:100E100008951F920F920FB60F9211242F933F93B4
:100E20008F939F93AF93BF93809104149091051477
:100E3000A0910614B09107143091031423E0230FFE
:100E40002D3720F40196A11DB11D05C026E8230F02
:100E50000296A11DB11D2093031480930414909356
:100E60000514A0930614B093071480910814909170
:100E70000914A0910A14B0910B140196A11DB11D83
:100E80008093081490930914A0930A14B0930B1440
:100E9000BF91AF919F918F913F912F910F900FBE76
:100EA0000F901F9018950F931F93CF93DF9300918E
:100EB000FB131091FC13C0911B07D0911C07B801C4
:100EC000CE010E94734D8823A1F0B801CE010E948B
:100ED0008B4D27E733E848EB5BE060E070E0809102
:100EE0001B0790911C070E94DA4D9093FC1380938E
:100EF000FB136091F5137091F61380911B0790918D
:100F00001C070E94734D81114CC01092F4138FEF97
:100F100090E09093F3138093F2130E948E8368E71E
:100F200070E080E090E00E94EB55DC01CB010A9676
:100F3000A11DB11D9093EF138093EE1368E270E052
:100F400080E090E00E94EB55DC01CB010A96A11DE8
:100F5000B11D66277727681B790B7093F113609397
:100F6000F01324E435E844E150E060E070E0809163
:100F70001B0790911C070E94E34D9093F6138093FA
:100F8000F51327E733E848EB5BE060E070E0809121
:100F90001B0790911C070E94DA4D9093FC138093DD
:100FA000FB13DF91CF911F910F9108958F929F9224
:100FB000AF92BF92CF92EF92FF920F931F93CF9376
:100FC000DF9320913907223008F07AC07B018C0131
:100FD0008090240790902507A0902607B0902707BF
:100FE00020E030E0A901C501B4010E94F1CB181640
:100FF00054F520E030E0A901C501B4010E94BFCE44
:10100000181654F420E030E048E452E4C501B4017D
:101010000E94F1CB1816D4F420E030E048E452E40A
:10102000C501B4010E94BFCE18169CF420E030E048
:1010300048EC52E4C501B4010E94F1CB87FF09C01E
:10104000CBE4D0E008C0C0E0D0E005C0C2E3D0E00F
:1010500002C0C4E6D0E08FEF8C0D823070F4209790
:1010600039F06C2FC8010E94D78E6C2FC7010DC0BC
:10107000C8010E94D477C70116C08DEF8C0D833054
:10108000F8F4209779F06C2FC801DF91CF911F9170
:101090000F91FF90EF90CF90BF90AF909F908F9067
:1010A0000C94D78EC801DF91CF911F910F91FF90C3
:1010B000EF90CF90BF90AF909F908F900C94D4778B
:1010C000DF91CF911F910F91FF90EF90CF90BF9044
:1010D000AF909F908F9008958F929F92AF92BF9202
:1010E000CF92DF92EF92FF92C0902407D090250715
:1010F000E0902607F090270720E030E0A901C70123
:10110000B6010E94BFCE20E030E040E05FE387FD03
:101110000BC0C701B6010E94ABCD4B015C010E9420
:1011200089CE97FD27C010C0C701B6010E94AACD85
:101130000E9489CE97FD1EC0653671058105910517
:10114000DCF424E6822F14C0C501B4010E9489CECC
:1011500065367105810591057CF420E030E040E0C2
:101160005FE3C701B6010E94ABCD0E9489CE84E641
:10117000861B03C084E601C080E0FF90EF90DF9003
:10118000CF90BF90AF909F908F9008950F931F9333
:10119000CF93DF930091140710911507C0911B079F
:1011A000D0911C07B801CE010E94734D882321F015
:1011B000B801CE010E948B4D8091E00B882341F055
:1011C0001092E00BDF91CF911F910F910C94098445
:1011D000DF91CF911F910F910895EC981092E10B40
:1011E00068EC70E082E00C94CC6C80913207811145
:1011F00006C080913607811102C00C94ED88809161
:10120000DC0B9091DD0B0E94C2A181E08093E10B89
:1012100064E670E00C94CC6C60E089E20E948F5927
:101220002EEF35E842E350E060E070E080911B076C
:1012300090911C070C94DA4D1F920F920FB60F92EB
:1012400011240BB60F922F933F934F935F936F939D
:101250007F938F939F93AF93BF93EF93FF9380916F
:10126000EA138823B1F048991FC0E89822E036E8D5
:101270004CE251E060E070E080911B0790911C0708
:101280000E94DA4D8091E913882371F00E94C5977E
:101290000BC061E070E080E090E00E94C386489B54
:1012A00003C0E8980E940286FF91EF91BF91AF9131
:1012B0009F918F917F916F915F914F913F912F916E
:1012C0000F900BBE0F900FBE0F901F90189561E00E
:1012D0008BE20E948F59E89A22E036E848E853E111
:1012E00060E070E080911B0790911C070E94DA4D2E
:1012F0009093EC138093EB13089561E08BE20E94CE
:101300008F59E89A22E036E848E853E160E070E05F
:1013100080911B0790911C070E94DA4D9093EC136B
:101320008093EB1308951092E20B40912C0750919B
:101330002D0760E070E027E336E880911B0790916D
:101340001C070C94DA4D80914E1490914F148068D4
:1013500090934F1480934E14089580914E14909161
:101360004F14806190934F1480934E140895FC01A4
:101370008281882371F08381882359F013828091C0
:101380004E1490914F1424E0822790934F14809331
:101390004E140895FC018281882371F083818111AC
:1013A0000BC081E0838380914E1490914F14846030
:1013B00090934F1480934E140895FC0184818823E8
:1013C00071F08581882359F0158280914E14909197
:1013D0004F1428E0822790934F1480934E14089561
:1013E000FC018481882371F0858181110BC081E02B
:1013F000858380914E1490914F14886090934F1480
:1014000080934E14089580914E1490914F1420E2D1
:10141000822790934F1480934E14089580914E1418
:1014200090914F14806290934F1480934E140895BE
:10143000DC01ED91FC910680F781E02D60E070E029
:10144000199477FF03C07195619571096F3F71051C
:1014500019F014F06FEF70E080914E1490914F14DA
:101460008C7B917090934F1480934E1480914E1406
:1014700090914F146F30710514F480641FC067336E
:10148000710514F481641AC06F3571051CF4816410
:10149000906114C0673871051CF4816490630EC0BC
:1014A0006F3A71051CF48164906408C0673D710552
:1014B0001CF48164906502C08164906690934F141F
:1014C00080934E14089580E094E090934F1480939D
:1014D0004E14089580914E1490914F149260909301
:1014E0004F1480934E140895089508950895089513
:1014F00008950895089508950895089580E0089541
:1015000008950895089508950895089508950895F3
:1015100008950895089508950895089508950895E3
:10152000089508950895089580E008950895089510
:101530000895FC0164830895FC0162830895FC0111
:1015400013821482158216821782108611860895DE
:10155000089508950895FC0183810895FC01658331
:101560000895FC0164830895FC0160870895FC01DF
:1015700066830895FC0182810895FC011282138222
:101580001482158261E086E10E94BF5961E086E124
:101590000E948F59E2E7F0E08081816080831092A1
:1015A0004F1410924E140895FF920F931F93CF93F0
:1015B000DF938C01C62FF42ED22F6AED70E0DC0190
:1015C0001A968D919C911B970E940583F801828544
:1015D0009385DC01ED91FC910190F081E02D6C2F61
:1015E0001995F80182859385DC01ED91FC910190BC
:1015F000F081E02D6F2D1995F80182859385DC012E
:10160000ED91FC910190F081E02D6D2F1995EC2F5B
:10161000F0E0BF0166527F4F6F0D711D6D0F711DA0
:101620006F777727F80182859385DF91CF911F919E
:101630000F91FF900C94058320E040E00C94D48A35
:1016400065E40C941C8B68E40C941C8BCF93DF93A3
:10165000FC012381222329F0EC0161E40E941C8B10
:101660001B82DF91CF910895CF93DF93FC012381FB
:10167000211106C0EC0160E40E941C8B81E08B8389
:10168000DF91CF91089563E50C941C8BFC012581BB
:10169000222319F060E50C941C8B0895FC01248131
:1016A000222319F06CE30C941C8B0895FC01208517
:1016B000222339F02185222321F011866BE30C943B
:1016C0001C8B0895FC012085222341F021852111E6
:1016D00005C021E021876AE30C941C8B0895FC016E
:1016E0002681222339F02781222321F0178269E302
:1016F0000C941C8B0895FC012681222341F0278144
:10170000211105C021E0278368E30C941C8B089508
:1017100067E30C941C8B6AE40C941C8B69E40C94B6
:101720001C8B66E30C941C8B65E30C941C8B6EE4A1
:101730000C941C8B64E30C941C8B63E30C941C8B47
:1017400062E30C941C8B61E30C941C8B60E30C949F
:101750001C8B64E50C941C8B6FE20C941C8B6DE26B
:101760000C941C8B6CE20C941C8B242F462F6CE485
:101770000C94D48A77FF03C071956195710920E0BC
:10178000462F6EE20C94D48A462F20E067E40C9436
:10179000D48A462F20E066E40C94D48A262F64E491
:1017A0000C94D48ACF92DF92FF920F931F93CF9322
:1017B000DF938C01F62E443F81E0580738F0413129
:1017C00087E2580728F040E157E202C044EF51E0B9
:1017D000243F81E0380738F0E9012131374228F011
:1017E000C0E1D7E202C0C4EFD1E0CA01845F9140FA
:1017F00022E3C22ED12CB6010E9469CF462F2F2D95
:1018000062E4C8010E94D48ACE01845F9140B6018F
:101810000E9469CF462F2F2D63E4C801DF91CF913D
:101820001F910F91FF90DF90CF900C94D48A242FBA
:10183000462F62E50C94D48A242F462F61E50C9440
:10184000D48A262F40E06FE30C94D48A262F40E000
:101850006EE30C94D48A262F40E06DE30C94D48A76
:10186000462F20E06FE40C94D48A462F20E06DE4EC
:101870000C94D48AFC016283611105C020E040E031
:101880006BE40C94D48A089577FF03C07195619539
:10189000710920E0462F6BE40C94D48A1F920F92BA
:1018A0000FB60F9211240BB60F920F931F932F9325
:1018B0003F934F935F936F937F938F939F93AF93D8
:1018C000BF93EF93FF93809114148F5F8093141450
:1018D00090911314891708F42FC110921414809159
:1018E000121490E08730910508F026C1FC0188278A
:1018F000E155FE4F8F4F0C9491CF60E086E10E943E
:101900008F5980E48093131481E048C061E086E140
:101910000E948F5988E08093131436C060E086E1FE
:101920000E948F59809110149091111497FF05C057
:1019300088E18093131484E031C088E0809313140D
:1019400083E02CC061E086E10E948F5988E180939A
:10195000131480910F148F5F80930F14803150F017
:1019600010920F1485E01AC061E086E10E948F5941
:1019700088E0EDCF8091101490911114880F991F79
:10198000909311148093101482E008C060E086E107
:101990000E948F5988E08093131486E0809312147C
:1019A000CBC061E086E10E948F5980EC80931314D4
:1019B00080914E1490914F149093111480931014B1
:1019C00080914E1490914F1491FF1CC080910E1481
:1019D000882369F080914E1490914F1422E0922751
:1019E00090934F1480934E1410920E140BC081E00C
:1019F00080930E1480930D1480930C1486E69BE064
:101A00000E94BF6C80910C148823D1F080910D143A
:101A10008823B1F00E94FD860091660B1091670B40
:101A20002091680B3091690BDC01CB01801B910B7D
:101A3000A20BB30B8D369042A105B10508F070C022
:101A400080914E1490914F1492FF12C080910E1409
:101A5000882339F010924F1410924E1410920E14E5
:101A600007C081E080930E1410920D1410920C1494
:101A700080914E1490914F1484FF14C080910E14E5
:101A8000882369F080914E1490914F1420E18227B1
:101A900090934F1480934E1410920E1403C081E063
:101AA00080930E1480914E1490914F1487FF13C0B1
:101AB00080910E14882361F080914E1490914F1400
:101AC000805890934F1480934E1410920E1403C0BC
:101AD00081E080930E1480914E1490914F1490FFEA
:101AE00014C080910E14882369F080914E14909157
:101AF0004F1421E0922790934F1480934E1410922C
:101B00000E1403C081E080930E1480914E149091C6
:101B10004F149093111480931014109212140CC04F
:101B200010920C1480914E1490914F1480649093F5
:101B30004F1480934E1484CFFF91EF91BF91AF91DA
:101B40009F918F917F916F915F914F913F912F91D5
:101B50001F910F910F900BBE0F900FBE0F901F9013
:101B6000189508950895089508951092DA0B089530
:101B70000F931F93CF93DF93EC011F8A1E8A8C0172
:101B8000075E1F4F40E060E0C8010E94575140E0EF
:101B900064E0C8010E9457510E94FD866C8F7D8FC2
:101BA0008E8F9F8FDF91CF911F910F9108950F938B
:101BB0001F93CF93DF93EC0180911514811112C014
:101BC0000A8D1B8D6AEA70E0C8010E940583D80166
:101BD000ED91FC910680F781E02DC801199581E017
:101BE000809315144AE06EE0CE0149960E94575149
:101BF00021E83FEF3B872A878FE790E09D878C871E
:101C00001F861E86398B288B9B8B8A8B1D8A1C8A8C
